 archba

 Timestamp is 5e5e5809 (Tue Mar  3 05:13:45 2020)

 Preferred load address is 0000000140000000

 Start         Length     Name                   Class
 0001:00000000 0001f290H .text$mn                CODE
 0001:0001f290 00000030H .text$mn$00             CODE
 0001:0001f2c0 00000430H .text$mn$21             CODE
 0001:0001f6f0 00009858H .text$s                 CODE
 0002:00000000 000000c0H .idata$5                DATA
 0002:000000c0 00000010H .00cfg                  DATA
 0002:000000d0 000000b0H .gfids                  DATA
 0002:00000174 00000000H .gfids$y                DATA
 0002:00000180 000002f8H .rdata                  DATA
 0002:00000478 000001b0H .rdata$zzzdbg           DATA
 0002:00000628 00001574H .xdata                  DATA
 0003:00000000 00000aa0H .data                   DATA
 0003:00000aa0 00000338H .bss                    DATA
 0004:00000000 00000c9cH .pdata                  DATA
 0005:00000000 0000005cH INIT                    CODE
 0005:0000005c 0000003cH .idata$2                CODE
 0005:00000098 00000018H .idata$3                CODE
 0005:000000b0 000000c0H .idata$4                CODE
 0005:00000170 00000228H .idata$6                CODE
 0006:00000000 000000d0H .rsrc$01                DATA
 0006:000000d0 00001108H .rsrc$02                DATA

  Address         Publics by Value              Rva+Base               Lib:Object

 0000:00000000       __enclave_config           0000000000000000     <absolute>
 0000:00000000       __dynamic_value_reloc_table 0000000000000000     <absolute>
 0000:00000000       __guard_longjmp_table      0000000000000000     <absolute>
 0000:00000000       __guard_longjmp_count      0000000000000000     <absolute>
 0000:00000000       ___safe_se_handler_table   0000000000000000     <absolute>
 0000:00000000       __hybrid_code_map_count    0000000000000000     <absolute>
 0000:00000000       __guard_iat_table          0000000000000000     <absolute>
 0000:00000000       __hybrid_code_map          0000000000000000     <absolute>
 0000:00000000       __guard_iat_count          0000000000000000     <absolute>
 0000:00000000       __hybrid_auxiliary_iat     0000000000000000     <absolute>
 0000:00000000       __volatile_metadata        0000000000000000     <absolute>
 0000:00000000       ___safe_se_handler_count   0000000000000000     <absolute>
 0000:00000029       __guard_fids_count         0000000000000029     <absolute>
 0000:00014500       __guard_flags              0000000000014500     <absolute>
 0000:00000000       __ImageBase                0000000140000000     <linker-defined>
 0001:00000000       DumpHandles                0000000140001000 f   rxdevice.obj
 0001:000003b0       DumpHandlesZeroPointer     00000001400013b0 f   rxdevice.obj
 0001:00000760       GetOutstandingIoCnt        0000000140001760 f   rxdevice.obj
 0001:00000770       NonMSIXInterruptHandler    0000000140001770 f   rxdevice.obj
 0001:00000b50       PMCDpcResponseHandler      0000000140001b50 f   rxdevice.obj
 0001:000012f0       PMCInterruptHandler        00000001400022f0 f   rxdevice.obj
 0001:000018f0       PMCPushMessageUnitQueueFib 00000001400028f0 f   rxdevice.obj
 0001:00001c10       RxAccessDeviceRegister     0000000140002c10 f   rxdevice.obj
 0001:00001db0       RxCheckAdapterHealth       0000000140002db0 f   rxdevice.obj
 0001:00001e20       RxCheckSyncCommandComplete 0000000140002e20 f   rxdevice.obj
 0001:00001f60       RxDpcInterruptHandler      0000000140002f60 f   rxdevice.obj
 0001:00001f60       _guard_check_icall_nop     0000000140002f60 f   BufferOverflowFastFailK:guard_support.obj
 0001:00001f70       RxGetIBW                   0000000140002f70 f   rxdevice.obj
 0001:00001fa0       RxGetOMRx0                 0000000140002fa0 f   rxdevice.obj
 0001:00001fd0       RxInterruptHandler         0000000140002fd0 f   rxdevice.obj
 0001:000022a0       RxMapMailBoxFirmwareBase   00000001400032a0 f   rxdevice.obj
 0001:00002390       RxNewCommProcessInterrupt  0000000140003390 f   rxdevice.obj
 0001:00002760       RxNotifyAdapter            0000000140003760 f   rxdevice.obj
 0001:000027e0       RxPullMessageUnitQueueCompletedFib 00000001400037e0 f   rxdevice.obj
 0001:00002980       RxPushMessageUnitQueueFib  0000000140003980 f   rxdevice.obj
 0001:00002a70       RxSendSynchCommand         0000000140003a70 f   rxdevice.obj
 0001:00003690       RxStartAdapter             0000000140004690 f   rxdevice.obj
 0001:00003d10       RxWaitForAdapterToBoot     0000000140004d10 f   rxdevice.obj
 0001:00003e00       RxWriteIBW                 0000000140004e00 f   rxdevice.obj
 0001:00003e30       RxWriteIDR                 0000000140004e30 f   rxdevice.obj
 0001:00003e60       RxWriteODR                 0000000140004e60 f   rxdevice.obj
 0001:00003ea0       RevCheckCompatibility      0000000140004ea0 f   revision.obj
 0001:00003f40       RevGetBuildNumber          0000000140004f40 f   revision.obj
 0001:00003f50       RevGetExternalRev          0000000140004f50 f   revision.obj
 0001:00003f60       CompareStrings             0000000140004f60 f   helpers.obj
 0001:00003fe0       GetDriverParameter         0000000140004fe0 f   helpers.obj
 0001:00004120       LongToAscii                0000000140005120 f   helpers.obj
 0001:000041f0       MatchRegistryString        00000001400051f0 f   helpers.obj
 0001:000042b0       ZeroStructure              00000001400052b0 f   helpers.obj
 0001:000042c0       ArcPrintf                  00000001400052c0 f   arcdebug.obj
 0001:000047d0       ProcessCompleteSrbToHost   00000001400057d0 f   arcdebug.obj
 0001:000047e0       RealSprintf                00000001400057e0 f   arcdebug.obj
 0001:00004c90       StorWmiTraceMessage        0000000140005c90 f i arcdebug.obj
 0001:00004cf0       WPP_SF_s                   0000000140005cf0 f i arcdebug.obj
 0001:00004d50       CheckingFWAfterPowerStateChange 0000000140005d50 f   timer.obj
 0001:00005140       MainTimeThread             0000000140006140 f   timer.obj
 0001:00005cf0       RequestTimer               0000000140006cf0 f   timer.obj
 0001:00005dc0       Reset_IOP_CompletionTimer  0000000140006dc0 f   timer.obj
 0001:00006290       StopTimer                  0000000140007290 f   timer.obj
 0001:00006330       UpdateThorHBAMappingTable  0000000140007330 f   timer.obj
 0001:00006610       VMCloseAllCompletionTimer  0000000140007610 f   timer.obj
 0001:00006860       AllocateConsumerProducerCommArea 0000000140007860 f   arcinit.obj
 0001:00006bb0       AllocateMessageUnitQueueCommArea 0000000140007bb0 f   arcinit.obj
 0001:00007160       ArcLogEventString          0000000140008160 f   arcinit.obj
 0001:000071e0       AtomicINTXReleaseSlot      00000001400081e0 f   arcinit.obj
 0001:00007200       CheckMSIxPossibility       0000000140008200 f   arcinit.obj
 0001:00007410       CleanHostSideRRQ           0000000140008410 f   arcinit.obj
 0001:00007630       ConfigureContainersRuntime 0000000140008630 f   arcinit.obj
 0001:00008f60       DecToHex                   0000000140009f60 f   arcinit.obj
 0001:00008fc0       DriverEntry                0000000140009fc0 f   arcinit.obj
 0001:000091e0       DumpFibsSentToFW60SecondsBefore 000000014000a1e0 f   arcinit.obj
 0001:000094c0       DynamicallyThrottleLunQueueDepth 000000014000a4c0 f   arcinit.obj
 0001:00009740       EventTracingCleanup        000000014000a740 f   arcinit.obj
 0001:000097c0       FindAdapter                000000014000a7c0 f   arcinit.obj
 0001:0000c180       GetElapsedSeconds          000000014000d180 f   arcinit.obj
 0001:0000c210       GetFreeSlot                000000014000d210 f   arcinit.obj
 0001:0000c240       GetThorHbaPhyDevInfo       000000014000d240 f   arcinit.obj
 0001:0000c790       HWSoftReset                000000014000d790 f   arcinit.obj
 0001:0000c8f0       HandleAdapterCommitConfig  000000014000d8f0 f   arcinit.obj
 0001:0000c9c0       HandleAdapterConfigIssues  000000014000d9c0 f   arcinit.obj
 0001:0000cb90       HandleAdapterGetConfig     000000014000db90 f   arcinit.obj
 0001:0000cca0       HwInitializeAdapter        000000014000dca0 f   arcinit.obj
 0001:0000d0f0       INTXGetFreeSlot            000000014000e0f0 f   arcinit.obj
 0001:0000d110       IOPReset                   000000014000e110 f   arcinit.obj
 0001:0000d660       InitializeConsumerProducerCommRegion 000000014000e660 f   arcinit.obj
 0001:0000d8f0       InitializeDPCs             000000014000e8f0 f   arcinit.obj
 0001:0000e020       IsAdapterReadyForConfigCommand 000000014000f020 f   arcinit.obj
 0001:0000e150       LogSystemEvent             000000014000f150 f   arcinit.obj
 0001:0000e230       MapDeviceBase              000000014000f230 f   arcinit.obj
 0001:0000e7b0       ReleaseSlot                000000014000f7b0 f   arcinit.obj
 0001:0000e7e0       ResetAdapter               000000014000f7e0 f   arcinit.obj
 0001:0000eef0       ReturnOutstandingFibOnTargetDevice 000000014000fef0 f   arcinit.obj
 0001:0000f0a0       ReturningLocalOutstandingRequestsToOS 00000001400100a0 f   arcinit.obj
 0001:0000f360       ReturningOutstandingSentToFWBeforeIOPResetToOS 0000000140010360 f   arcinit.obj
 0001:0000f510       SA4ACI2Interface           0000000140010510 f   arcinit.obj
 0001:0000f6a0       SA4StatusBatching          00000001400106a0 f   arcinit.obj
 0001:0000f830       SMCrashDumpModeInitAdapter 0000000140010830 f   arcinit.obj
 0001:0000fad0       SMNormalModeInitAdapter    0000000140010ad0 f   arcinit.obj
 0001:0000ffa0       SendEvent2OS               0000000140010fa0 f   arcinit.obj
 0001:00010930       SendEvent2OSChild          0000000140011930 f   arcinit.obj
 0001:00010dc0       SendEvent2OSDelayed        0000000140011dc0 f   arcinit.obj
 0001:00011510       SendInitStructure          0000000140012510 f   arcinit.obj
 0001:000118e0       SendWellnessCmnd           00000001400128e0 f   arcinit.obj
 0001:00011ae0       SetArcsasFwTime            0000000140012ae0 f   arcinit.obj
 0001:00011bc0       SetFwTime                  0000000140012bc0 f   arcinit.obj
 0001:00012050       SetPciSlotNumber           0000000140013050 f   arcinit.obj
 0001:00012130       WppTraceCallback           0000000140013130 f   arcinit.obj
 0001:00012410       CompleteQueuedRequest      0000000140013410 f   cmddelivery.obj
 0001:00012510       DequeueCertainLD           0000000140013510 f   cmddelivery.obj
 0001:000125c0       DequeueRawIoReadWriteRequest 00000001400135c0 f   cmddelivery.obj
 0001:000126f0       HandleInterrupt            00000001400136f0 f   cmddelivery.obj
 0001:00012710       HandleMSIXInterrupt        0000000140013710 f   cmddelivery.obj
 0001:000127f0       PollSmartHBAFIBCompletion  00000001400137f0 f   cmddelivery.obj
 0001:00012b90       PostProcessScsiCommand     0000000140013b90 f   cmddelivery.obj
 0001:00012ee0       ProcessContainerInquiry    0000000140013ee0 f   cmddelivery.obj
 0001:000134b0       ProcessScsiCommand         00000001400144b0 f   cmddelivery.obj
 0001:00014110       QueuePrintf                0000000140015110 f   cmddelivery.obj
 0001:000141d0       QueueRawIoReadWriteRequest 00000001400151d0 f   cmddelivery.obj
 0001:00014470       SaveNFHandle               0000000140015470 f   cmddelivery.obj
 0001:000144b0       SendFib                    00000001400154b0 f   cmddelivery.obj
 0001:00014af0       SendRawIoFib               0000000140015af0 f   cmddelivery.obj
 0001:00014ce0       SendSynchFib               0000000140015ce0 f   cmddelivery.obj
 0001:00014ee0       StartIo                    0000000140015ee0 f   cmddelivery.obj
 0001:00015940       AdapterControl             0000000140016940 f   cmdproc.obj
 0001:00016070       BuildHBAFib                0000000140017070 f   cmdproc.obj
 0001:00016560       BuildHBAIoctlFib           0000000140017560 f   cmdproc.obj
 0001:00016810       BuildIo                    0000000140017810 f   cmdproc.obj
 0001:000173e0       BuildRawIo2ScatterGather   00000001400183e0 f   cmdproc.obj
 0001:000175c0       BuildRawIo2ScatterGather4HBAIoctl 00000001400185c0 f   cmdproc.obj
 0001:00017790       BuildRawIoFib              0000000140018790 f   cmdproc.obj
 0001:00017af0       BuildRawIoScatterGather    0000000140018af0 f   cmdproc.obj
 0001:00017ce0       BuildReadWriteFib          0000000140018ce0 f   cmdproc.obj
 0001:000180b0       BuildScatterGather         00000001400190b0 f   cmdproc.obj
 0001:00018160       BuildScatterGather64       0000000140019160 f   cmdproc.obj
 0001:00018220       BuildSrbFib                0000000140019220 f   cmdproc.obj
 0001:000184c0       ConvertRawIo2ScatterGather 00000001400194c0 f   cmdproc.obj
 0001:00018600       InitializeFib              0000000140019600 f   cmdproc.obj
 0001:00018630       PrepareBMIC15              0000000140019630 f   cmdproc.obj
 0001:00018870       BuildRawScatterGather      0000000140019870 f   ioctl.obj
 0001:00018920       BuildRawScatterGather64    0000000140019920 f   ioctl.obj
 0001:000189d0       CSMIGetRAIDConfig          00000001400199d0 f   ioctl.obj
 0001:00018c40       CSMIGetRAIDInfo            0000000140019c40 f   ioctl.obj
 0001:00019100       CSMISTPPassThru            000000014001a100 f   ioctl.obj
 0001:000193a0       HandleCSMI                 000000014001a3a0 f   ioctl.obj
 0001:000199a0       ProcessIoctl               000000014001a9a0 f   ioctl.obj
 0001:0001c290       AdapterIsAlive             000000014001d290 f   comm.obj
 0001:0001c2d0       CompleteBufferedRequest    000000014001d2d0 f   comm.obj
 0001:0001c390       DpcDequeueRawIoReadWriteRequest 000000014001d390 f   comm.obj
 0001:0001c400       FreeConsumerProducerAif    000000014001d400 f   comm.obj
 0001:0001c550       GetConsumerProducerCompletedFib 000000014001d550 f   comm.obj
 0001:0001c5e0       GetMessageUnitQueueCompletedFib 000000014001d5e0 f   comm.obj
 0001:0001c600       ProcessAif                 000000014001d600 f   comm.obj
 0001:0001cf30       ProcessHbaErrors           000000014001df30 f   comm.obj
 0001:0001d540       ProcessNormalFib           000000014001e540 f   comm.obj
 0001:0001e060       QueueEvent                 000000014001f060 f   comm.obj
 0001:0001e100       SendConsumerProducerFib    000000014001f100 f   comm.obj
 0001:0001e200       SendMessageUnitQueueFib    000000014001f200 f   comm.obj
 0001:0001e270       ServiceHostCommandNormalQueue 000000014001f270 f   comm.obj
 0001:0001e360       ServiceHostResponseNormalQueue 000000014001f360 f   comm.obj
 0001:0001e780       ServiceInternalAifQueue    000000014001f780 f   comm.obj
 0001:0001e850       HwScsiWmiExecuteMethod     000000014001f850 f   wmi.obj
 0001:0001e8f0       HwScsiWmiFunctionControl   000000014001f8f0 f   wmi.obj
 0001:0001e8f0       HwScsiWmiQueryDataBlock    000000014001f8f0 f   wmi.obj
 0001:0001e910       HwScsiWmiQueryReginfo      000000014001f910 f   wmi.obj
 0001:0001e920       HwScsiWmiSetDataItem       000000014001f920 f   wmi.obj
 0001:0001e920       HwScsiWmiSetDataBlock      000000014001f920 f   wmi.obj
 0001:0001e930       InitializeWmiInterface     000000014001f930 f   wmi.obj
 0001:0001ea40       ProcessWmi                 000000014001fa40 f   wmi.obj
 0001:0001ead0       __security_check_cookie    000000014001fad0 f   BufferOverflowFastFailK:amdsecgs.obj
 0001:0001eaf0       __report_gsfailure         000000014001faf0 f   BufferOverflowFastFailK:gs_report.obj
 0001:0001eaf8       __report_rangecheckfailure 000000014001faf8 f   BufferOverflowFastFailK:gs_report.obj
 0001:0001eb00       __GSHandlerCheck           000000014001fb00 f   ntoskrnl:gshandler.obj
 0001:0001eb20       __GSHandlerCheckCommon     000000014001fb20 f   ntoskrnl:gshandler.obj
 0001:0001eb80       ExSystemTimeToLocalTime    000000014001fb80 f   ntoskrnl:ntoskrnl.exe
 0001:0001eb86       RtlTimeToTimeFields        000000014001fb86 f   ntoskrnl:ntoskrnl.exe
 0001:0001eb8c       KeQueryPerformanceCounter  000000014001fb8c f   hal:HAL.dll
 0001:0001eb94       ScsiPortWmiDispatchFunction 000000014001fb94 f   scsiwmi:wmilib.obj
 0001:0001ec34       ScsiPortWmiPostProcess     000000014001fc34 f   scsiwmi:wmilib.obj
 0001:0001ec70       ScsiWmipFindGuid           000000014001fc70 f   scsiwmi:wmilib.obj
 0001:0001ecd0       ScsiWmipPostProcess        000000014001fcd0 f   scsiwmi:wmilib.obj
 0001:0001ee20       ScsiWmipProcessRequest     000000014001fe20 f   scsiwmi:wmilib.obj
 0001:0001f2a0       _guard_dispatch_icall_nop  00000001400202a0 f   BufferOverflowFastFailK:guard_dispatch.obj
 0001:0001f2c0       memmove                    00000001400202c0 f   ntoskrnl:memcpy.obj
 0001:0001f2c0       memcpy                     00000001400202c0 f   ntoskrnl:memcpy.obj
 0001:0001f600       memset                     0000000140020600 f   ntoskrnl:memset.obj
 0001:0001f6f0       ??_C@_0CJ@KAGJNHLI@OMR?5value?5in?5Check?5Adapter?5Heal@FNODOBFM@ 00000001400206f0     rxdevice.obj
 0001:0001f720       ??_C@_0DE@IHDJGLJF@This?5should?5not?5happen?4?5We?5only@FNODOBFM@ 0000000140020720     rxdevice.obj
 0001:0001f760       ??_C@_0CP@PEAJGKJE@?$CK?5NonMSIXInterruptHandle?3?5pFibC@FNODOBFM@ 0000000140020760     rxdevice.obj
 0001:0001f790       ??_C@_0EM@CCDNION@?$CK?5Start?5a?5timer?5to?5update?5conta@FNODOBFM@ 0000000140020790     rxdevice.obj
 0001:0001f7e0       ??_C@_0DL@ELHJEKAJ@?$CK?57?124?3?5pFibContext?$DNNULL?5?$CB?$CBline@FNODOBFM@ 00000001400207e0     rxdevice.obj
 0001:0001f820       ??_C@_0DA@IEDLNFHE@?$CK?55?124?3?5?9VectorIndex?9?5?$CB?$CBline?5?$CFd@FNODOBFM@ 0000000140020820     rxdevice.obj
 0001:0001f850       ??_C@_0CN@FKDOCGDJ@?$CK?55?124?3?5OutStanding?5IO?5?$CB?$CBline?5?$CF@FNODOBFM@ 0000000140020850     rxdevice.obj
 0001:0001f880       ??_C@_0CD@PAEIGALF@?$CK?57?124?3?5?$CB?$CBline?5?$CFd?5?$CIhandle?5?9?51?$CJ?5@FNODOBFM@ 0000000140020880     rxdevice.obj
 0001:0001f8b0       ??_C@_0ED@DAJFCMJP@?$CK?5Start?5a?5timer?5to?5update?5Conta@FNODOBFM@ 00000001400208b0     rxdevice.obj
 0001:0001f900       ??_C@_0DK@JKKKPJCO@Dumping?5Normal?5Fib?5handles?0?5?5pD@FNODOBFM@ 0000000140020900     rxdevice.obj
 0001:0001f940       ??_C@_0DG@FEIEMBNE@?$CFd?3?5?$CFd?5?$CFd?5?$CFd?5?$CFd?5?$CFd?5?$CFd?5?$CFd?5?$CFd?5?$CFd?5@FNODOBFM@ 0000000140020940     rxdevice.obj
 0001:0001f980       ??_C@_0GP@CPJOGFCD@Dumping?5Free?5handle?5list?0?5?5pDev@FNODOBFM@ 0000000140020980     rxdevice.obj
 0001:0001f9f0       ??_C@_0DN@IDNOKJK@ZP?5Dumping?5Normal?5Fib?5handles?0?5@FNODOBFM@ 00000001400209f0     rxdevice.obj
 0001:0001fa30       ??_C@_0DJ@BENIEDOK@ZP?5?$CFd?3?5?$CFd?5?$CFd?5?$CFd?5?$CFd?5?$CFd?5?$CFd?5?$CFd?5?$CFd?5@FNODOBFM@ 0000000140020a30     rxdevice.obj
 0001:0001fa70       ??_C@_0HC@OLAIGIPB@ZP?5Dumping?5Free?5handle?5list?0?5?5p@FNODOBFM@ 0000000140020a70     rxdevice.obj
 0001:0001faf0       ??_C@_0CG@KADALDIK@?$CK?5?$CFd?5call?5of?5CheckForDupHandles@FNODOBFM@ 0000000140020af0     rxdevice.obj
 0001:0001fb20       ??_C@_0EK@CPNBBJGG@?$CK?5duplicated?5handle?5found?5?$CFd?4?5?$CF@FNODOBFM@ 0000000140020b20     rxdevice.obj
 0001:0001fb70       ??_C@_0BP@BKKLPPMO@pFibContext?$DNNULL?5?$CB?$CB?5Handle?5?$CFd?6@FNODOBFM@ 0000000140020b70     rxdevice.obj
 0001:0001fb90       ??_C@_0EI@DKKBIMEF@?$CK?5Start?5a?5timer?5to?5update?5conta@FNODOBFM@ 0000000140020b90     rxdevice.obj
 0001:0001fbe0       ??_C@_0FE@JLKFMCPA@?$CK?5PMCPushMessageUnitQueueFib?3?5C@FNODOBFM@ 0000000140020be0     rxdevice.obj
 0001:0001fc40       ??_C@_0FE@JICOMBJP@?$CK?5PMCPushMessageUnitQueueFib?3?5C@FNODOBFM@ 0000000140020c40     rxdevice.obj
 0001:0001fca0       ??_C@_0HN@JEPKAECC@?$CK?5RxSendSynchCommand?3?5Thor?5AIF?5@FNODOBFM@ 0000000140020ca0     rxdevice.obj
 0001:0001fd20       ??_C@_0EC@LAPIEKPJ@?$CK?5RxSendSynchCommand?3?5mailbox?$FL0@FNODOBFM@ 0000000140020d20     rxdevice.obj
 0001:0001fd70       ??_C@_0DJ@GJNDHOED@?$CK?5RxSendSynchCommand?3?5mailbox?$FL0@FNODOBFM@ 0000000140020d70     rxdevice.obj
 0001:0001fdb0       ??_C@_0HK@NJDHDGMI@?$CK?5RxSendSynchCommand?3?5There?5is?5@FNODOBFM@ 0000000140020db0     rxdevice.obj
 0001:0001fe30       ??_C@_0HB@PLCHFMAA@?$CK?5RxSendSynchCommand?3?5synch?5cmd@FNODOBFM@ 0000000140020e30     rxdevice.obj
 0001:0001feb0       ??_C@_0FD@ECFFGBJE@?5RxSendSynchCommand?3?5FW?5doing?5I@FNODOBFM@ 0000000140020eb0     rxdevice.obj
 0001:0001ff10       ??_C@_0FE@DOFCONDK@?$CK?5RxSendSynchCommand?3?5wait?5for?5@FNODOBFM@ 0000000140020f10     rxdevice.obj
 0001:0001ff70       ??_C@_0GF@LFEFAJKJ@?5RxSendSynchCommand?5?$CIcrash?5dump@FNODOBFM@ 0000000140020f70     rxdevice.obj
 0001:0001ffe0       ??_C@_0GF@CDCMENMG@?$CK?5RxSendSynchCommand?5?$CIcrash?5dum@FNODOBFM@ 0000000140020fe0     rxdevice.obj
 0001:00020050       ??_C@_0EL@HOIBIGPI@?$CK?5RxSendSynchCommand?3?5Got?5respo@FNODOBFM@ 0000000140021050     rxdevice.obj
 0001:000200a0       ??_C@_0EJ@DGPABBLG@?$CK?5RxSendSynchCommand?3?5Should?5NO@FNODOBFM@ 00000001400210a0     rxdevice.obj
 0001:000200f0       ??_C@_0FA@HKIBFKMH@?$CK?5RxSendSynchCommand?3?5Still?5NO?5@FNODOBFM@ 00000001400210f0     rxdevice.obj
 0001:00020140       ??_C@_0KI@HMCHOJIN@?5RxSendSynchCommand?$FLMSIX?5mode?$FN?5@FNODOBFM@ 0000000140021140     rxdevice.obj
 0001:000201f0       ??_C@_0JP@JKCHEOCJ@?5RxSendSynchCommand?$FLMSIX?5mode?$FN?3@FNODOBFM@ 00000001400211f0     rxdevice.obj
 0001:00020290       ??_C@_0CN@BCCBJMEA@?5RxSendSynchCommand?5Failed?5?$CFd?0w@FNODOBFM@ 0000000140021290     rxdevice.obj
 0001:000202c0       ??_C@_0DB@JEAHJGPL@?$CK?5pDeviceExtension?9?$DOMaxMSIXVect@FNODOBFM@ 00000001400212c0     rxdevice.obj
 0001:00020300       ??_C@_0CB@JPABDNKH@?$CK?5Begins?5StatusBatching?0?5Yeaaa?$CB@FNODOBFM@ 0000000140021300     rxdevice.obj
 0001:00020330       ??_C@_0CF@BPKEMKA@?$CK?5ACI2?5Command?5Delivery?5is?5enab@FNODOBFM@ 0000000140021330     rxdevice.obj
 0001:00020360       ??_C@_1DK@JBHFOPMP@?$AAA?$AAd?$AAa?$AAp?$AAt?$AAe?$AAr?$AA?5?$AAC?$AAo?$AAn?$AAf?$AAi?$AAg?$AAu@FNODOBFM@ 0000000140021360     rxdevice.obj
 0001:000203a0       ??_C@_04HIBGFPH@NULL@FNODOBFM@ 00000001400213a0     arcdebug.obj
 0001:000203b0       ??_C@_02DKCKIIND@?$CFs@FNODOBFM@ 00000001400213b0     arcdebug.obj
 0001:000203c0       ??_C@_06NBLAGFFP@Archba@FNODOBFM@ 00000001400213c0     arcdebug.obj
 0001:000203d0       ??_C@_0BC@JKBDDNDF@DelayNotification@FNODOBFM@ 00000001400213d0     timer.obj
 0001:000203f0       ??_C@_0CK@BKKGBKDP@?$CK?5Scan?5Notification?5sent?5in?5?$CFs?5@FNODOBFM@ 00000001400213f0     timer.obj
 0001:00020420       ??_C@_0GB@FAGGLJPH@?$CK?5First?58?5HBA?5devices?3?5?$CI0x?$CFx?0?$CFd@FNODOBFM@ 0000000140021420     timer.obj
 0001:00020490       ??_C@_0FN@EKAEFPGA@?$CK?5HBA?5mapping?5table?5updated?0?5ti@FNODOBFM@ 0000000140021490     timer.obj
 0001:000204f0       ??_C@_0GF@PMGNJLIM@?$CK?5Start?5a?5timer?5to?5update?5Conta@FNODOBFM@ 00000001400214f0     timer.obj
 0001:00020560       ??_C@_0CK@JLKEFPAM@entering?5CheckingFWAfterPowerSt@FNODOBFM@ 0000000140021560     timer.obj
 0001:00020590       ??_C@_0GN@GHJFFNOA@?$CK?5set?5timer?5AGAIN?5in?5CheckingFW@FNODOBFM@ 0000000140021590     timer.obj
 0001:00020600       ??_C@_0FK@MIIMDOAD@?$CK?5set?5timer?5AGAIN?5in?5CheckingFW@FNODOBFM@ 0000000140021600     timer.obj
 0001:00020660       ??_C@_0GB@EDFGCDFC@?$CK?5set?5timer?5AGAIN?5in?5CheckingFW@FNODOBFM@ 0000000140021660     timer.obj
 0001:000206d0       ??_C@_0N@BOCOJDCO@7?45?40?459002?$AA@FNODOBFM@ 00000001400216d0     timer.obj
 0001:000206e0       ??_C@_0DO@GCDGNMH@?$CK?5FW?5is?5back?5from?5S3?1S4?4?5StorPo@FNODOBFM@ 00000001400216e0     timer.obj
 0001:00020720       ??_C@_0DM@JABFAEPO@?$CK?5?9?5Reset?5AIFSrb?5to?5NULL?5when?5b@FNODOBFM@ 0000000140021720     timer.obj
 0001:00020760       ??_C@_0DN@ELHOMNDM@?$CK?5leaving?5CheckingFWAfterPowerS@FNODOBFM@ 0000000140021760     timer.obj
 0001:000207a0       ??_C@_0DO@OBELKDEH@?$CK?5set?5timer?5AGAIN?5to?5check?5the?5@FNODOBFM@ 00000001400217a0     timer.obj
 0001:000207e0       ??_C@_0CI@JPJEKICG@DPC?9Timeout?5may?5happen?5in?5Reset@FNODOBFM@ 00000001400217e0     timer.obj
 0001:00020810       ??_C@_0DH@JNGKJDAE@One?5kidnapped?5FIB?5released?$CB?5FIB@FNODOBFM@ 0000000140021810     timer.obj
 0001:00020850       ??_C@_0EJ@PCDGPKJP@?$CK?5Driver?5was?5not?5able?5to?5send?5?$CF@FNODOBFM@ 0000000140021850     timer.obj
 0001:000208a0       ??_C@_0DM@PNDEAHOI@?$CK?5Send?5BusChangeDetected?5to?5OS?5@FNODOBFM@ 00000001400218a0     timer.obj
 0001:000208e0       ??_C@_0EH@FCLGCKBJ@?$CK?5Start?5a?5timer?5to?5update?5HBA?5d@FNODOBFM@ 00000001400218e0     timer.obj
 0001:00020930       ??_C@_0GE@IFJDDHGE@?$CK?5Start?5a?5timer?5to?5update?5Conta@FNODOBFM@ 0000000140021930     timer.obj
 0001:000209a0       ??_C@_0DC@ODEFHEA@?$CK?5ConfigureContainersTimer?3?5Con@FNODOBFM@ 00000001400219a0     timer.obj
 0001:000209e0       ??_C@_0DL@DODBJONE@?$CK?5SynchCommandCompletionTimer?3?5@FNODOBFM@ 00000001400219e0     timer.obj
 0001:00020a20       ??_C@_0EO@CBNEAKKI@?$CK?5VMCloseAllCompletionTimer?3?5se@FNODOBFM@ 0000000140021a20     timer.obj
 0001:00020a70       ??_C@_0FI@MJCPBEAD@?$CK?5VMCloseAllCompletionTimer?3?5wa@FNODOBFM@ 0000000140021a70     timer.obj
 0001:00020ad0       ??_C@_0DO@ELMMCKMD@?$CK?5VMCloseAllCompletionTimer?3?5SR@FNODOBFM@ 0000000140021ad0     timer.obj
 0001:00020b10       ??_C@_0EH@BGEEAOIJ@?$CK?5VMCloseAllCompletionTimer?3?5Sh@FNODOBFM@ 0000000140021b10     timer.obj
 0001:00020b60       ??_C@_0EF@HLMPMNBN@?$CK?5VMCloseAllCompletionTimer?3?5Sy@FNODOBFM@ 0000000140021b60     timer.obj
 0001:00020bb0       ??_C@_0DH@IBACIAED@?$CK?5SynchFibCompletionTimer?3?5Sync@FNODOBFM@ 0000000140021bb0     timer.obj
 0001:00020bf0       ??_C@_0DP@OKLOLMOG@?5IBW_SWR?5register?5value?50?0?5rese@FNODOBFM@ 0000000140021bf0     timer.obj
 0001:00020c30       ??_C@_0CK@IHFMNBPG@?$CK?5IOP?5Reset?5TSR?3?5State?5Machine?5@FNODOBFM@ 0000000140021c30     timer.obj
 0001:00020c60       ??_C@_0DH@KAAGAFOD@?$CK?5leaving?5Reset_IOP_CompletionT@FNODOBFM@ 0000000140021c60     timer.obj
 0001:00020ca0       ??_C@_0CD@MKPFBJDC@leaving?5Reset_IOP_CompletionTim@FNODOBFM@ 0000000140021ca0     timer.obj
 0001:00020cd0       ??_C@_0DL@DOEFCINE@?$CK?5HW?5SOFT?5RESET?5done?4?5StorPort?5@FNODOBFM@ 0000000140021cd0     timer.obj
 0001:00020d10       ??_C@_0EA@DAIPACKH@?$CK?5RESET?5IOP?5done?5?$CFd?5times?4?5Stor@FNODOBFM@ 0000000140021d10     timer.obj
 0001:00020d50       ??_C@_0CJ@HBOEHNNB@Kernel?5Panic?5BlinkLed?5Code?5?$CFx?0?5@FNODOBFM@ 0000000140021d50     timer.obj
 0001:00020d80       ??_C@_0CK@CJGFOJPA@IOP_HWSOFT_RESET?3?5FW?5status?5?$CFx?0@FNODOBFM@ 0000000140021d80     timer.obj
 0001:00020db0       ??_C@_0BP@HJBLFCEF@?$CK?5PCIE?5reset?5issued?0?5line?5?$CD?$CFd?6@FNODOBFM@ 0000000140021db0     timer.obj
 0001:00020dd0       ??_C@_0DE@KOMJIKJE@?$CK?5set?5timer?5AGAIN?5to?5check?5the?5@FNODOBFM@ 0000000140021dd0     timer.obj
 0001:00020e10       ??_C@_0EF@BBNOBECH@?$CK?5set?5timer?5AGAIN?5to?5check?5the?5@FNODOBFM@ 0000000140021e10     timer.obj
 0001:00020e60       ??_C@_0EC@MICIKMJM@?$CK?5set?5timer?5AGAIN?5to?5check?5the?5@FNODOBFM@ 0000000140021e60     timer.obj
 0001:00020eb0       ??_C@_0DI@CMFOGNCK@?$CK?5RequestAif?3?5do?5not?5handle?5AIF@FNODOBFM@ 0000000140021eb0     timer.obj
 0001:00020ef0       ??_C@_0CL@MJMGCLDD@entering?5AllocateConsumerProduc@FNODOBFM@ 0000000140021ef0     arcinit.obj
 0001:00020f20       ??_C@_0DK@IJIOFPFH@leaving?5AllocateConsumerProduce@FNODOBFM@ 0000000140021f20     arcinit.obj
 0001:00020f60       ??_C@_0CI@FFOEPFMJ@?$CK?5ConsumerProducerCommArea?0?5VAd@FNODOBFM@ 0000000140021f60     arcinit.obj
 0001:00020f90       ??_C@_0CN@MBHLABKL@?$CK?5Adapter?5got?5an?5invalid?5host?5m@FNODOBFM@ 0000000140021f90     arcinit.obj
 0001:00020fc0       ??_C@_0DJ@JGKEIEFI@leaving?5AllocateConsumerProduce@FNODOBFM@ 0000000140021fc0     arcinit.obj
 0001:00021000       ??_C@_0CL@KCDMGIOM@entering?5AllocateMessageUnitQue@FNODOBFM@ 0000000140022000     arcinit.obj
 0001:00021030       ??_C@_0FP@JFBPKCDF@?$CK?5AllocateMessageUnitQueueCommA@FNODOBFM@ 0000000140022030     arcinit.obj
 0001:00021090       ??_C@_0DM@JMMHKBOC@?$CK?5AllocateMessageUnitQueueCommA@FNODOBFM@ 0000000140022090     arcinit.obj
 0001:000210d0       ??_C@_0DK@BKFHOPDI@leaving?5AllocateMessageUnitQueu@FNODOBFM@ 00000001400220d0     arcinit.obj
 0001:00021110       ??_C@_0DA@ICFHAOHF@?$CK?5AllocateMessageUnitQueueCommA@FNODOBFM@ 0000000140022110     arcinit.obj
 0001:00021140       ??_C@_0FB@FDJPGKAF@?$CK?5StorPortAllocateContiguousMem@FNODOBFM@ 0000000140022140     arcinit.obj
 0001:000211a0       ??_C@_0FB@MMEFOJJL@?$CK?5StorPortAllocateContiguousMem@FNODOBFM@ 00000001400221a0     arcinit.obj
 0001:00021200       ??_C@_0BJ@OICKMJHC@?$CK?5pBuf1?$DN0x?$CFp?0pBuf2?$DN0x?$CFp?6@FNODOBFM@ 0000000140022200     arcinit.obj
 0001:00021220       ??_C@_0BO@DPONBFMO@?$CK?5MemoryPhysicalAddress?$DN0x?$CFp?6@FNODOBFM@ 0000000140022220     arcinit.obj
 0001:00021240       ??_C@_0EL@ELLGMDMB@?$CK?5Allocate?5big?5IOCTL?5buffer?5suc@FNODOBFM@ 0000000140022240     arcinit.obj
 0001:00021290       ??_C@_0DJ@EGOLHGNF@leaving?5AllocateMessageUnitQueu@FNODOBFM@ 0000000140022290     arcinit.obj
 0001:000212d0       ??_C@_0CF@DNFJFJLG@entering?5ConfigureContainersRun@FNODOBFM@ 00000001400222d0     arcinit.obj
 0001:00021300       ??_C@_0EJ@GFICDCBB@?$CK?5ConfigureContainersRuntime?3?5R@FNODOBFM@ 0000000140022300     arcinit.obj
 0001:00021350       ??_C@_0EF@KJEEMCEN@?$CK?5ConfigureContainersRuntime?3?5G@FNODOBFM@ 0000000140022350     arcinit.obj
 0001:000213a0       ??_C@_0EF@JADMGPAN@?$CK?5ConfigureContainersRuntime?3?5G@FNODOBFM@ 00000001400223a0     arcinit.obj
 0001:000213f0       ??_C@_0EM@NKPEDKJ@?$CK?5ConfigureContainersRuntime?3?5n@FNODOBFM@ 00000001400223f0     arcinit.obj
 0001:00021440       ??_C@_0EF@ECHMIPBP@?$CK?5Found?5a?5new?5container?5?9?5tid?3?5@FNODOBFM@ 0000000140022440     arcinit.obj
 0001:00021490       ??_C@_0DK@FCJKMAGD@ConfigureContainersRuntime?3?5UID@FNODOBFM@ 0000000140022490     arcinit.obj
 0001:000214d0       ??_C@_0DK@PHPDGAOG@?$CK?5ConfigureContainersRuntime?3?5d@FNODOBFM@ 00000001400224d0     arcinit.obj
 0001:00021510       ??_C@_0GG@BFFFADFC@?$CK?5ConfigureContainersRuntime?3?5F@FNODOBFM@ 0000000140022510     arcinit.obj
 0001:00021580       ??_C@_0EA@JBBLNOGE@?$CK?5ConfigureContainersRuntime?3?5R@FNODOBFM@ 0000000140022580     arcinit.obj
 0001:000215c0       ??_C@_0FJ@MOJFHLFO@?$CK?5ConfigureContainersRuntime?3?5D@FNODOBFM@ 00000001400225c0     arcinit.obj
 0001:00021620       ??_C@_0CO@FOBCLEMJ@?$CK?5ConfigureContainersRuntime?3?5d@FNODOBFM@ 0000000140022620     arcinit.obj
 0001:00021650       ??_C@_0DO@KMBICFHC@?$CK?5ConfigureContainersRuntime?3?5S@FNODOBFM@ 0000000140022650     arcinit.obj
 0001:00021690       ??_C@_0DB@JMFIFBDA@leaving?5ConfigureContainersRunt@FNODOBFM@ 0000000140022690     arcinit.obj
 0001:000216d0       ??_C@_0CC@KOGKIGDL@entering?5CheckForVersionMisMatc@FNODOBFM@ 00000001400226d0     arcinit.obj
 0001:00021700       ??_C@_0CB@BOFDNAKM@This?5is?5a?5code?5stream?5identifie@FNODOBFM@ 0000000140022700     arcinit.obj
 0001:00021730       ??_C@_1CE@PCDJGPON@?$AAB?$AAa?$AAd?$AA?5?$AAV?$AAe?$AAr?$AAs?$AAi?$AAo?$AAn?$AA?5?$AAM?$AAa?$AAt@FNODOBFM@ 0000000140022730     arcinit.obj
 0001:00021760       ??_C@_0DF@MNNMPGOO@?$CK?5Version?5Mismatch?3?5Bios?3?$CFd?0?5Fi@FNODOBFM@ 0000000140022760     arcinit.obj
 0001:000217a0       ??_C@_0EC@DEDLMEPI@leving?5CheckForVersionMisMatch?5@FNODOBFM@ 00000001400227a0     arcinit.obj
 0001:000217f0       ??_C@_0BN@GKEKJNDP@?$CFs?5Driver?5entry?5rtnval?5?$DN?5?$CFx?6@FNODOBFM@ 00000001400227f0     arcinit.obj
 0001:00021810       ??_C@_0DD@FIIKPLIC@?$CFs?3?5Driver?5FindAdapter?5?9?5invali@FNODOBFM@ 0000000140022810     arcinit.obj
 0001:00021850       ??_C@_0M@NCHBOPE@kernalprint@FNODOBFM@ 0000000140022850     arcinit.obj
 0001:00021860       ??_C@_0BE@IDLOJBGB@?$CK?5KERNAL?5PRINT?5?$DN?51?6@FNODOBFM@ 0000000140022860     arcinit.obj
 0001:00021880       ??_C@_0BG@INJAEJHE@entering?5FindAdapter?6@FNODOBFM@ 0000000140022880     arcinit.obj
 0001:000218a0       ??_C@_0FD@NLKPIIHJ@?$CK?5This?5is?5WS03?5R2?0?5Vista?5or?5Lon@FNODOBFM@ 00000001400228a0     arcinit.obj
 0001:00021900       ??_C@_0FF@EIPBDAPC@?$CK?$CK?$CK?$CK?$CK?5Size?5of?5PORT_CONFIGURATIO@FNODOBFM@ 0000000140022900     arcinit.obj
 0001:00021960       ??_C@_0EF@MDPAOPOH@?$CK?5HwScsiFindAdapter?3?5DeviceExte@FNODOBFM@ 0000000140022960     arcinit.obj
 0001:000219b0       ??_C@_0CD@BBBDOKPE@?$CK?5Returned?5PCI?5bus?5data?5length?$DN@FNODOBFM@ 00000001400229b0     arcinit.obj
 0001:000219e0       ??_C@_0BB@ELNGMCEN@BreakPointHelper@FNODOBFM@ 00000001400229e0     arcinit.obj
 0001:00021a00       ??_C@_0BN@NMODDHNP@?$CK?53?5seconds?5waiting?5is?5done?6@FNODOBFM@ 0000000140022a00     arcinit.obj
 0001:00021a20       ??_C@_0DD@OAOECDIB@leaving?5FindAdapter?5?9?5StorPortG@FNODOBFM@ 0000000140022a20     arcinit.obj
 0001:00021a60       ??_C@_0DF@ODNFGMFG@?$CK?5leaving?5FindAdapter?5?9?5StorPor@FNODOBFM@ 0000000140022a60     arcinit.obj
 0001:00021aa0       ??_C@_0BN@FJDEMAMC@?$CK?50x40?5PCI?5Bus?5Data?5read?5in?6@FNODOBFM@ 0000000140022aa0     arcinit.obj
 0001:00021ac0       ??_C@_0BN@INBKDNHG@?$CK?50xFF?5PCI?5Bus?5Data?5read?5in?6@FNODOBFM@ 0000000140022ac0     arcinit.obj
 0001:00021ae0       ??_C@_0DB@DAIGEFPJ@?$CK?5No?5Support?5on?5Capabilties?5lis@FNODOBFM@ 0000000140022ae0     arcinit.obj
 0001:00021b20       ??_C@_0BM@KCLFMKNE@?$CK?5Capability_offset?5?$DN?50x?$CFx?5@FNODOBFM@ 0000000140022b20     arcinit.obj
 0001:00021b40       ??_C@_0BJ@KNABCMMM@?5?9?9?$DOcapabilty_id?5?$DN?50x?$CFx?6@FNODOBFM@ 0000000140022b40     arcinit.obj
 0001:00021b60       ??_C@_0BK@JIIOJNIO@?$CK?5Message_control?5?$DN?50x?$CFx?6@FNODOBFM@ 0000000140022b60     arcinit.obj
 0001:00021b80       ??_C@_0BF@HNFCBKLM@?$CK?5HW?5supports?5MSI?9X?6@FNODOBFM@ 0000000140022b80     arcinit.obj
 0001:00021ba0       ??_C@_0L@BLEMHNKF@archbamode@FNODOBFM@ 0000000140022ba0     arcinit.obj
 0001:00021bb0       ??_C@_0BM@OFPMAGCK@?$CK?5ARC?5HBA?5MODE?5setting?3?5?$CFd?6@FNODOBFM@ 0000000140022bb0     arcinit.obj
 0001:00021bd0       ??_C@_07IICIIOGL@fibdump@FNODOBFM@ 0000000140022bd0     arcinit.obj
 0001:00021be0       ??_C@_0BI@NEHBJBBP@?$CK?5FIB?5DUMP?5setting?3?5?$CFd?6@FNODOBFM@ 0000000140022be0     arcinit.obj
 0001:00021c00       ??_C@_09LEIBFFMJ@forceintx@FNODOBFM@ 0000000140022c00     arcinit.obj
 0001:00021c10       ??_C@_0N@FCLAIEBP@forcepolling@FNODOBFM@ 0000000140022c10     arcinit.obj
 0001:00021c20       ??_C@_0DI@MNEPEDIK@?$CK?5StorPortGetActiveGroupCount?5h@FNODOBFM@ 0000000140022c20     arcinit.obj
 0001:00021c60       ??_C@_0ED@JJDFFHPI@?$CK?5StorPortGetActiveGroupCount?5r@FNODOBFM@ 0000000140022c60     arcinit.obj
 0001:00021cb0       ??_C@_0DJ@FDFDEBND@?$CK?5StorPortGetHighestNodeNumber?5@FNODOBFM@ 0000000140022cb0     arcinit.obj
 0001:00021cf0       ??_C@_0EL@PIGODLHL@?$CK?5StorPortGetHighestNodeNumber?5@FNODOBFM@ 0000000140022cf0     arcinit.obj
 0001:00021d40       ??_C@_0EM@HBPALBEJ@?$CK?5StorPortGetHighestNodeNumber?5@FNODOBFM@ 0000000140022d40     arcinit.obj
 0001:00021d90       ??_C@_0DF@EDOFIEGL@?$CK?5StorPortGetGroupAffinity?5has?5@FNODOBFM@ 0000000140022d90     arcinit.obj
 0001:00021dd0       ??_C@_0HE@CADMEBCK@?$CK?5StorPortGetGroupAffinity?5retu@FNODOBFM@ 0000000140022dd0     arcinit.obj
 0001:00021e50       ??_C@_0EI@OFPHCHHN@?$CK?5StorPortGetGroupAffinity?5retu@FNODOBFM@ 0000000140022e50     arcinit.obj
 0001:00021ea0       ??_C@_0EO@MADFJJKE@?$CK?5StorPortGetGroupAffinity?5retu@FNODOBFM@ 0000000140022ea0     arcinit.obj
 0001:00021ef0       ??_C@_0P@JECJMKHH@runspecialcode@FNODOBFM@ 0000000140022ef0     arcinit.obj
 0001:00021f00       ??_C@_0BI@LHEEIHDL@?$CK?5RUN?5SPECIAL?5CODE?5?$DN?51?6@FNODOBFM@ 0000000140022f00     arcinit.obj
 0001:00021f20       ??_C@_0BI@LGIGONAM@?$CK?5RUN?5SPECIAL?5CODE?5?$DN?50?6@FNODOBFM@ 0000000140022f20     arcinit.obj
 0001:00021f40       ??_C@_0N@DDALOBCN@enablekidnap@FNODOBFM@ 0000000140022f40     arcinit.obj
 0001:00021f50       ??_C@_0BE@NKPEGEFN@?$CK?5Catchfib?5enabled?6@FNODOBFM@ 0000000140022f50     arcinit.obj
 0001:00021f70       ??_C@_0BI@PLLAPJLO@?$CK?5Catchfib?5not?5enabled?6@FNODOBFM@ 0000000140022f70     arcinit.obj
 0001:00021f90       ??_C@_0M@KNIKEID@kidnapvalve@FNODOBFM@ 0000000140022f90     arcinit.obj
 0001:00021fa0       ??_C@_0BF@CEDJMGLL@?$CK?5KIDNAP?5VALVE?5?$DN?5?$CFd?6@FNODOBFM@ 0000000140022fa0     arcinit.obj
 0001:00021fc0       ??_C@_0O@OCGMBHKL@checkinterval@FNODOBFM@ 0000000140022fc0     arcinit.obj
 0001:00021fd0       ??_C@_0CM@FEFEBKKC@?$CK?5IOP?5RESET?5COMPLETION?5Check?5In@FNODOBFM@ 0000000140022fd0     arcinit.obj
 0001:00022000       ??_C@_0N@MOEJGNKK@stallseconds@FNODOBFM@ 0000000140023000     arcinit.obj
 0001:00022010       ??_C@_0BG@DLFLFJEO@?$CK?5STALL?5SECONDS?5?$DN?5?$CFd?6@FNODOBFM@ 0000000140023010     arcinit.obj
 0001:00022030       ??_C@_0O@BPMKJHCJ@hbaqueuedepth@FNODOBFM@ 0000000140023030     arcinit.obj
 0001:00022040       ??_C@_0BI@IIHNBKPK@?$CK?5HBA?5QUEUE?5DEPTH?5?$DN?5?$CFd?6@FNODOBFM@ 0000000140023040     arcinit.obj
 0001:00022060       ??_C@_04GGLOKIEE@dump@FNODOBFM@ 0000000140023060     arcinit.obj
 0001:00022070       ??_C@_05FDLGEGEK@ntldr@FNODOBFM@ 0000000140023070     arcinit.obj
 0001:00022080       ??_C@_05PMICOLGA@hiber@FNODOBFM@ 0000000140023080     arcinit.obj
 0001:00022090       ??_C@_0CD@JEMNEMMP@?$CK?$CK?$CK?$CK?5dump?5?$HM?5ntldr?5?$HM?5hiber?5is?5TR@FNODOBFM@ 0000000140023090     arcinit.obj
 0001:000220c0       ??_C@_0BK@NELCFLHO@?$CK?5Switching?5to?5INTx?5mode?6@FNODOBFM@ 00000001400230c0     arcinit.obj
 0001:000220e0       ??_C@_09IPELKJIO@BLEDCheck@FNODOBFM@ 00000001400230e0     arcinit.obj
 0001:000220f0       ??_C@_0L@NIPCGJOG@DPCAllowed@FNODOBFM@ 00000001400230f0     arcinit.obj
 0001:00022100       ??_C@_09CHINNNMJ@CSMI?$DNNone@FNODOBFM@ 0000000140023100     arcinit.obj
 0001:00022110       ??_C@_0BA@BKKNJKOP@CSMI?$DNRestricted@FNODOBFM@ 0000000140023110     arcinit.obj
 0001:00022120       ??_C@_09PKBPEONE@CSMI?$DNFull@FNODOBFM@ 0000000140023120     arcinit.obj
 0001:00022130       ??_C@_0CJ@JHBMKCEI@leaving?5FindAdapter?5?9?5PCI?5Id?5no@FNODOBFM@ 0000000140023130     arcinit.obj
 0001:00022160       ??_C@_0CL@HDBMPJMP@?$CK?5leaving?5FindAdapter?5?9?5PCI?5Id?5@FNODOBFM@ 0000000140023160     arcinit.obj
 0001:00022190       ??_C@_0CH@LNPKNDMP@Rx?3?5BAR0?5Range?50x?$CFlx?5MappedSize@FNODOBFM@ 0000000140023190     arcinit.obj
 0001:000221c0       ??_C@_0DF@OFCBAPFL@leaving?5FindAdapter?5?9?5fail?5mapp@FNODOBFM@ 00000001400231c0     arcinit.obj
 0001:00022200       ??_C@_0DH@MNDLADLD@?$CK?5leaving?5FindAdapter?5?9?5fail?5ma@FNODOBFM@ 0000000140023200     arcinit.obj
 0001:00022240       ??_C@_0DC@NODBFDAD@leaving?5FindAdapter?5?9?5illegal?5F@FNODOBFM@ 0000000140023240     arcinit.obj
 0001:00022280       ??_C@_0EH@FLDBENFC@?$CK?5leaving?5FindAdapter?5?9?5illegal@FNODOBFM@ 0000000140023280     arcinit.obj
 0001:000222d0       ??_C@_0CK@GPLIPCCC@?$CK?5FULL?564?5BIT?5addressing?5suppor@FNODOBFM@ 00000001400232d0     arcinit.obj
 0001:00022300       ??_C@_0CD@NJEIKDOH@?$CK?5New?5outstanding?5number?5chose?3@FNODOBFM@ 0000000140023300     arcinit.obj
 0001:00022330       ??_C@_0CD@CCLGIJ@?$CK?5Old?5outstanding?5number?5chose?3@FNODOBFM@ 0000000140023330     arcinit.obj
 0001:00022360       ??_C@_05JGHMLIKJ@devqd@FNODOBFM@ 0000000140023360     arcinit.obj
 0001:00022370       ??_C@_0O@EPNNFPIH@?$CK?5DEV?5QD?3?5?$CFd?6@FNODOBFM@ 0000000140023370     arcinit.obj
 0001:00022380       ??_C@_0N@OEGLNJCG@ioctlbufsize@FNODOBFM@ 0000000140023380     arcinit.obj
 0001:00022390       ??_C@_0CI@LFOBEGIG@?$CK?5This?5is?564?9bit?5Vista?5or?5Longh@FNODOBFM@ 0000000140023390     arcinit.obj
 0001:000223c0       ??_C@_0DB@NLEKMFMO@?$CK?5This?5is?532?9bit?5WS03?5R2?0?5Vista@FNODOBFM@ 00000001400233c0     arcinit.obj
 0001:00022400       ??_C@_0CA@DJAEOOFI@?$CK?5This?5is?564?9bit?5WS03?5SP1?5?4?4?4?5?6@FNODOBFM@ 0000000140023400     arcinit.obj
 0001:00022420       ??_C@_0CA@IELABMFO@?$CK?5This?5is?532?9bit?5WS03?5SP1?5?4?4?4?5?6@FNODOBFM@ 0000000140023420     arcinit.obj
 0001:00022440       ??_C@_0CA@MNGBKCLD@?$CK?5This?5is?532?9bit?5WS03?5RTM?5?4?4?4?5?6@FNODOBFM@ 0000000140023440     arcinit.obj
 0001:00022460       ??_C@_0BL@FPDNGGII@?$CK?5Adapter?5is?5in?5poll?5mode?6@FNODOBFM@ 0000000140023460     arcinit.obj
 0001:00022480       ??_C@_0CO@NGAJFGIM@?$CK?5pDeviceExtension?9?$DONewCommInte@FNODOBFM@ 0000000140023480     arcinit.obj
 0001:000224b0       ??_C@_0CE@MCFGELJ@?$CK?5pDeviceExtension?9?$DOVendorId?3?50@FNODOBFM@ 00000001400234b0     arcinit.obj
 0001:000224e0       ??_C@_0CE@PNKCKBKJ@?$CK?5pDeviceExtension?9?$DODeviceId?3?50@FNODOBFM@ 00000001400234e0     arcinit.obj
 0001:00022510       ??_C@_0CH@NNKEKBEL@?$CK?5pDeviceExtension?9?$DOSubVendorId@FNODOBFM@ 0000000140023510     arcinit.obj
 0001:00022540       ??_C@_0CH@BEBMHIHH@?$CK?5pDeviceExtension?9?$DOSubSystemId@FNODOBFM@ 0000000140023540     arcinit.obj
 0001:00022570       ??_C@_0CB@ELGCJIGA@?$CK?5Uncached?5Memory?5address?3?50x?$CFp@FNODOBFM@ 0000000140023570     arcinit.obj
 0001:000225a0       ??_C@_0CH@CKCEEBMD@?$CK?5Uncached?5Memory?5allocated?3?50x@FNODOBFM@ 00000001400235a0     arcinit.obj
 0001:000225d0       ??_C@_0DK@INJPNBCP@?$CK?5MailBox?51?3?$CFx?0?5MailBox?52?3?$CFx?0?5M@FNODOBFM@ 00000001400235d0     arcinit.obj
 0001:00022610       ??_C@_0DB@DBAPOAM@?$CK?5pDeviceExtension?9?$DOMaxOutstand@FNODOBFM@ 0000000140023610     arcinit.obj
 0001:00022650       ??_C@_0DF@CKKIGFIG@?$CK?5pDeviceExtension?9?$DOMaxMSIXVect@FNODOBFM@ 0000000140023650     arcinit.obj
 0001:00022690       ??_C@_0M@EHMNKBMA@forcev8tov7@FNODOBFM@ 0000000140023690     arcinit.obj
 0001:000226a0       ??_C@_0CA@HGCPDEFI@?$CK?5SupportV8InitStruct?5Flag?3?5?$CFd?6@FNODOBFM@ 00000001400236a0     arcinit.obj
 0001:000226c0       ??_C@_0BA@EOIIECBM@loopbacklatency@FNODOBFM@ 00000001400236c0     arcinit.obj
 0001:000226d0       ??_C@_0BC@BDCJEMN@?$CK?5FORCE?5INTX?3?5?$CFd?6@FNODOBFM@ 00000001400236d0     arcinit.obj
 0001:000226f0       ??_C@_0BF@FJIEGFMA@?$CK?5FORCE?5POLLING?3?5?$CFd?6@FNODOBFM@ 00000001400236f0     arcinit.obj
 0001:00022710       ??_C@_0CN@OMCAJNOM@?$CK?5?$DN?$DN?$DN?$DN?$DN?$DN?$DO?5Front?5Vector?5Number?5i@FNODOBFM@ 0000000140023710     arcinit.obj
 0001:00022740       ??_C@_0CI@BJJEDHMG@?$CK?5pDeviceExtension?9?$DOVectorCapac@FNODOBFM@ 0000000140023740     arcinit.obj
 0001:00022770       ??_C@_0DE@JJAKLEJD@?$CK?5pDeviceExtension?9?$DOMSIXIoThrot@FNODOBFM@ 0000000140023770     arcinit.obj
 0001:000227b0       ??_C@_0DF@LMKAIIEG@?$CK?5pDeviceExtension?9?$DOMSIXIoThrot@FNODOBFM@ 00000001400237b0     arcinit.obj
 0001:000227f0       ??_C@_0BK@NKHDFADJ@?$CK?5CPU?5Group?5number?5is?5?$CFd?6@FNODOBFM@ 00000001400237f0     arcinit.obj
 0001:00022810       ??_C@_0BJ@OBKJCBPL@?$CK?5CPU?5Node?5number?5is?5?$CFd?6@FNODOBFM@ 0000000140023810     arcinit.obj
 0001:00022830       ??_C@_0BI@KNCDOCH@?$CK?5Node?5per?5Group?5is?5?$CFd?6@FNODOBFM@ 0000000140023830     arcinit.obj
 0001:00022850       ??_C@_0BH@FMFCFLGH@?$CK?5Core?5per?5Node?5is?5?$CFd?6@FNODOBFM@ 0000000140023850     arcinit.obj
 0001:00022870       ??_C@_0CB@HDFPBACC@?$CK?5System?5processor?5number?5is?5?$CFd@FNODOBFM@ 0000000140023870     arcinit.obj
 0001:000228a0       ??_C@_0CI@EOOKBOFL@?$CK?5?$DN?$DN?$DN?$DN?$DN?$DN?$DO?5End?5of?5Front?5summary?5@FNODOBFM@ 00000001400238a0     arcinit.obj
 0001:000228d0       ??_C@_0DE@FBKNPKIG@?$CK?5?$DN?$DN?$DN?$DN?$DN?$DN?$DO?5inside?5finalizing?5vec@FNODOBFM@ 00000001400238d0     arcinit.obj
 0001:00022910       ??_C@_06DCBAGJIF@vecnum@FNODOBFM@ 0000000140023910     arcinit.obj
 0001:00022920       ??_C@_0EB@PLAOEAEF@?$CK?5Valid_MSIX_Vectors?5is?5reset?5t@FNODOBFM@ 0000000140023920     arcinit.obj
 0001:00022970       ??_C@_0CN@KPEBIFEO@?$CK?5?$DN?$DN?$DN?$DN?$DN?$DN?$DO?5Final?5Vector?5Number?5i@FNODOBFM@ 0000000140023970     arcinit.obj
 0001:000229a0       ??_C@_0CC@CEGCGDDK@?$CK?5?$DN?$DN?$DN?$DN?$DN?$DN?$DO?5End?5of?5summary?5?$DM?$DN?$DN?$DN?$DN?$DN@FNODOBFM@ 00000001400239a0     arcinit.obj
 0001:000229d0       ??_C@_0EC@KMMHNEKL@?$CK?5ConfigInfo?9?$DOHwMSInterruptRout@FNODOBFM@ 00000001400239d0     arcinit.obj
 0001:00022a20       ??_C@_0BH@CDLDBOJF@?$CK?5SrbExtensionSize?3?$CFx?6@FNODOBFM@ 0000000140023a20     arcinit.obj
 0001:00022a40       ??_C@_0EK@GNODIBNL@?$CK?5MiniARC?5Interface?5?9?5?5CommandS@FNODOBFM@ 0000000140023a40     arcinit.obj
 0001:00022a90       ??_C@_0EL@HJMLPDNI@?$CK?5New?5Comm?5Interface?5?9?5?5Command@FNODOBFM@ 0000000140023a90     arcinit.obj
 0001:00022ae0       ??_C@_0CM@NKHNJDEG@leaving?5FindAdapter?5?9?5fail?5init@FNODOBFM@ 0000000140023ae0     arcinit.obj
 0001:00022b10       ??_C@_0CO@GHEIBKDI@?$CK?5leaving?5FindAdapter?5?9?5fail?5in@FNODOBFM@ 0000000140023b10     arcinit.obj
 0001:00022b40       ??_C@_1EA@GNKDGDHK@?$AAA?$AAd?$AAa?$AAp?$AAt?$AAe?$AAr?$AA?5?$AAg?$AAo?$AAt?$AA?5?$AAi?$AAn?$AAv@FNODOBFM@ 0000000140023b40     arcinit.obj
 0001:00022b80       ??_C@_1EI@NELDFHEH@?$AAA?$AAd?$AAa?$AAp?$AAt?$AAe?$AAr?$AA?5?$AAd?$AAo?$AAe?$AAs?$AA?5?$AAn?$AAo@FNODOBFM@ 0000000140023b80     arcinit.obj
 0001:00022bd0       ??_C@_0DC@BFHJHJOO@?$CK?5fail?5SynFibCT_SET_MINIARC_HOS@FNODOBFM@ 0000000140023bd0     arcinit.obj
 0001:00022c10       ??_C@_0DF@KABMIJBB@?$CK?5RequestSupplementAdapterInfo?0@FNODOBFM@ 0000000140023c10     arcinit.obj
 0001:00022c50       ??_C@_0CE@IADADNNA@?$CK?5Use?5MU?5Register?5for?5IOP_Reset@FNODOBFM@ 0000000140023c50     arcinit.obj
 0001:00022c80       ??_C@_0CJ@LHHNJCHI@?$CK?5Use?5inbound?5doorbell?5for?5IOP_@FNODOBFM@ 0000000140023c80     arcinit.obj
 0001:00022cb0       ??_C@_0DI@LGINDMLA@?$CK?5ERROR?3?5FW?5does?5not?5provide?5wh@FNODOBFM@ 0000000140023cb0     arcinit.obj
 0001:00022cf0       ??_C@_0BP@DJKPJIGJ@?$CK?5Ignore_IOP_Reset?5is?5set?5?4?4?4?6@FNODOBFM@ 0000000140023cf0     arcinit.obj
 0001:00022d10       ??_C@_0CK@LEDHDPPJ@?$CK?5Disk?5Power?5Management?5is?5supp@FNODOBFM@ 0000000140023d10     arcinit.obj
 0001:00022d40       ??_C@_0CJ@PJOACPGJ@?$CK?5This?5firmware?5supports?5fast?5J@FNODOBFM@ 0000000140023d40     arcinit.obj
 0001:00022d70       ??_C@_0DB@HEHLEMPI@?$CK?5Controller?5Firmware?5supports?5@FNODOBFM@ 0000000140023d70     arcinit.obj
 0001:00022db0       ??_C@_0CI@CJPAOACI@?$CK?5Controller?5Firmware?5supports?5@FNODOBFM@ 0000000140023db0     arcinit.obj
 0001:00022de0       ??_C@_0BM@LNCHEOOO@?$CK?5Virtual?5B?1T?1L?5?$CI?$CFd?1?$CFd?1?$CFd?$CJ?6@FNODOBFM@ 0000000140023de0     arcinit.obj
 0001:00022e00       ??_C@_0DA@OBMGONKI@?$CK?5Driver?5got?5SUPPORTED_NATIVE_H@FNODOBFM@ 0000000140023e00     arcinit.obj
 0001:00022e30       ??_C@_0DI@GIKAIFLA@?$CK?5Driver?5did?5not?5get?5SUPPORTED_@FNODOBFM@ 0000000140023e30     arcinit.obj
 0001:00022e70       ??_C@_0BH@LMHJIEKF@?$CK?5ExposeNonDASD?5is?5?$CFx?6@FNODOBFM@ 0000000140023e70     arcinit.obj
 0001:00022e90       ??_C@_0BB@JIKBMNNG@QueueDepthPerLun@FNODOBFM@ 0000000140023e90     arcinit.obj
 0001:00022eb0       ??_C@_0N@GDDJMKFE@PauseIOLimit@FNODOBFM@ 0000000140023eb0     arcinit.obj
 0001:00022ec0       ??_C@_0O@LIIBGGCF@ResumeIOLimit@FNODOBFM@ 0000000140023ec0     arcinit.obj
 0001:00022ed0       ??_C@_0O@OKMDGJBG@ConvertSGList@FNODOBFM@ 0000000140023ed0     arcinit.obj
 0001:00022ee0       ??_C@_0BE@IIJOOEPG@QueueStartThreshold@FNODOBFM@ 0000000140023ee0     arcinit.obj
 0001:00022f00       ??_C@_0BD@CEDPKLI@QueueDumpThreshold@FNODOBFM@ 0000000140023f00     arcinit.obj
 0001:00022f20       ??_C@_0BA@NLIGFJMK@MaxIoSizeQueued@FNODOBFM@ 0000000140023f20     arcinit.obj
 0001:00022f30       ??_C@_0N@MLHJOFDC@QueueAllowed@FNODOBFM@ 0000000140023f30     arcinit.obj
 0001:00022f40       ??_C@_0BC@IEBJFOIJ@FlushSizeInBlocks@FNODOBFM@ 0000000140023f40     arcinit.obj
 0001:00022f60       ??_C@_0EA@OJJGPBKL@leaving?5FindAdapter?5?9?5fail?5Hand@FNODOBFM@ 0000000140023f60     arcinit.obj
 0001:00022fa0       ??_C@_0EC@HNCBOCML@?$CK?5leaving?5FindAdapter?5?9?5fail?5Ha@FNODOBFM@ 0000000140023fa0     arcinit.obj
 0001:00022ff0       ??_C@_09NBOIBGGK@EnableWMI@FNODOBFM@ 0000000140023ff0     arcinit.obj
 0001:00023000       ??_C@_0DH@OIMAJCMK@?$CK?5?9?5Driver?5version?5?$CFs?0?5adapter?5@FNODOBFM@ 0000000140024000     arcinit.obj
 0001:00023040       ??_C@_0DF@NGIHOECA@?$CK?5?9?5Size?5of?5HwDevExt?$DN0x?$CFx?4?5Size@FNODOBFM@ 0000000140024040     arcinit.obj
 0001:00023080       ??_C@_0IC@BPBMMOAO@?$CK?5?9?5Size?$CISrbExt?$CJ?$DN0x?$CFx?4?5sizeof?$CIF@FNODOBFM@ 0000000140024080     arcinit.obj
 0001:00023110       ??_C@_0CA@ENCHFGMA@?$CK?5?9?5reported?5Size?$CISrbExt?$CJ?$DN0x?$CFx?6@FNODOBFM@ 0000000140024110     arcinit.obj
 0001:00023130       ??_C@_0BG@JAEBOKND@?$CK?5?9?5Done?5FindAdapter?6@FNODOBFM@ 0000000140024130     arcinit.obj
 0001:00023150       ??_C@_0FF@LMEIGAGF@?$CK?5?9?5ConfigInfo?9?$DOMaximumTransfer@FNODOBFM@ 0000000140024150     arcinit.obj
 0001:000231b0       ??_C@_0CG@GOHAMHPA@leaving?5FindAdapter?5?9?5adapter?5f@FNODOBFM@ 00000001400241b0     arcinit.obj
 0001:000231e0       ??_C@_0BN@DGMFEGDN@entering?5GetElapsedSeconds?5?6@FNODOBFM@ 00000001400241e0     arcinit.obj
 0001:00023200       ??_C@_0DD@GOLHMOHG@leaving?5GetElapsedSeconds?5?9?5sec@FNODOBFM@ 0000000140024200     arcinit.obj
 0001:00023240       ??_C@_0CJ@KCPJKGH@entering?5IsAdapterReadyForConfi@FNODOBFM@ 0000000140024240     arcinit.obj
 0001:00023270       ??_C@_0DB@PNDBFHEI@IsAdapterReadyForConfigCommand?3@FNODOBFM@ 0000000140024270     arcinit.obj
 0001:000232b0       ??_C@_0CH@PFKKGKLP@IsAdapterReadyForConfigCommand?3@FNODOBFM@ 00000001400242b0     arcinit.obj
 0001:000232e0       ??_C@_0DJ@FMKIDFML@?$CK?5leaving?5IsAdapterReadyForConf@FNODOBFM@ 00000001400242e0     arcinit.obj
 0001:00023320       ??_C@_0CI@LLJGECEO@leaving?5IsAdapterReadyForConfig@FNODOBFM@ 0000000140024320     arcinit.obj
 0001:00023350       ??_C@_0BD@LJONEFCN@entering?5IOPReset?6@FNODOBFM@ 0000000140024350     arcinit.obj
 0001:00023370       ??_C@_0EN@CPGMGMBD@?$CK?$CK?5Fail?5to?5iopreset?5the?5adapter@FNODOBFM@ 0000000140024370     arcinit.obj
 0001:000233c0       ??_C@_0GF@NGDIBMBA@?$CK?5Driver?5has?5been?5waiting?55?5sec@FNODOBFM@ 00000001400243c0     arcinit.obj
 0001:00023430       ??_C@_1CG@OOCCJMGE@?$AAI?$AAO?$AAP?$AA?5?$AAR?$AAE?$AAS?$AAE?$AAT?$AA?5?$AAd?$AAi?$AAs?$AAa?$AAb@FNODOBFM@ 0000000140024430     arcinit.obj
 0001:00023460       ??_C@_1CC@HLNFBNCO@?$AAI?$AAO?$AAP?$AA?5?$AAR?$AAE?$AAS?$AAE?$AAT?$AA?5?$AAf?$AAa?$AAi?$AAl?$AAe@FNODOBFM@ 0000000140024460     arcinit.obj
 0001:00023490       ??_C@_0DE@GCJLBNBN@?$CK?$CK?5Fail?5to?5iopreset?5the?5adapter@FNODOBFM@ 0000000140024490     arcinit.obj
 0001:000234d0       ??_C@_0BI@DKKBLGKC@?$CK?$CK?5IOPReset?5succeeded?4?6@FNODOBFM@ 00000001400244d0     arcinit.obj
 0001:000234f0       ??_C@_0DG@MCABGJKN@Driver?5should?5not?5work?5under?5MS@FNODOBFM@ 00000001400244f0     arcinit.obj
 0001:00023530       ??_C@_0DE@DDNIODIO@?$CK?5Set?5pInitStruct?9?$DONoOfMsiVecto@FNODOBFM@ 0000000140024530     arcinit.obj
 0001:00023570       ??_C@_0BC@JKJGEENA@leaving?5IOPReset?6@FNODOBFM@ 0000000140024570     arcinit.obj
 0001:00023590       ??_C@_0HE@MJKNAGNA@?$CK?$CK?5Fib2?5sent?560?5seconds?5ago?3?5B?1@FNODOBFM@ 0000000140024590     arcinit.obj
 0001:00023610       ??_C@_0HE@MLFEGAEP@?$CK?$CK?5Fib1?5sent?560?5seconds?5ago?3?5B?1@FNODOBFM@ 0000000140024610     arcinit.obj
 0001:00023690       ??_C@_0EB@NJFNJFPK@?$CK?$CK?5Driver?5internal?5AIF?5FIB?5has?5@FNODOBFM@ 0000000140024690     arcinit.obj
 0001:000236e0       ??_C@_0EN@EHHFOLPM@?$CK?$CK?5returned?5?$CFd?5SRB?5to?5OS?5at?5Ret@FNODOBFM@ 00000001400246e0     arcinit.obj
 0001:00023730       ??_C@_0EB@JKABANOB@?$CK?$CK?5Returned?5?$CFd?5SRB?5to?5OS?5at?5Ret@FNODOBFM@ 0000000140024730     arcinit.obj
 0001:00023780       ??_C@_0BK@OLLEIHIC@?$CK?5Switching?5to?5MSIx?5mode?6@FNODOBFM@ 0000000140024780     arcinit.obj
 0001:000237a0       ??_C@_0BA@EAOKKBLN@?$CK?5MSIx?5Enabled?6@FNODOBFM@ 00000001400247a0     arcinit.obj
 0001:000237b0       ??_C@_0EB@JEEKIEDM@?$CK?5Set?5pInitStruct?9?$DONoOfMsiVecto@FNODOBFM@ 00000001400247b0     arcinit.obj
 0001:00023800       ??_C@_0EA@DFHNCIMC@?$CK?5Set?5pInitStruct?9?$DONoOfMsiVecto@FNODOBFM@ 0000000140024800     arcinit.obj
 0001:00023840       ??_C@_0FP@EFJPBKEO@?$CK?5Valid?5Vector?$CI?$CFd?$CJ?0?5msix?5capabi@FNODOBFM@ 0000000140024840     arcinit.obj
 0001:000238a0       ??_C@_0CE@KCFAPPCO@?$CK?5Coalescing?5Disabled?5in?5INTx?5M@FNODOBFM@ 00000001400248a0     arcinit.obj
 0001:000238d0       ??_C@_0BE@OKKJEBLK@?$CK?5MSIX?5NOT?5Enabled?6@FNODOBFM@ 00000001400248d0     arcinit.obj
 0001:000238f0       ??_C@_0DJ@NFBMPICJ@?$CK?5Thor?5V8?5INIT?5structure?5sent?5s@FNODOBFM@ 00000001400248f0     arcinit.obj
 0001:00023930       ??_C@_0DK@LLCEGMEJ@?$CK?5NON?9Thor?5INIT?5structure?5sent?5@FNODOBFM@ 0000000140024930     arcinit.obj
 0001:00023970       ??_C@_0DE@DCIDKABN@?$CK?5V8?5INIT?5structure?5sent?5succes@FNODOBFM@ 0000000140024970     arcinit.obj
 0001:000239b0       ??_C@_0DI@LJKDAFIG@?$CK?5NON?9V8?5INIT?5structure?5sent?5su@FNODOBFM@ 00000001400249b0     arcinit.obj
 0001:000239f0       ??_C@_0ED@LLOJEJPI@leaving?5HandleAdapterGetConfig?5@FNODOBFM@ 00000001400249f0     arcinit.obj
 0001:00023a40       ??_C@_0EF@MHNEOFPB@?$CK?5leaving?5HandleAdapterGetConfi@FNODOBFM@ 0000000140024a40     arcinit.obj
 0001:00023a90       ??_C@_0DP@PECHNPGJ@leaving?5HandleAdapterGetConfig?5@FNODOBFM@ 0000000140024a90     arcinit.obj
 0001:00023ad0       ??_C@_0EB@CHAPDLOA@?$CK?5leaving?5HandleAdapterGetConfi@FNODOBFM@ 0000000140024ad0     arcinit.obj
 0001:00023b20       ??_C@_0EC@JNDOKFCE@leaving?5HandleAdapterCommitConf@FNODOBFM@ 0000000140024b20     arcinit.obj
 0001:00023b70       ??_C@_0EE@HMHNBLOK@?$CK?5leaving?5HandleAdapterCommitCo@FNODOBFM@ 0000000140024b70     arcinit.obj
 0001:00023bc0       ??_C@_0CE@FDDAIENL@entering?5HandleAdapterConfigIss@FNODOBFM@ 0000000140024bc0     arcinit.obj
 0001:00023bf0       ??_C@_0EG@EOLGKFDM@leaving?5HandleAdapterConfigIssu@FNODOBFM@ 0000000140024bf0     arcinit.obj
 0001:00023c40       ??_C@_0EI@BLLNCBDL@?$CK?5leaving?5HandleAdapterConfigIs@FNODOBFM@ 0000000140024c40     arcinit.obj
 0001:00023c90       ??_C@_0EC@KFDDDOGD@leaving?5HandleAdapterConfigIssu@FNODOBFM@ 0000000140024c90     arcinit.obj
 0001:00023ce0       ??_C@_0EE@EEHAIAKN@?$CK?5leaving?5HandleAdapterConfigIs@FNODOBFM@ 0000000140024ce0     arcinit.obj
 0001:00023d30       ??_C@_0EC@EGKDAAOP@leaving?5HandleAdapterConfigIssu@FNODOBFM@ 0000000140024d30     arcinit.obj
 0001:00023d80       ??_C@_0EE@KHOALOCB@?$CK?5leaving?5HandleAdapterConfigIs@FNODOBFM@ 0000000140024d80     arcinit.obj
 0001:00023dd0       ??_C@_0CD@FIHDJCJC@leaving?5HandleAdapterConfigIssu@FNODOBFM@ 0000000140024dd0     arcinit.obj
 0001:00023e00       ??_C@_0BK@LNIBADPE@?$CK?5Setting?5StatusBatching?6@FNODOBFM@ 0000000140024e00     arcinit.obj
 0001:00023e20       ??_C@_0EF@JDALIICL@?$CK?5Firmware?5should?5support?5ACI2?5@FNODOBFM@ 0000000140024e20     arcinit.obj
 0001:00023e70       ??_C@_0CB@DDHFLEBF@?$CK?5FW?5sets?5KERNEL_UP_AND_RUNNING@FNODOBFM@ 0000000140024e70     arcinit.obj
 0001:00023ea0       ??_C@_0CC@HECBNNJJ@?$CK?5FW?5is?5ready?5for?5config?5comman@FNODOBFM@ 0000000140024ea0     arcinit.obj
 0001:00023ed0       ??_C@_0BJ@GODFBPEB@?$CK?5Get?5config?5from?5FW?5ok?6@FNODOBFM@ 0000000140024ed0     arcinit.obj
 0001:00023ef0       ??_C@_0BK@PANMBLHC@?$CK?5Commit?5config?5to?5FW?5ok?6@FNODOBFM@ 0000000140024ef0     arcinit.obj
 0001:00023f10       ??_C@_0CA@BDIKNGAL@?$CK?5INIT?5Structure?5sent?5to?5FW?5ok?6@FNODOBFM@ 0000000140024f10     arcinit.obj
 0001:00023f30       ??_C@_0EE@GNMBAHCA@?$CK?5Get?5FW?5debug?5buffer?5failed?0?5b@FNODOBFM@ 0000000140024f30     arcinit.obj
 0001:00023f80       ??_C@_0BH@FLOGONBD@?$CK?5?9?5Driver?5version?5?$CFs?6@FNODOBFM@ 0000000140024f80     arcinit.obj
 0001:00023fa0       ??_C@_0DN@NNHBAELD@SMNormalModeInitAdapter?3?5Soft?5R@FNODOBFM@ 0000000140024fa0     arcinit.obj
 0001:00023fe0       ??_C@_0BO@IEENCLHE@entering?5HwInitializeAdapter?6@FNODOBFM@ 0000000140024fe0     arcinit.obj
 0001:00024000       ??_C@_1CA@OFEHMOBK@?$AAB?$AAa?$AAd?$AA?5?$AAP?$AAo?$AAr?$AAt?$AA?5?$AAD?$AAr?$AAi?$AAv?$AAe?$AAr@FNODOBFM@ 0000000140025000     arcinit.obj
 0001:00024020       ??_C@_0FM@FIFECPG@?$CK?5pDeviceExtension?9?$DOValid_MSIX_@FNODOBFM@ 0000000140025020     arcinit.obj
 0001:00024080       ??_C@_0EH@ONHPKJKD@?$CK?5StorPortGetMSIInfo?5returned?5F@FNODOBFM@ 0000000140025080     arcinit.obj
 0001:000240d0       ??_C@_0EC@KLPNNIKH@?$CK?5StorPortGetMSIInfo?5returned?5s@FNODOBFM@ 00000001400250d0     arcinit.obj
 0001:00024120       ??_C@_0EE@OLLCNNAO@?$CK?5StorPortGetMSIInfo?5returned?5s@FNODOBFM@ 0000000140025120     arcinit.obj
 0001:00024170       ??_C@_0EJ@OBPFJGIJ@?$CK?5StorPortGetMSIInfo?5returned?5s@FNODOBFM@ 0000000140025170     arcinit.obj
 0001:000241c0       ??_C@_0CF@FDBIIPFF@?$CK?5This?5Tupelo?5driver?5is?5MSI?5ena@FNODOBFM@ 00000001400251c0     arcinit.obj
 0001:000241f0       ??_C@_0BO@FHHBMMGN@?$CK?5PerfConfigData?4Flags?3?50x?$CFx?6@FNODOBFM@ 00000001400251f0     arcinit.obj
 0001:00024210       ??_C@_0FE@LBLIGLIO@GetDoorbellMaskForIOPReset?5retu@FNODOBFM@ 0000000140025210     arcinit.obj
 0001:00024270       ??_C@_0DN@IMFNPMPP@?$CK?5Failed?5to?5Initialize?5Adapter?5@FNODOBFM@ 0000000140025270     arcinit.obj
 0001:000242b0       ??_C@_0DE@CMNGFMDL@?$CK?5Succeed?5to?5Initialize?5Adapter@FNODOBFM@ 00000001400252b0     arcinit.obj
 0001:000242f0       ??_C@_0EG@KGJBNOFG@?$CK?5Failed?5to?5Initialize?5Adapter?5@FNODOBFM@ 00000001400252f0     arcinit.obj
 0001:00024340       ??_C@_0BP@MCCOMIEF@?$CK?5leaving?5HwInitializeAdapter?6@FNODOBFM@ 0000000140025340     arcinit.obj
 0001:00024360       ??_C@_0FN@OJHBJJGK@?$CK?5StorPortAllocateContiguousMem@FNODOBFM@ 0000000140025360     arcinit.obj
 0001:000243c0       ??_C@_0FD@MKBBGMOP@?$CK?5PROBLEM?3?5returnedSize?5?$DN?50?5?$CISt@FNODOBFM@ 00000001400253c0     arcinit.obj
 0001:00024420       ??_C@_0IH@LCJNFDMG@?$CK?5StorPortAllocateContiguousMem@FNODOBFM@ 0000000140025420     arcinit.obj
 0001:000244b0       ??_C@_0BI@BOGNCAIA@entering?5InitializeDPC?6@FNODOBFM@ 00000001400254b0     arcinit.obj
 0001:000244d0       ??_C@_0BL@ICGKMMAJ@?$CK?5Start?5scanning?5group?5?$CFd?6@FNODOBFM@ 00000001400254d0     arcinit.obj
 0001:000244f0       ??_C@_0CO@FDNLALKJ@?$CK?5Group?5Affinity?5for?5msix?5vecto@FNODOBFM@ 00000001400254f0     arcinit.obj
 0001:00024520       ??_C@_0DA@FPNPLEPN@?$CK?5NUMA?5node?5for?5MSIX?5vector?5?$CFd?5@FNODOBFM@ 0000000140025520     arcinit.obj
 0001:00024550       ??_C@_0DP@MAPFHEEH@?$CK?5Outbound?5Queue?5Memory?5allocat@FNODOBFM@ 0000000140025550     arcinit.obj
 0001:00024590       ??_C@_0CG@GFDFODNM@?$CK?5MemoryBlock?5?$CFd?5assigned?5in?5no@FNODOBFM@ 0000000140025590     arcinit.obj
 0001:000245c0       ??_C@_0DG@CGCBEMEO@?$CK?5MSG?5CAP?5setup?5failed?5?$CIbecause@FNODOBFM@ 00000001400255c0     arcinit.obj
 0001:00024600       ??_C@_0ED@CJAGENOE@?$CK?5we?5are?5processing?5last?5MSIX?5v@FNODOBFM@ 0000000140025600     arcinit.obj
 0001:00024650       ??_C@_0HA@GKDMKHHO@?$CK?5we?5have?5a?5problem?4?5All?5groups@FNODOBFM@ 0000000140025650     arcinit.obj
 0001:000246c0       ??_C@_0FD@LFCJJKMC@?$CK?5StorPortGetLogicalProcessorRe@FNODOBFM@ 00000001400256c0     arcinit.obj
 0001:00024720       ??_C@_0BG@FAIHHGLA@?$CK?5Vector?5?$CFd?5is?5done?6?6@FNODOBFM@ 0000000140025720     arcinit.obj
 0001:00024740       ??_C@_0DJ@MGMHFMAN@?$CK?5Failed?5to?5Initialize?5Adapter?5@FNODOBFM@ 0000000140025740     arcinit.obj
 0001:00024780       ??_C@_0DA@GDJCAINB@?$CK?5Succeed?5to?5Initialize?5Adapter@FNODOBFM@ 0000000140025780     arcinit.obj
 0001:000247b0       ??_C@_0BJ@CFFELFMJ@?$CK?5MSIx?5DPCs?5initialized?6@FNODOBFM@ 00000001400257b0     arcinit.obj
 0001:000247d0       ??_C@_0BI@LAPEOFCN@?$CK?5?9?5Done?5InitializeDPC?6@FNODOBFM@ 00000001400257d0     arcinit.obj
 0001:000247f0       ??_C@_0BH@PAHICDNJ@leaving?5InitializeDPC?6@FNODOBFM@ 00000001400257f0     arcinit.obj
 0001:00024810       ??_C@_0CP@OJKLKHLO@entering?5InitializeConsumerProd@FNODOBFM@ 0000000140025810     arcinit.obj
 0001:00024840       ??_C@_0DE@MJJEGAKI@leaving?5InitializeConsumerProdu@FNODOBFM@ 0000000140025840     arcinit.obj
 0001:00024880       ??_C@_0CO@NEGLFCOP@leaving?5InitializeConsumerProdu@FNODOBFM@ 0000000140025880     arcinit.obj
 0001:000248b0       ??_C@_0CP@IKCNDLML@entering?5InitializeConsumerProd@FNODOBFM@ 00000001400258b0     arcinit.obj
 0001:000248e0       ??_C@_0DF@IICIHNDP@leaving?5InitializeConsumerProdu@FNODOBFM@ 00000001400258e0     arcinit.obj
 0001:00024920       ??_C@_0DE@OBANPGHF@leaving?5InitializeConsumerProdu@FNODOBFM@ 0000000140025920     arcinit.obj
 0001:00024960       ??_C@_0CP@GDFIJJML@entering?5InitializeMessageUnitQ@FNODOBFM@ 0000000140025960     arcinit.obj
 0001:00024990       ??_C@_0DF@CLHHLLI@leaving?5InitializeMessageUnitQu@FNODOBFM@ 0000000140025990     arcinit.obj
 0001:000249d0       ??_C@_0DE@BBDIIBAC@leaving?5InitializeMessageUnitQu@FNODOBFM@ 00000001400259d0     arcinit.obj
 0001:00024a10       ??_C@_0BI@PNFIHJKN@entering?5MapDeviceBase?6@FNODOBFM@ 0000000140025a10     arcinit.obj
 0001:00024a30       ??_C@_1CM@FGGDGCGC@?$AAA?$AAd?$AAa?$AAp?$AAt?$AAe?$AAr?$AA?5?$AAb?$AAo?$AAo?$AAt?$AA?5?$AAt?$AAi@FNODOBFM@ 0000000140025a30     arcinit.obj
 0001:00024a60       ??_C@_0CO@NHBGNFPE@?$CK?5Driver?5got?564?5bit?5FIB?5support@FNODOBFM@ 0000000140025a60     arcinit.obj
 0001:00024a90       ??_C@_0DG@EECBHNEJ@?$CK?5Driver?5did?5not?5get?564?5bit?5FIB@FNODOBFM@ 0000000140025a90     arcinit.obj
 0001:00024ad0       ??_C@_0CB@MHHOKKDH@?$CK?5Smart?5Array?5Based?5FW?5detected@FNODOBFM@ 0000000140025ad0     arcinit.obj
 0001:00024b00       ??_C@_0CG@INGLDPEA@?$CK?5This?5is?5NOT?5a?5Smart?5Array?5Bas@FNODOBFM@ 0000000140025b00     arcinit.obj
 0001:00024b30       ??_C@_0DL@HHJHAPNC@?$CK?5StorPortGetDeviceBase?5failed?0@FNODOBFM@ 0000000140025b30     arcinit.obj
 0001:00024b70       ??_C@_0FM@FAGAFMJI@?$CK?5StorPortGetDeviceBaseB1?5faile@FNODOBFM@ 0000000140025b70     arcinit.obj
 0001:00024bd0       ??_C@_0FM@DFFNMELK@?$CK?5StorPortGetDeviceBaseB0?5faile@FNODOBFM@ 0000000140025bd0     arcinit.obj
 0001:00024c30       ??_C@_0DH@GMHBCEJM@?$CK?5GET_MINIARC_PROPERTIES?5fails?0@FNODOBFM@ 0000000140025c30     arcinit.obj
 0001:00024c70       ??_C@_0CE@JIIGOPEA@?$CK?5This?5is?5a?5BEDROC?5inplementati@FNODOBFM@ 0000000140025c70     arcinit.obj
 0001:00024ca0       ??_C@_0CF@HKNELPOC@leaving?5MapDeviceBase?5?9?5rtnval?5@FNODOBFM@ 0000000140025ca0     arcinit.obj
 0001:00024cd0       ??_C@_0BG@LOIMFNHP@entering?5MatchPciIds?6@FNODOBFM@ 0000000140025cd0     arcinit.obj
 0001:00024cf0       ??_C@_08HNOCAICB@Adaptec?5@FNODOBFM@ 0000000140025cf0     arcinit.obj
 0001:00024d00       ??_C@_0CC@GEDCIDMJ@leaving?5MatchPciIds?0?5rtnval?5?$DN?5?$CF@FNODOBFM@ 0000000140025d00     arcinit.obj
 0001:00024d30       ??_C@_0DG@MJCHKBMN@?$CK?5Calling?5CompleteBufferedReque@FNODOBFM@ 0000000140025d30     arcinit.obj
 0001:00024d70       ??_C@_0HF@LDMKNKBL@?$CK?5Calling?5DequeueRawIoReadWrite@FNODOBFM@ 0000000140025d70     arcinit.obj
 0001:00024df0       ??_C@_0CG@EHFONFB@ReturningLocalOutstandingReques@FNODOBFM@ 0000000140025df0     arcinit.obj
 0001:00024e20       ??_C@_0CL@CGNJGHDF@?$CK?5?$CFd?5outstanding?5IO?5left?5after?5@FNODOBFM@ 0000000140025e20     arcinit.obj
 0001:00024e50       ??_C@_0DI@FDADMONL@?$CK?5CleanHostSideRRQ?3?5Host?5RRQ?5cl@FNODOBFM@ 0000000140025e50     arcinit.obj
 0001:00024e90       ??_C@_0CF@IKJOOFLA@?$CK?5ResetAdapter?3?5Entering?5Routin@FNODOBFM@ 0000000140025e90     arcinit.obj
 0001:00024ec0       ??_C@_0FI@OABPGHMC@?$CK?5ResetAdapter?3?5FW?5is?5processin@FNODOBFM@ 0000000140025ec0     arcinit.obj
 0001:00024f20       ??_C@_0DK@DMNFFNOF@?$CK?5ResetAdapter?3?5OS?5calls?5ResetA@FNODOBFM@ 0000000140025f20     arcinit.obj
 0001:00024f60       ??_C@_0CF@DGMKAPOJ@?$CK?5ResetAdapter?3?5BlinkLed?5Code?3?5@FNODOBFM@ 0000000140025f60     arcinit.obj
 0001:00024f90       ??_C@_0CL@MJAGNJPB@?$CK?5ResetAdapter?3?5IOP?5RESET?5due?5t@FNODOBFM@ 0000000140025f90     arcinit.obj
 0001:00024fc0       ??_C@_0DG@CLNGJPOA@?$CK?5ResetAdapter?3?5SendSynchFib?5fa@FNODOBFM@ 0000000140025fc0     arcinit.obj
 0001:00025000       ??_C@_0FF@JLPFKNGK@?$CK?5ResetAdapter?3?5There?5is?5a?5pend@FNODOBFM@ 0000000140026000     arcinit.obj
 0001:00025060       ??_C@_0EC@MMLNJELN@?$CK?5ResetAdapter?3?5set?5TriggerIOPR@FNODOBFM@ 0000000140026060     arcinit.obj
 0001:000250b0       ??_C@_0EH@BGKKNIMJ@?$CK?5ResetAdapter?3?5synch?5command?5R@FNODOBFM@ 00000001400260b0     arcinit.obj
 0001:00025100       ??_C@_0EE@KPCKIKGP@?$CK?5ResetAdapter?3?5AdapterIsAlive?5@FNODOBFM@ 0000000140026100     arcinit.obj
 0001:00025150       ??_C@_0DN@OJOIDCGM@?$CK?5ResetAdapter?3?5leaving?5Routine@FNODOBFM@ 0000000140026150     arcinit.obj
 0001:00025190       ??_C@_0DN@MKLLHNDH@?$CK?5ResetAdapter?3?5IOP?5RESET?5due?5t@FNODOBFM@ 0000000140026190     arcinit.obj
 0001:000251d0       ??_C@_0DA@IHJFMKGH@?$CK?5ResetAdapter?3?5IOP?5RESET?5due?5t@FNODOBFM@ 00000001400261d0     arcinit.obj
 0001:00025200       ??_C@_0FJ@HDBMDLNL@?$CK?5ResetAdapter?3?5RAID?5volume?5?$CFd?5@FNODOBFM@ 0000000140026200     arcinit.obj
 0001:00025260       ??_C@_0DC@DFLLLKCM@?$CK?5ResetAdapter?3?5IOP_RESET_FW_FI@FNODOBFM@ 0000000140026260     arcinit.obj
 0001:000252a0       ??_C@_0DM@IMELCPEN@?$CK?5ResetAdapter?3?5Failed?5to?5send?5@FNODOBFM@ 00000001400262a0     arcinit.obj
 0001:000252e0       ??_C@_0EG@FKMCGCCN@?$CK?5ResetAdapter?3?5IOP?5RESET?5due?5t@FNODOBFM@ 00000001400262e0     arcinit.obj
 0001:00025330       ??_C@_0DE@IDNFNJBF@?$CK?5ResetAdapter?3?5NO?5lun?5reset?5co@FNODOBFM@ 0000000140026330     arcinit.obj
 0001:00025370       ??_C@_0DM@KJNOMFJC@?$CK?5ResetAdapter?3?5leaving?5Routine@FNODOBFM@ 0000000140026370     arcinit.obj
 0001:000253b0       ??_C@_0EK@OOPLAGOO@?$CK?5ResetAdapter?3?5set?5timer?5to?5ch@FNODOBFM@ 00000001400263b0     arcinit.obj
 0001:00025400       ??_C@_0DM@LMPLKKMJ@?$CK?5ResetAdapter?3?5leaving?5Routine@FNODOBFM@ 0000000140026400     arcinit.obj
 0001:00025440       ??_C@_0EJ@DNGMPOBO@?$CK?5ResetAdapter?3?5HWSoftReset?5lea@FNODOBFM@ 0000000140026440     arcinit.obj
 0001:00025490       ??_C@_0CJ@PCBCCJEM@?$DMHW?$DOTD?$AI?$AA?$AA?$AA?$AA?$AA?$AA?$AA?$AA?$AADW?$AA?$AADV?$BK?$AA?$AA?$AA?$AA?$AA?$AA?$AA?$AA@FNODOBFM@ 0000000140026490     arcinit.obj
 0001:000254c0       ??_C@_0BP@BFNIMKLC@?$CK?5SetFwTime?3?5Time?5sent?5failed?6@FNODOBFM@ 00000001400264c0     arcinit.obj
 0001:000254e0       ??_C@_0BL@IIHDOJJO@?$CK?5Time?3?5?$CFd?4?$CFd?4?$CFd?5?$CFd?3?$CFd?3?$CFd?6@FNODOBFM@ 00000001400264e0     arcinit.obj
 0001:00025500       ??_C@_0BG@NCOEMLFM@?$CK?5Driver?5version?5?$CFs?5?6@FNODOBFM@ 0000000140026500     arcinit.obj
 0001:00025520       ??_C@_0CF@KGAABJAP@?$CK?5SetFwTime?3?5Time?5sent?5successf@FNODOBFM@ 0000000140026520     arcinit.obj
 0001:00025550       ??_C@_0DB@DBHKEEOM@?$CK?5SendWellnessCommand?3?5Wellness@FNODOBFM@ 0000000140026550     arcinit.obj
 0001:00025590       ??_C@_0DG@CHJDHKJC@?$CK?5SendWellnessCommand?3?5Wellness@FNODOBFM@ 0000000140026590     arcinit.obj
 0001:000255d0       ??_C@_0N@GDIDOMEJ@?$DMHW?$DOPS?$AC?$AA?$AA?$AAZZ@FNODOBFM@ 00000001400265d0     arcinit.obj
 0001:000255e0       ??_C@_0CM@KDDJKBII@?$CK?5SetPciSlotNumber?3?5Update?5PCI?5@FNODOBFM@ 00000001400265e0     arcinit.obj
 0001:00025610       ??_C@_0BL@CAAHKIPO@?$CK?5PCI?5Slot?5Number?5Set?5?$CFx?5?6@FNODOBFM@ 0000000140026610     arcinit.obj
 0001:00025630       ??_C@_0DB@KLKDBGPC@?$CK?5current?5ElapsedTime?5is?5?$CFx?4?5Dr@FNODOBFM@ 0000000140026630     arcinit.obj
 0001:00025670       ??_C@_0EE@NDLKAFLN@?$CK?5SetArcsasFwTime?3?5SendSyncFib?5@FNODOBFM@ 0000000140026670     arcinit.obj
 0001:000256c0       ??_C@_0DN@BMDNNOBN@?$CK?5GetThorHbaPhyDevInfo?3?5synch?5F@FNODOBFM@ 00000001400266c0     arcinit.obj
 0001:00025700       ??_C@_0FG@PNEDCHMO@?$CK?5one?5dual?5port?5entry?5?$CIB?1T?1nexu@FNODOBFM@ 0000000140026700     arcinit.obj
 0001:00025760       ??_C@_0EM@BKPAJHPD@?$CK?5One?5entry?5?$CIB?1T?1nexus?3?5?$CFd?1?$CFd?10@FNODOBFM@ 0000000140026760     arcinit.obj
 0001:000257b0       ??_C@_0BI@NKGGGHHE@?$CK?5?$CFd?5HBA?5devices?5found?6@FNODOBFM@ 00000001400267b0     arcinit.obj
 0001:000257d0       ??_C@_0DD@PLCLGMJE@?$CK?5All?5HBA?5devices?8?5average?5Queu@FNODOBFM@ 00000001400267d0     arcinit.obj
 0001:00025810       ??_C@_0BF@GFOGGOIF@GetThorHbaPhyDevInfo@FNODOBFM@ 0000000140026810     arcinit.obj
 0001:00025830       ??_C@_0CL@OHPEFDNF@?$CK?5There?5is?5a?5synch?5SRB?5pending?0@FNODOBFM@ 0000000140026830     arcinit.obj
 0001:00025860       ??_C@_0DJ@HDKNIPML@?$CK?5Not?5a?5Thor?5product?5OR?5virtual@FNODOBFM@ 0000000140026860     arcinit.obj
 0001:000258a0       ??_C@_1FE@JLJHJCGF@?$AAA?$AAr?$AAr?$AAa?$AAy?$AA?5?$AAm?$AAi?$AAg?$AAr?$AAa?$AAt?$AAi?$AAo?$AAn@FNODOBFM@ 00000001400268a0     arcinit.obj
 0001:00025900       ??_C@_1CK@DJNKNDAB@?$AAR?$AAa?$AAw?$AA?5?$AAD?$AAr?$AAi?$AAv?$AAe?$AA?5?$AAr?$AAe?$AAm?$AAo?$AAv@FNODOBFM@ 0000000140026900     arcinit.obj
 0001:00025930       ??_C@_1DG@JPPGPNNE@?$AAN?$AAa?$AAt?$AAi?$AAv?$AAe?$AA?5?$AAH?$AAB?$AAA?$AA?5?$AAd?$AAe?$AAv?$AAi@FNODOBFM@ 0000000140026930     arcinit.obj
 0001:00025970       ??_C@_1DK@DMPEAPAK@?$AAN?$AAa?$AAt?$AAi?$AAv?$AAe?$AA?5?$AAH?$AAB?$AAA?$AA?5?$AAd?$AAe?$AAv?$AAi@FNODOBFM@ 0000000140026970     arcinit.obj
 0001:000259b0       ??_C@_1EO@PNKAKFGH@?$AAH?$AAa?$AAr?$AAd?$AAw?$AAa?$AAr?$AAe?$AA?5?$AAn?$AAo?$AAt?$AA?5?$AAp?$AAr@FNODOBFM@ 00000001400269b0     arcinit.obj
 0001:00025a00       ??_C@_1CI@IELPCEHF@?$AAS?$AAu?$AAp?$AAe?$AAr?$AAc?$AAa?$AAp?$AA?5?$AAh?$AAe?$AAa?$AAl?$AAt?$AAh@FNODOBFM@ 0000000140026a00     arcinit.obj
 0001:00025a30       ??_C@_1CK@BAADJOPA@?$AAS?$AAu?$AAp?$AAe?$AAr?$AAc?$AAa?$AAp?$AA?5?$AAh?$AAe?$AAa?$AAl?$AAt?$AAh@FNODOBFM@ 0000000140026a30     arcinit.obj
 0001:00025a60       ??_C@_1CA@DNJAAJKJ@?$AAC?$AAa?$AAc?$AAh?$AAe?$AA?5?$AAd?$AAa?$AAt?$AAa?$AA?5?$AAl?$AAo?$AAs?$AAs@FNODOBFM@ 0000000140026a60     arcinit.obj
 0001:00025a80       ??_C@_1DG@KILEJPC@?$AAT?$AAe?$AAm?$AAp?$AAe?$AAr?$AAa?$AAt?$AAu?$AAr?$AAe?$AA?5?$AAB?$AAa?$AAc@FNODOBFM@ 0000000140026a80     arcinit.obj
 0001:00025ac0       ??_C@_1DG@IHOODPDN@?$AAS?$AAu?$AAp?$AAe?$AAr?$AAc?$AAa?$AAp?$AA?5?$AAT?$AAe?$AAm?$AAp?$AAe?$AAr@FNODOBFM@ 0000000140026ac0     arcinit.obj
 0001:00025b00       ??_C@_1DK@KKLIINGO@?$AAS?$AAu?$AAp?$AAe?$AAr?$AAc?$AAa?$AAp?$AA?5?$AAT?$AAe?$AAm?$AAp?$AAe?$AAr@FNODOBFM@ 0000000140026b00     arcinit.obj
 0001:00025b40       ??_C@_1DK@HENHBAOO@?$AAB?$AAa?$AAc?$AAk?$AAu?$AAp?$AA?5?$AAu?$AAn?$AAi?$AAt?$AA?5?$AAs?$AAe?$AAl@FNODOBFM@ 0000000140026b40     arcinit.obj
 0001:00025b80       ??_C@_1DK@GKIHJFEC@?$AAF?$AAa?$AAt?$AAa?$AAl?$AA?5?$AAE?$AAr?$AAr?$AAo?$AAr?$AA?3?$AA?5?$AAB?$AAa@FNODOBFM@ 0000000140026b80     arcinit.obj
 0001:00025bc0       ??_C@_1CO@DFMHCOAI@?$AAL?$AAo?$AAg?$AAi?$AAc?$AAa?$AAl?$AA?5?$AAD?$AAr?$AAi?$AAv?$AAe?$AA?5?$AAa@FNODOBFM@ 0000000140026bc0     arcinit.obj
 0001:00025bf0       ??_C@_1DC@CMPCKFLI@?$AAL?$AAo?$AAg?$AAi?$AAc?$AAa?$AAl?$AA?5?$AAD?$AAr?$AAi?$AAv?$AAe?$AA?5?$AAd@FNODOBFM@ 0000000140026bf0     arcinit.obj
 0001:00025c30       ??_C@_1CI@JDGBIDGK@?$AAA?$AA?5?$AAn?$AAe?$AAw?$AA?5?$AAJ?$AAB?$AAO?$AAD?$AA?5?$AAi?$AAs?$AA?5?$AAa@FNODOBFM@ 0000000140026c30     arcinit.obj
 0001:00025c60       ??_C@_1CE@CICPDMOD@?$AAA?$AA?5?$AAJ?$AAB?$AAO?$AAD?$AA?5?$AAi?$AAs?$AA?5?$AAd?$AAe?$AAl?$AAe?$AAt@FNODOBFM@ 0000000140026c60     arcinit.obj
 0001:00025c90       ??_C@_1DI@CCPBOJAM@?$AAL?$AAu?$AAn?$AA?5?$AAR?$AAe?$AAs?$AAe?$AAt?$AA?5?$AAt?$AAh?$AAr?$AAe?$AAs@FNODOBFM@ 0000000140026c90     arcinit.obj
 0001:00025cd0       ??_C@_1DG@OJKKJGHC@?$AAA?$AAd?$AAa?$AAp?$AAt?$AAe?$AAr?$AA?5?$AAa?$AAl?$AAi?$AAv?$AAe?$AA?5?$AAr@FNODOBFM@ 0000000140026cd0     arcinit.obj
 0001:00025d10       ??_C@_1FC@MIPJHMMM@?$AAR?$AAe?$AAq?$AAu?$AAe?$AAs?$AAt?$AAA?$AAd?$AAa?$AAp?$AAt?$AAe?$AAr?$AAI@FNODOBFM@ 0000000140026d10     arcinit.obj
 0001:00025d70       ??_C@_1DC@FGMGNGA@?$AAF?$AAW?$AA?5?$AAK?$AAe?$AAr?$AAn?$AAe?$AAl?$AA?5?$AAP?$AAa?$AAn?$AAi?$AAc@FNODOBFM@ 0000000140026d70     arcinit.obj
 0001:00025db0       ??_C@_1CA@BBEOIBOD@?$AAU?$AAn?$AAd?$AAe?$AAf?$AAi?$AAn?$AAe?$AAd?$AA?5?$AAE?$AAv?$AAe?$AAn?$AAt@FNODOBFM@ 0000000140026db0     arcinit.obj
 0001:00025dd0       ??_C@_1EG@MMOHKHFO@?$AAC?$AAT?$AA_?$AAC?$AAO?$AAN?$AAF?$AAI?$AAG?$AA_?$AAS?$AAT?$AAA?$AAT?$AAU@FNODOBFM@ 0000000140026dd0     arcinit.obj
 0001:00025e20       ??_C@_1EC@LINPOIBA@?$AAC?$AAT?$AA_?$AAG?$AAE?$AAT?$AA_?$AAC?$AAO?$AAN?$AAF?$AAI?$AAG?$AA_?$AAS@FNODOBFM@ 0000000140026e20     arcinit.obj
 0001:00025e70       ??_C@_1DI@OLCGHNCB@?$AAC?$AAT?$AA_?$AAC?$AAO?$AAM?$AAM?$AAI?$AAT?$AA_?$AAC?$AAO?$AAN?$AAF?$AAI@FNODOBFM@ 0000000140026e70     arcinit.obj
 0001:00025eb0       ??_C@_1FA@NIJNEMHE@?$AAA?$AAD?$AAA?$AAP?$AAT?$AAE?$AAR?$AA_?$AAI?$AAN?$AAI?$AAT?$AA_?$AAS?$AAT@FNODOBFM@ 0000000140026eb0     arcinit.obj
 0001:00025f00       ??_C@_1DM@EFGMNBLE@?$AAV?$AAM?$AA_?$AAC?$AAo?$AAn?$AAt?$AAa?$AAi?$AAn?$AAe?$AAr?$AAC?$AAo?$AAn@FNODOBFM@ 0000000140026f00     arcinit.obj
 0001:00025f40       ??_C@_1DC@PCLINFGL@?$AAT?$AAi?$AAm?$AAe?$AAd?$AAo?$AAu?$AAt?$AA?0?$AA?5?$AAI?$AAn?$AAi?$AAt?$AA?5@FNODOBFM@ 0000000140026f40     arcinit.obj
 0001:00025f80       ??_C@_1FE@PCKFJNFD@?$AAR?$AAe?$AAs?$AAe?$AAt?$AA?5?$AAf?$AAr?$AAo?$AAm?$AA?5?$AAO?$AAS?$AA?3?$AAp@FNODOBFM@ 0000000140026f80     arcinit.obj
 0001:00025fe0       ??_C@_1FC@CLHIPIHG@?$AAG?$AAo?$AAt?$AA?5?$AAL?$AAU?$AAN?$AA?5?$AAR?$AAE?$AAS?$AAE?$AAT?$AA?5?$AAf@FNODOBFM@ 0000000140026fe0     arcinit.obj
 0001:00026040       ??_C@_1FI@HJHKOPPE@?$AAG?$AAo?$AAt?$AA?5?$AAT?$AAa?$AAr?$AAg?$AAe?$AAt?$AA?5?$AAR?$AAE?$AAS?$AAE@FNODOBFM@ 0000000140027040     arcinit.obj
 0001:000260a0       ??_C@_1EC@DEFLMBHE@?$AAI?$AAO?$AAP?$AA?5?$AAR?$AAE?$AAS?$AAE?$AAT?$AA?5?$AAb?$AAe?$AAc?$AAa?$AAu@FNODOBFM@ 00000001400270a0     arcinit.obj
 0001:000260f0       ??_C@_1FA@GLBMBCFD@?$AAR?$AAe?$AAq?$AAu?$AAe?$AAs?$AAt?$AAA?$AAd?$AAa?$AAp?$AAt?$AAe?$AAr?$AAI@FNODOBFM@ 00000001400270f0     arcinit.obj
 0001:00026140       ??_C@_1EK@DPFNMDNI@?$AAI?$AAO?$AAP?$AAR?$AAE?$AAS?$AAE?$AAT?$AA?3?$AA?5?$AAR?$AAe?$AAq?$AAu?$AAe@FNODOBFM@ 0000000140027140     arcinit.obj
 0001:00026190       ??_C@_1EC@JONMGECF@?$AAR?$AAA?$AA?3?$AA?5?$AAA?$AAd?$AAa?$AAp?$AAt?$AAe?$AAr?$AAI?$AAs?$AAA?$AAl@FNODOBFM@ 0000000140027190     arcinit.obj
 0001:000261e0       ??_C@_1EA@KMCOFCE@?$AAI?$AAO?$AAP?$AA?5?$AAR?$AAE?$AAS?$AAE?$AAT?$AA?5?$AAf?$AAo?$AAr?$AA?5?$AAS@FNODOBFM@ 00000001400271e0     arcinit.obj
 0001:00026220       ??_C@_1EK@EBJJOFBF@?$AAR?$AAE?$AAS?$AAE?$AAT?$AA?$CI?$AAc?$AAn?$AAt?$AA?$DO?$AA?$DN?$AA5?$AA?$CJ?$AA?3?$AA?5@FNODOBFM@ 0000000140027220     arcinit.obj
 0001:00026270       ??_C@_1DA@EFMGPIMG@?$AAS?$AAO?$AAF?$AAT?$AA?5?$AAR?$AAE?$AAS?$AAE?$AAT?$AA?5?$AAI?$AAs?$AAs?$AAu@FNODOBFM@ 0000000140027270     arcinit.obj
 0001:000262a0       ??_C@_1CO@GBDEAPLE@?$AAI?$AAO?$AAP?$AA?5?$AAR?$AAE?$AAS?$AAE?$AAT?$AA?5?$AAI?$AAs?$AAs?$AAu?$AAe@FNODOBFM@ 00000001400272a0     arcinit.obj
 0001:000262d0       ??_C@_1EI@KMCCOKBI@?$AAF?$AAW?$AA?5?$AAK?$AAE?$AAR?$AAN?$AAE?$AAL?$AA?5?$AAP?$AAA?$AAN?$AAI?$AAC@FNODOBFM@ 00000001400272d0     arcinit.obj
 0001:00026320       ??_C@_1EK@GGMELPLN@?$AAF?$AAW?$AA?5?$AAN?$AAo?$AAt?$AA?5?$AAU?$AAp?$AA?5?$AA?$CG?$AA?5?$AAR?$AAu?$AAn@FNODOBFM@ 0000000140027320     arcinit.obj
 0001:00026370       ??_C@_0BG@HHGGAPDG@entering?5HWSoftReset?6@FNODOBFM@ 0000000140027370     arcinit.obj
 0001:00026390       ??_C@_0CB@CNHAMPIN@HwSoftReset?3?5Soft?5Reset?5Issued?4@FNODOBFM@ 0000000140027390     arcinit.obj
 0001:000263c0       ??_C@_0DJ@CBPNBDFH@?$CK?5Set?5pInitStruct?9?$DONoOfMsiVecto@FNODOBFM@ 00000001400273c0     arcinit.obj
 0001:00026400       ??_C@_0BG@FGBHCKJG@CompleteQueuedRequest@FNODOBFM@ 0000000140027400     cmddelivery.obj
 0001:00026420       ??_C@_0DM@OFFCECMD@IN?5?$CFs?0?5WE?5ARE?5SEEING?5AIF?5FIB?4?5D@FNODOBFM@ 0000000140027420     cmddelivery.obj
 0001:00026460       ??_C@_0L@ENAJINDB@Management@FNODOBFM@ 0000000140027460     cmddelivery.obj
 0001:00026470       ??_C@_0BB@JIADCMFJ@Array?5?5?5?5?5?5?5?5?5?5?5@FNODOBFM@ 0000000140027470     cmddelivery.obj
 0001:00026490       ??_C@_0BB@HJODFKJH@ARRAY?5?5?5?5?5?5?5?5?5?5?5@FNODOBFM@ 0000000140027490     cmddelivery.obj
 0001:000264b0       ??_C@_0CB@IIENMBOI@?$CK?5Got?5an?5AIF?5in?5crash?5dump?5mode@FNODOBFM@ 00000001400274b0     cmddelivery.obj
 0001:000264e0       ??_C@_0DO@NPBDNHBG@?$CK?5Should?5not?5be?5here?0?5we?5should@FNODOBFM@ 00000001400274e0     cmddelivery.obj
 0001:00026520       ??_C@_0CO@PDPAIINM@?$CK?5PollSmartHBAFIBCompletion?3?5wa@FNODOBFM@ 0000000140027520     cmddelivery.obj
 0001:00026550       ??_C@_0FC@DFPAPIBO@?$CK?5?9?9?5SCSIOP_START_STOP_UNIT?3?5Pa@FNODOBFM@ 0000000140027550     cmddelivery.obj
 0001:000265b0       ??_C@_0CP@GPLNGCJB@?$CK?5?9?5Cannot?5start?1stop?5a?5unit?0?5e@FNODOBFM@ 00000001400275b0     cmddelivery.obj
 0001:000265e0       ??_C@_0FM@ENJACBOF@?$CK?5SCSIOP_SYNCHRONIZE_CACHE?$CICDM?$CJ@FNODOBFM@ 00000001400275e0     cmddelivery.obj
 0001:00026640       ??_C@_0GA@MEOEEOJH@?$CK?5SCSIOP_SYNCHRONIZE_CACHE?$CICDM?$CJ@FNODOBFM@ 0000000140027640     cmddelivery.obj
 0001:000266a0       ??_C@_0GO@DFFGFOPL@?$CK?$CK?57?124?5SendFib?3?5Line?5?$CFd?5Outsta@FNODOBFM@ 00000001400276a0     cmddelivery.obj
 0001:00026710       ??_C@_0EI@ELGPOPDD@?$CK?$CK?57?124?5SendFib?3?5Line?5?$CFd?5MsgCap@FNODOBFM@ 0000000140027710     cmddelivery.obj
 0001:00026760       ??_C@_0GF@HHOGHLFF@?$CK?5This?5should?5not?5happen?4?5Srb?5p@FNODOBFM@ 0000000140027760     cmddelivery.obj
 0001:000267d0       ??_C@_0DC@IHNBNMNO@?$CK?$CK?5One?5FIB?5kidnapped?0?5FIB_Conte@FNODOBFM@ 00000001400277d0     cmddelivery.obj
 0001:00026810       ??_C@_0HI@CALKOMHC@?$CK?5SendSynchFib?3?5There?5is?5a?5pend@FNODOBFM@ 0000000140027810     cmddelivery.obj
 0001:00026890       ??_C@_0FM@IHOMFPBM@?$CK?5In?5StartIo?0?5FW?5is?5still?5NOT?5b@FNODOBFM@ 0000000140027890     cmddelivery.obj
 0001:000268f0       ??_C@_0CN@EPOHBMBH@?$CK?5path?5?$CFd?5target?5?$CFd?5reset?5count@FNODOBFM@ 00000001400278f0     cmddelivery.obj
 0001:00026920       ??_C@_0CB@KIAHGGON@?5RESET?5is?5for?5Smart?5HBA?5device?5@FNODOBFM@ 0000000140027920     cmddelivery.obj
 0001:00026950       ??_C@_0BP@PAHACOBL@?$CK?5Got?5path?5?$CFd?5target?5?$CFd?5reset?6@FNODOBFM@ 0000000140027950     cmddelivery.obj
 0001:00026970       ??_C@_0CC@BGHDODBG@?$CK?5SRB_FUNCTION_POWER?3?5action?3?5?$CF@FNODOBFM@ 0000000140027970     cmddelivery.obj
 0001:000269a0       ??_C@_0BP@DFKLHFDI@?$CK?5SRB_FUNCTION_POWER?3?5sleep?51?6@FNODOBFM@ 00000001400279a0     cmddelivery.obj
 0001:000269c0       ??_C@_0DL@PCKMOFFE@?$CK?5SRB_FUNCTION_POWER?3?5coming?5ba@FNODOBFM@ 00000001400279c0     cmddelivery.obj
 0001:00026a00       ??_C@_0CG@NCNALCOB@?$CK?5SRB_FUNCTION_POWER?3?5going?5to?5@FNODOBFM@ 0000000140027a00     cmddelivery.obj
 0001:00026a30       ??_C@_0CA@IBGDOHDE@?$CK?5SRB_FUNCTION_POWER?3?5shutdown?6@FNODOBFM@ 0000000140027a30     cmddelivery.obj
 0001:00026a50       ??_C@_0CD@NOANDIPK@?$CK?5SRB_FUNCTION_POWER?3?5shutdownO@FNODOBFM@ 0000000140027a50     cmddelivery.obj
 0001:00026a80       ??_C@_0BO@KPPCGIPP@?$CK?5SRB_FUNCTION_POWER?3?5reboot?6@FNODOBFM@ 0000000140027a80     cmddelivery.obj
 0001:00026aa0       ??_C@_0BJ@NDPKABON@entering?5AdapterControl?6@FNODOBFM@ 0000000140027aa0     cmdproc.obj
 0001:00026ac0       ??_C@_0CF@FDIANAIH@?$CK?5?9?5AdapterControl?3?5ScsiStopAda@FNODOBFM@ 0000000140027ac0     cmdproc.obj
 0001:00026af0       ??_C@_0FJ@DLLPOCIO@?$CK?5?9?5AdapterControl?3?5ScsiStopAda@FNODOBFM@ 0000000140027af0     cmdproc.obj
 0001:00026b50       ??_C@_0DK@JIECJOFO@?$CK?5Set?5pInitStruct?9?$DONoOfMsiVecto@FNODOBFM@ 0000000140027b50     cmdproc.obj
 0001:00026b90       ??_C@_0HA@BIJAMPMG@?$CK?5?9?5AdapterControl?3?5ScsiSetBoot@FNODOBFM@ 0000000140027b90     cmdproc.obj
 0001:00026c00       ??_C@_0DL@CMAPNHGC@?$CK?5?9?5AdapterControl?3?5ScsiSetBoot@FNODOBFM@ 0000000140027c00     cmdproc.obj
 0001:00026c40       ??_C@_0DI@IPKKLNPP@?$CK?5?9?5AdapterControl?3?5ScsiSetBoot@FNODOBFM@ 0000000140027c40     cmdproc.obj
 0001:00026c80       ??_C@_0HE@CIFLMEO@?$CK?5?9?5AdapterControl?3?5ScsiSetRunn@FNODOBFM@ 0000000140027c80     cmdproc.obj
 0001:00026d00       ??_C@_0CI@NDPGKLNN@?$CK?5?9?5AdapterControl?3?5ScsiRestart@FNODOBFM@ 0000000140027d00     cmdproc.obj
 0001:00026d30       ??_C@_0CM@CNGCOMHH@?$CK?5Before?5checking?5Adapter?5Healt@FNODOBFM@ 0000000140027d30     cmdproc.obj
 0001:00026d60       ??_C@_0BF@GMFKAGLA@?$CK?$CK?5BlinLed?5Code?3?5?$CFx?6@FNODOBFM@ 0000000140027d60     cmdproc.obj
 0001:00026d80       ??_C@_1CE@ENBAPEOO@?$AAB?$AAl?$AAi?$AAn?$AAk?$AAL?$AAE?$AAD?$AA?5?$AAd?$AAe?$AAt?$AAe?$AAc?$AAt@FNODOBFM@ 0000000140027d80     cmdproc.obj
 0001:00026db0       ??_C@_0DM@EBNPFHJD@?$CK?5set?5timer?5to?5check?5the?5FW?5sta@FNODOBFM@ 0000000140027db0     cmdproc.obj
 0001:00026df0       ??_C@_0CM@LGOLDMAP@?$CK?5leaving?5AdapterControl?5Routin@FNODOBFM@ 0000000140027df0     cmdproc.obj
 0001:00026e20       ??_C@_0EF@MIBINBLP@?$CK?5Hw?5Soft?5Reset?5Set?5Timer?0?5leav@FNODOBFM@ 0000000140027e20     cmdproc.obj
 0001:00026e70       ??_C@_0CG@MHIDKAIN@?$CK?5HW?5Soft?5Reset?0?5Set?5Timer?0?5lin@FNODOBFM@ 0000000140027e70     cmdproc.obj
 0001:00026ea0       ??_C@_0IF@DDPMHFDG@?$CK?5SMNormalModeInitAdapter?5faile@FNODOBFM@ 0000000140027ea0     cmdproc.obj
 0001:00026f30       ??_C@_0IE@BILJPPDJ@?$CK?5SMNormalModeInitAdapter?5faile@FNODOBFM@ 0000000140027f30     cmdproc.obj
 0001:00026fc0       ??_C@_0CO@CEANCDOF@?$CK?5?9?5AdapterControl?3?5Reset?5HostR@FNODOBFM@ 0000000140027fc0     cmdproc.obj
 0001:00026ff0       ??_C@_0CN@OHJICFOG@?$CK?5?9?5AdapterControl?3?5ScsiQuery?5w@FNODOBFM@ 0000000140027ff0     cmdproc.obj
 0001:00027020       ??_C@_0DA@CMHNEFAA@?$CK?5?9?5AdapterControl?3?5ScsiQuery?5W@FNODOBFM@ 0000000140028020     cmdproc.obj
 0001:00027050       ??_C@_0DB@DKFDCCOB@?$CK?5Unsupported?5AdapterControl?5co@FNODOBFM@ 0000000140028050     cmdproc.obj
 0001:00027090       ??_C@_0BI@MBKDPNLO@leaving?5AdapterControl?6@FNODOBFM@ 0000000140028090     cmdproc.obj
 0001:000270b0       ??_C@_0EC@JJCHBELF@?$CI?$CFx?0?$CFx?0?$CFx?$CJ?0?5Function?5?$DN?5?$CFx?0?5Opco@FNODOBFM@ 00000001400280b0     cmdproc.obj
 0001:00027100       ??_C@_0EG@JJEEJEDP@?$CI?$CFx?0?$CFx?0?$CFx?$CJ?0?5Function?5?$DN?5?$CFx?0?5Opco@FNODOBFM@ 0000000140028100     cmdproc.obj
 0001:00027150       ??_C@_0CO@NKBJPPMA@?$CK?5buildio?3?5LBA?5OUT?5OF?5RANGE?0?5se@FNODOBFM@ 0000000140028150     cmdproc.obj
 0001:00027180       ??_C@_0FN@LKLFGDKL@?$CK?5buildio?3?5LBA?5OUT?5OF?5RANGE?0?5se@FNODOBFM@ 0000000140028180     cmdproc.obj
 0001:000271e0       ??_C@_0FA@MOKLGDID@?$CK?5buildio?3?5LBA?5OUT?5OF?5RANGE?0?5se@FNODOBFM@ 00000001400281e0     cmdproc.obj
 0001:00027230       ??_C@_0GA@IGOANHED@?$CK?5buildio?3?5LBA?5OUT?5OF?5RANGE?0?5se@FNODOBFM@ 0000000140028230     cmdproc.obj
 0001:00027290       ??_C@_0DM@NPKIKBA@?$CK?5IOP?5RESET?5is?5done?5in?5ProcessI@FNODOBFM@ 0000000140028290     ioctl.obj
 0001:000272d0       ??_C@_0DH@EIBEBELL@?$CK?5ProcessIoctl?3?5HWSoftReset?5lea@FNODOBFM@ 00000001400282d0     ioctl.obj
 0001:00027310       ??_C@_0DL@IOLCNFHG@?$CK?5IOP?5RESET?5failed?5in?5ProcessIo@FNODOBFM@ 0000000140028310     ioctl.obj
 0001:00027350       ??_C@_07MPDDHOMN@CSMIALL@FNODOBFM@ 0000000140028350     ioctl.obj
 0001:00027360       ??_C@_07OODOBGKD@CSMIARY@FNODOBFM@ 0000000140028360     ioctl.obj
 0001:00027370       ??_C@_07PAKBHMBE@CSMISAS@FNODOBFM@ 0000000140028370     ioctl.obj
 0001:00027380       ??_C@_07BHCKAAPP@CSMIPHY@FNODOBFM@ 0000000140028380     ioctl.obj
 0001:00027390       ??_C@_0ED@COAGKFGB@?$CK?5IOP?5RESET?5is?5in?5progress?4?5Rej@FNODOBFM@ 0000000140028390     ioctl.obj
 0001:000273e0       ??_C@_0CF@JOCBDLKJ@?$CK?5Allocate?5big?5IOCTL?5buffer?5fai@FNODOBFM@ 00000001400283e0     ioctl.obj
 0001:00027410       ??_C@_0DF@CHPLNPBM@?$CK?5ProcessIoctl?3?5Internal?5Print?5@FNODOBFM@ 0000000140028410     ioctl.obj
 0001:00027450       ??_C@_0CE@NGAHOGLJ@?$CK?5ProcessIoctl?3?5private?5cdb?8s?5h@FNODOBFM@ 0000000140028450     ioctl.obj
 0001:00027480       ??_C@_0CH@HPKPAOCF@?$CK?5ProcessIoctl?3?5DBG_IO_TRACE?5fl@FNODOBFM@ 0000000140028480     ioctl.obj
 0001:000274b0       ??_C@_0CK@OFFABCEM@?$CK?5ProcessIoctl?3?5DBG_IOCTL_TRACE@FNODOBFM@ 00000001400284b0     ioctl.obj
 0001:000274e0       ??_C@_0CM@CGIIOCGI@?$CK?5ProcessIoctl?3?5DBG_CLUSTER_TRA@FNODOBFM@ 00000001400284e0     ioctl.obj
 0001:00027510       ??_C@_0CI@LPOJHEHM@?$CK?5ProcessIoctl?3?5DBG_ISR_TRACE?5f@FNODOBFM@ 0000000140028510     ioctl.obj
 0001:00027540       ??_C@_0DC@NOLFHCLF@?$CK?5ProcessIoctl?3?5DBG_IO_FUNC_ENT@FNODOBFM@ 0000000140028540     ioctl.obj
 0001:00027580       ??_C@_0DE@PFEFFOBG@?$CK?5ProcessIoctl?3?5DBG_INIT_FUNC_E@FNODOBFM@ 0000000140028580     ioctl.obj
 0001:000275c0       ??_C@_0DF@DPLBBPBM@?$CK?5ProcessIoctl?3?5DBG_IOCTL_FUNC_@FNODOBFM@ 00000001400285c0     ioctl.obj
 0001:00027600       ??_C@_0CL@GAIHEBC@?$CK?5ProcessIoctl?3?5DBG_IO_TRACE?5fl@FNODOBFM@ 0000000140028600     ioctl.obj
 0001:00027630       ??_C@_0CO@NGOEBBKH@?$CK?5ProcessIoctl?3?5DBG_IOCTL_TRACE@FNODOBFM@ 0000000140028630     ioctl.obj
 0001:00027660       ??_C@_0DA@HPMIGAD@?$CK?5ProcessIoctl?3?5DBG_CLUSTER_TRA@FNODOBFM@ 0000000140028660     ioctl.obj
 0001:00027690       ??_C@_0CM@NECMPDIP@?$CK?5ProcessIoctl?3?5DBG_ISR_TRACE?5f@FNODOBFM@ 0000000140028690     ioctl.obj
 0001:000276c0       ??_C@_0DG@PHFPGNCH@?$CK?5ProcessIoctl?3?5DBG_IO_FUNC_ENT@FNODOBFM@ 00000001400286c0     ioctl.obj
 0001:00027700       ??_C@_0DI@CBNGHMLF@?$CK?5ProcessIoctl?3?5DBG_INIT_FUNC_E@FNODOBFM@ 0000000140028700     ioctl.obj
 0001:00027740       ??_C@_0DJ@DEFCHEDB@?$CK?5ProcessIoctl?3?5DBG_IOCTL_FUNC_@FNODOBFM@ 0000000140028740     ioctl.obj
 0001:00027780       ??_C@_0CC@ELKJFKAD@?$CK?5ProcessIoctl?3?5DebugFlags?3?50x?$CF@FNODOBFM@ 0000000140028780     ioctl.obj
 0001:000277b0       ??_C@_0DI@PNEPHAGL@?$CK?5Set?5pInitStruct?9?$DONoOfMsiVecto@FNODOBFM@ 00000001400287b0     ioctl.obj
 0001:000277f0       ??_C@_0DF@KDDHBOCK@?$CK?5when?5back?5from?5IOP_RESET?0?5we?5@FNODOBFM@ 00000001400287f0     ioctl.obj
 0001:00027830       ??_C@_0DO@IBFHJCIJ@?$CK?5IOP?5RESET?5is?5done?5in?5ProcessI@FNODOBFM@ 0000000140028830     ioctl.obj
 0001:00027870       ??_C@_0DN@EJCEJBIF@?$CK?5IOP?5RESET?5failed?5in?5ProcessIo@FNODOBFM@ 0000000140028870     ioctl.obj
 0001:000278b0       ??_C@_0CF@GENCHGED@?$CK?5ProcessIoctl?3?5coalescing?5disa@FNODOBFM@ 00000001400288b0     ioctl.obj
 0001:000278e0       ??_C@_0CE@KOEFFOB@?$CK?5ProcessIoctl?3?5coalescing?5enab@FNODOBFM@ 00000001400288e0     ioctl.obj
 0001:00027910       ??_C@_0GG@KLCLOEBM@?$CK?5ProcessIoctl?3?5Get?5a?5request?5f@FNODOBFM@ 0000000140028910     ioctl.obj
 0001:00027980       ??_C@_0IA@OEPDMML@?$CK?5ProcessIoctl?3?5Get?5a?5request?5f@FNODOBFM@ 0000000140028980     ioctl.obj
 0001:00027a00       ??_C@_0GG@JMGDPGEE@?$CK?5ProcessIoctl?3?5Get?5a?5request?5f@FNODOBFM@ 0000000140028a00     ioctl.obj
 0001:00027a70       ??_C@_0IA@HMGAPIGO@?$CK?5ProcessIoctl?3?5Get?5a?5request?5f@FNODOBFM@ 0000000140028a70     ioctl.obj
 0001:00027af0       ??_C@_0DH@GFOJOHEG@?$CK?5ProcessIoctl?3?5TTYPE_CHANGE_IO@FNODOBFM@ 0000000140028af0     ioctl.obj
 0001:00027b30       ??_C@_0CN@FFFLABJM@?$CK?5ProcessIoctl?3?5AIF?5commands?5pr@FNODOBFM@ 0000000140028b30     ioctl.obj
 0001:00027b60       ??_C@_0CO@EKDJMEJG@?$CK?5ProcessIoctl?3?5AIF?5commands?5pr@FNODOBFM@ 0000000140028b60     ioctl.obj
 0001:00027b90       ??_C@_0CP@DNDOBHJJ@?$CK?5ProcessIoctl?3?5synch?5commands?5@FNODOBFM@ 0000000140028b90     ioctl.obj
 0001:00027bc0       ??_C@_0DA@DKDLFFAP@?$CK?5ProcessIoctl?3?5synch?5commands?5@FNODOBFM@ 0000000140028bc0     ioctl.obj
 0001:00027bf0       ??_C@_0DD@OCMBIILM@?$CK?5ProcessIoctl?3?5RUN_CODE_IN_SPE@FNODOBFM@ 0000000140028bf0     ioctl.obj
 0001:00027c30       ??_C@_0FD@PBJMMHDI@?$CK?5ProcessIoctl?3?5RUN_CODE_IN_SPE@FNODOBFM@ 0000000140028c30     ioctl.obj
 0001:00027c90       ??_C@_0EG@IJGFKELB@?$CK?5ProcessIoctl?3?5bus?$DN?$CFd?0?5target?$DN@FNODOBFM@ 0000000140028c90     ioctl.obj
 0001:00027ce0       ??_C@_0GB@LAAKBHJK@?$CK?5ProcessIoctl?3?5wrong?5parameter@FNODOBFM@ 0000000140028ce0     ioctl.obj
 0001:00027d50       ??_C@_0DA@LCPJHFEI@?$CK?5ProcessIoctl?3?5Max?5Data?5Transf@FNODOBFM@ 0000000140028d50     ioctl.obj
 0001:00027d80       ??_C@_0CE@DJCKDJAF@?$CK?5ProcessIoctl?3?5Max?5SG?5items?3?50@FNODOBFM@ 0000000140028d80     ioctl.obj
 0001:00027db0       ??_C@_0BF@JHMLOOKE@?$CK?5outstanding?5IO?3?$CFd?6@FNODOBFM@ 0000000140028db0     ioctl.obj
 0001:00027dd0       ??_C@_0CK@EPAOGNLF@?$CK?5ProcessIoctl?3?5BUILDIO?5LOOPBAC@FNODOBFM@ 0000000140028dd0     ioctl.obj
 0001:00027e00       ??_C@_0CK@DADBMBLL@?$CK?5ProcessIoctl?3?5STARTIO?5LOOPBAC@FNODOBFM@ 0000000140028e00     ioctl.obj
 0001:00027e30       ??_C@_0CK@BMBGJMJA@?$CK?5ProcessIoctl?3?5PUSHFIB?5LOOPBAC@FNODOBFM@ 0000000140028e30     ioctl.obj
 0001:00027e60       ??_C@_0CL@DANMEPHG@?$CK?5ProcessIoctl?3?5BUILDIO?5LOOPBAC@FNODOBFM@ 0000000140028e60     ioctl.obj
 0001:00027e90       ??_C@_0CL@NHBLFNNN@?$CK?5ProcessIoctl?3?5STARTIO?5LOOPBAC@FNODOBFM@ 0000000140028e90     ioctl.obj
 0001:00027ec0       ??_C@_0CL@HLILIDMA@?$CK?5ProcessIoctl?3?5PUSHFIB?5LOOPBAC@FNODOBFM@ 0000000140028ec0     ioctl.obj
 0001:00027ef0       ??_C@_0DB@MDNCKDFE@?$CK?5ProcessIoctl?3?5Simulate?5SCSI?5s@FNODOBFM@ 0000000140028ef0     ioctl.obj
 0001:00027f30       ??_C@_0EC@KMBGJBEG@?$CK?5ProcessIoctl?3?5Simulate?5FW?5Tar@FNODOBFM@ 0000000140028f30     ioctl.obj
 0001:00027f80       ??_C@_0BI@COAKNOP@?$CK?5?9?5IOCTL?5MESSAGE?3?5?$CFs?5?6@FNODOBFM@ 0000000140028f80     ioctl.obj
 0001:00027fa0       ??_C@_0BP@PHOOCPMJ@?$CK?5?9?5IOCTL?3?5FSAMPCTL_RESET_IOP?6@FNODOBFM@ 0000000140028fa0     ioctl.obj
 0001:00027fc0       ??_C@_0CE@ONNDCLIE@FSAMPCTL_RESET_IOP?5?3?5ResetFlag?5@FNODOBFM@ 0000000140028fc0     ioctl.obj
 0001:00027ff0       ??_C@_0CM@ILCOJJDE@FSAMPCTL_RESET_IOP?3?5IOP?5Reset?5O@FNODOBFM@ 0000000140028ff0     ioctl.obj
 0001:00028020       ??_C@_0CP@PMFIDFBA@?$CK?5IOP?5RESET?5is?5done?5in?5ProcessI@FNODOBFM@ 0000000140029020     ioctl.obj
 0001:00028050       ??_C@_0EB@EJNKCDGF@?$CK?5IOP?5RESET?5failed?5in?5ProcessIo@FNODOBFM@ 0000000140029050     ioctl.obj
 0001:000280a0       ??_C@_0DA@ILCCCIHD@FSAMPCTL_RESET_IOP?3?5HW?5Soft?5Res@FNODOBFM@ 00000001400290a0     ioctl.obj
 0001:000280d0       ??_C@_0DI@EHOOKHPF@?$CK?5when?5back?5from?5HWSOFT_RESET?0?5@FNODOBFM@ 00000001400290d0     ioctl.obj
 0001:00028110       ??_C@_0DN@BHCOMBAH@?$CK?5set?5timer?5to?5check?5the?5FW?5sta@FNODOBFM@ 0000000140029110     ioctl.obj
 0001:00028150       ??_C@_0DD@GMMMAFI@?$CK?5HW?5SOFT?5RESET?5is?5done?5in?5Proc@FNODOBFM@ 0000000140029150     ioctl.obj
 0001:00028190       ??_C@_0DJ@HKOHJJPL@HW?5SOFT?5RESET?5is?5not?5support?4?5I@FNODOBFM@ 0000000140029190     ioctl.obj
 0001:000281d0       ??_C@_0EM@EEFCGCAM@FSAMPCTL_RESET_IOP?3?5IOP?5Reset?5F@FNODOBFM@ 00000001400291d0     ioctl.obj
 0001:00028220       ??_C@_0DC@MOKOJMEO@?$CK?5HW?5IOP?5RESET?5is?5done?5in?5Proce@FNODOBFM@ 0000000140029220     ioctl.obj
 0001:00028260       ??_C@_0EF@IPKPNMPC@?$CK?5HW?5SOFT?5RESET?5failed?5in?5Proce@FNODOBFM@ 0000000140029260     ioctl.obj
 0001:000282b0       ??_C@_0DP@HKHFJHOF@ProcessIoctl?5FSAMPCTL_RESET_IOP@FNODOBFM@ 00000001400292b0     ioctl.obj
 0001:000282f0       ??_C@_0L@BGLGDCOP@archba?4sys@FNODOBFM@ 00000001400292f0     ioctl.obj
 0001:00028300       ??_C@_0CA@HJMENHI@Adaptec?5SAS?5HBA?5Storport?5Driver@FNODOBFM@ 0000000140029300     ioctl.obj
 0001:00028320       ??_C@_0DJ@MIENLJJJ@OMR?5value?5in?5Check?5Adapter?5Heal@FNODOBFM@ 0000000140029320     comm.obj
 0001:00028360       ??_C@_0DB@LCMFMKOG@?$CK?5Event?5array?5FULL?4?5Event?5?$CI?$CFd?$CJ?5@FNODOBFM@ 0000000140029360     comm.obj
 0001:000283a0       ??_C@_0EJ@PCHGGBBF@?$CK?5ProcessAif?3?5request?5timer?5for@FNODOBFM@ 00000001400293a0     comm.obj
 0001:000283f0       ??_C@_0BL@NHJOLJMJ@AIF?5EVENT?5?$CIThor?$CJ?3?5HotPlug?6@FNODOBFM@ 00000001400293f0     comm.obj
 0001:00028410       ??_C@_0CD@EMEGIPDM@AIF?5EVENT?5?$CIThor?$CJ?3?5Hardware?5chan@FNODOBFM@ 0000000140029410     comm.obj
 0001:00028440       ??_C@_0DC@LGHJMKLE@AIF?5EVENT?5?$CIThor?$CJ?3?5Physical?5Devi@FNODOBFM@ 0000000140029440     comm.obj
 0001:00028480       ??_C@_0DB@CEOPCOBC@AIF?5EVENT?5?$CIThor?$CJ?3?5Logical?5Devic@FNODOBFM@ 0000000140029480     comm.obj
 0001:000284c0       ??_C@_0DC@PEAKFMNI@AIF?5EVENT?5?$CIThor?$CJ?3?5FW?5IO?5bypass?5@FNODOBFM@ 00000001400294c0     comm.obj
 0001:00028500       ??_C@_0DK@MABGHGOH@AIF?5EVENT?5?$CIThor?$CJ?3?5FW?5IO?5bypass?5@FNODOBFM@ 0000000140029500     comm.obj
 0001:00028540       ??_C@_0CP@MLBBLAGJ@AIF?5EVENT?5?$CIThor?$CJ?3?5Not?5a?5recogni@FNODOBFM@ 0000000140029540     comm.obj
 0001:00028570       ??_C@_0DL@CJKFCOBN@?$CK?5ProcessAif?3?5request?5timer?5to?5@FNODOBFM@ 0000000140029570     comm.obj
 0001:000285b0       ??_C@_0CH@PCLLKGG@?$CK?5ProcessAif?3?5Physical?5Drives?5s@FNODOBFM@ 00000001400295b0     comm.obj
 0001:000285e0       ??_C@_0DK@NNFHFOND@?$CK?5ProcessAif?3?5request?5timer?5to?5@FNODOBFM@ 00000001400295e0     comm.obj
 0001:00028620       ??_C@_0CG@CDKKDOHL@?$CK?5ProcessAif?3?5Logical?5Drives?5sc@FNODOBFM@ 0000000140029620     comm.obj
 0001:00028650       ??_C@_0CM@GEHGCFFI@?$CK?5ProcessAif?3?5AIF?5cmd?3?5?$CFd?0?5AIF?5@FNODOBFM@ 0000000140029650     comm.obj
 0001:00028680       ??_C@_0CJ@ELNMEDDG@AIF?5EVENT?3?5Container?5?$CD?$CFd?5Morph?5@FNODOBFM@ 0000000140029680     comm.obj
 0001:000286b0       ??_C@_0CF@GOGNODAJ@AIF?5EVENT?3?5a?5RAW?5device?5?$CD?$CFd?5rem@FNODOBFM@ 00000001400296b0     comm.obj
 0001:000286e0       ??_C@_0CL@PFPKJCEB@AIF?5EVENT?3?5AifEnNativeHBADevice@FNODOBFM@ 00000001400296e0     comm.obj
 0001:00028710       ??_C@_0CO@KNHKMPNF@AIF?5EVENT?3?5AifEnNativeHBADevice@FNODOBFM@ 0000000140029710     comm.obj
 0001:00028740       ??_C@_0DD@GCBHPPGK@AIF?5EVENT?3?5Hardware?5not?5present@FNODOBFM@ 0000000140029740     comm.obj
 0001:00028780       ??_C@_0EJ@OLDMFEFC@AIF?5EVENT?3?5Super?5cap?5health?5is?5@FNODOBFM@ 0000000140029780     comm.obj
 0001:000287d0       ??_C@_0DM@BNKBKMII@AIF?5EVENT?3?5Super?5cap?5health?5is?5@FNODOBFM@ 00000001400297d0     comm.obj
 0001:00028810       ??_C@_0BM@DGCCGGOI@AIF?5EVENT?3?5Cache?5data?5loss?6@FNODOBFM@ 0000000140029810     comm.obj
 0001:00028830       ??_C@_0CH@EOEMJJE@AIF?5EVENT?3?5Temperature?5Back?5to?5@FNODOBFM@ 0000000140029830     comm.obj
 0001:00028860       ??_C@_0EA@EGACBNC@AIF?5EVENT?3?5Temperature?5has?5cros@FNODOBFM@ 0000000140029860     comm.obj
 0001:000288a0       ??_C@_0ED@CGHEBKG@AIF?5EVENT?3?5Temperature?5is?5in?5th@FNODOBFM@ 00000001400298a0     comm.obj
 0001:000288f0       ??_C@_0CJ@JLLJHFCM@AIF?5EVENT?3?5Backup?5unit?5self?9tes@FNODOBFM@ 00000001400298f0     comm.obj
 0001:00028920       ??_C@_0CJ@NHDLILDM@AIF?5EVENT?3?5Fatal?5Error?3?5Backup?5@FNODOBFM@ 0000000140029920     comm.obj
 0001:00028950       ??_C@_0CA@GLOIGEIG@AIF?5EVENT?3?5Container?5?$CD?$CFd?5added?6@FNODOBFM@ 0000000140029950     comm.obj
 0001:00028970       ??_C@_0CC@IGLGEBDK@AIF?5EVENT?3?5Container?5?$CD?$CFd?5remove@FNODOBFM@ 0000000140029970     comm.obj
 0001:000289a0       ??_C@_0FE@GFLJPFDG@AIF?5EVENT?3?5AifEnEnclosureManage@FNODOBFM@ 00000001400299a0     comm.obj
 0001:00028a00       ??_C@_0BJ@NJMLAEMO@AIF?5EVENT?3?5a?5JBOD?5added?6@FNODOBFM@ 0000000140029a00     comm.obj
 0001:00028a20       ??_C@_0BL@PDKEFHEM@AIF?5EVENT?3?5a?5JBOD?5removed?6@FNODOBFM@ 0000000140029a20     comm.obj
 0001:00028a40       ??_C@_0DO@DNJOKEFB@AIF?5EVENT?3?5AifCmdJobProgress?5fo@FNODOBFM@ 0000000140029a40     comm.obj
 0001:00028a80       ??_C@_0EM@MHLKFBIP@AIF?5EVENT?3?5AifCmdJobProgress?5fo@FNODOBFM@ 0000000140029a80     comm.obj
 0001:00028ad0       ??_C@_0EO@LMDDDIBO@?$CK?5RestoreBMIC15Srb?3?5QD?5limitati@FNODOBFM@ 0000000140029ad0     comm.obj
 0001:00028b20       ??_C@_0EI@IBBGKNJF@?$CK?5ProcessNormalFib?9Set?5QD?54?5HBA@FNODOBFM@ 0000000140029b20     comm.obj
 0001:00028b70       ??_C@_0CG@IPLFJLPL@Smart?5HBA?5Scsi?5response?5Status?5@FNODOBFM@ 0000000140029b70     comm.obj
 0001:00028ba0       ??_C@_0DO@HNDDHFGA@?5HBA?5Error?5HBA_MODE_DISABLED?5Sr@FNODOBFM@ 0000000140029ba0     comm.obj
 0001:00028be0       ??_C@_0DA@CPGPCCBA@?5HBA?5Error?5code?5?$CFx?5For?5Path?5ID?5@FNODOBFM@ 0000000140029be0     comm.obj
 0001:00028c10       ??_C@_0FA@CPHJLELC@?5HBA?5Error?5SCSI_COMPL_TRANSL_ST@FNODOBFM@ 0000000140029c10     comm.obj
 0001:00028c60       ??_C@_0FE@JFIIIBKF@?5HBA?5Error?5SCSI_COMPL_TRANSL_ST@FNODOBFM@ 0000000140029c60     comm.obj
 0001:00028cc0       ??_C@_0EO@DHIENLOG@?5HBA?5Error?3?5Length?5from?5OS?$CI0x?$CFx@FNODOBFM@ 0000000140029cc0     comm.obj
 0001:00028d10       ??_C@_0HP@ECKDIFKN@?5HBA?5Error?3?5hbaCmd?9?$DOdata_length@FNODOBFM@ 0000000140029d10     comm.obj
 0001:00028d90       ??_C@_0FK@IBAGLEPN@?5HBA?5Error?5SCSI_COMPL_TRANSL_ST@FNODOBFM@ 0000000140029d90     comm.obj
 0001:00028df0       ??_C@_0FJ@DMCDLFNM@?5HBA?5Error?5SCSI_COMPL_TRANSL_ST@FNODOBFM@ 0000000140029df0     comm.obj
 0001:00028e50       ??_C@_0EP@JHLDIODO@?$CK?5NO?5ERROR?5handling?5for?5pHbaRes@FNODOBFM@ 0000000140029e50     comm.obj
 0001:00028ea0       ??_C@_0CG@PJJANG@TMF?5Function?5Completed?5Successf@FNODOBFM@ 0000000140029ea0     comm.obj
 0001:00028ed0       ??_C@_0FJ@OIALMBME@?$CK?5NO?5ERROR?5handling?5for?5pHbaRes@FNODOBFM@ 0000000140029ed0     comm.obj
 0001:00028f30       ??_C@_1BI@BHAHBMFJ@?$AAM?$AAo?$AAf?$AAR?$AAe?$AAs?$AAo?$AAu?$AAr?$AAc?$AAe@FNODOBFM@ 0000000140029f30     wmi.obj
 0002:00000000       __imp_KeQueryPerformanceCounter 000000014002a000     hal:HAL.dll
 0002:00000008       \177HAL_NULL_THUNK_DATA    000000014002a008     hal:HAL.dll
 0002:00000010       __imp_RtlTimeToTimeFields  000000014002a010     ntoskrnl:ntoskrnl.exe
 0002:00000018       __imp_ExSystemTimeToLocalTime 000000014002a018     ntoskrnl:ntoskrnl.exe
 0002:00000020       \177ntoskrnl_NULL_THUNK_DATA 000000014002a020     ntoskrnl:ntoskrnl.exe
 0002:00000028       __imp_StorPortGetPhysicalAddress 000000014002a028     storport:storport.sys
 0002:00000030       __imp_StorPortPause        000000014002a030     storport:storport.sys
 0002:00000038       __imp_StorPortNotification 000000014002a038     storport:storport.sys
 0002:00000040       __imp_StorPortStallExecution 000000014002a040     storport:storport.sys
 0002:00000048       __imp_StorPortDebugPrint   000000014002a048     storport:storport.sys
 0002:00000050       __imp_StorPortExtendedFunction 000000014002a050     storport:storport.sys
 0002:00000058       __imp_StorPortGetDeviceBase 000000014002a058     storport:storport.sys
 0002:00000060       __imp_StorPortResume       000000014002a060     storport:storport.sys
 0002:00000068       __imp_StorPortInitialize   000000014002a068     storport:storport.sys
 0002:00000070       __imp_StorPortFreeDeviceBase 000000014002a070     storport:storport.sys
 0002:00000078       __imp_StorPortGetBusData   000000014002a078     storport:storport.sys
 0002:00000080       __imp_StorPortGetUncachedExtension 000000014002a080     storport:storport.sys
 0002:00000088       __imp_StorPortSetDeviceQueueDepth 000000014002a088     storport:storport.sys
 0002:00000090       __imp_StorPortQuerySystemTime 000000014002a090     storport:storport.sys
 0002:00000098       __imp_StorPortPauseDevice  000000014002a098     storport:storport.sys
 0002:000000a0       __imp_StorPortResumeDevice 000000014002a0a0     storport:storport.sys
 0002:000000a8       __imp_StorPortBusy         000000014002a0a8     storport:storport.sys
 0002:000000b0       __imp_StorPortGetScatterGatherList 000000014002a0b0     storport:storport.sys
 0002:000000b8       \177storport_NULL_THUNK_DATA 000000014002a0b8     storport:storport.sys
 0002:000000c0       __guard_check_icall_fptr   000000014002a0c0     BufferOverflowFastFailK:guard_support.obj
 0002:000000c8       __guard_dispatch_icall_fptr 000000014002a0c8     BufferOverflowFastFailK:guard_support.obj
 0002:000000d0       __guard_fids_table         000000014002a0d0     <linker-defined>
 0002:00000180       RevCompareTable            000000014002a180     revision.obj
 0002:00000280       RevCompareTableLength      000000014002a280     revision.obj
 0002:00000288       WPP_ThisDir_CTLGUID_archba 000000014002a288     arcdebug.obj
 0002:00000298       WPP_564d9f83b95836092d7383fb0050d933_Traceguids 000000014002a298     arcdebug.obj
 0002:000002a8       ??_C@_08HNOCAICB@Adaptec?5@ 000000014002a2a8     archba.obj
 0002:000002b4       ??_C@_04ODJNANJC@9005@     000000014002a2b4     archba.obj
 0002:000002bc       ??_C@_04EKJHPGNA@0285@     000000014002a2bc     archba.obj
 0002:000002c4       ??_C@_04GBLKKFBD@0286@     000000014002a2c4     archba.obj
 0002:000002cc       ??_C@_04PPDJIIJN@0288@     000000014002a2cc     archba.obj
 0002:000002d4       ??_C@_04LPGNDNED@028b@     000000014002a2d4     archba.obj
 0002:000002dc       ??_C@_04KGHGAMAC@028c@     000000014002a2dc     archba.obj
 0002:000002e4       ??_C@_04OJDHJKMF@028d@     000000014002a2e4     archba.obj
 0002:000002f0       ??_C@_0BB@BOPAMEAE@ARC?9HBA?5?5?5?5?5?5?5?5?5@ 000000014002a2f0     archba.obj
 0002:00000304       ??_C@_06DFBHEALI@AACAPI@   000000014002a304     archba.obj
 0002:00000310       ??_C@_1BK@EPHGJNJ@?$AAS?$AAc?$AAs?$AAi?$AAM?$AAi?$AAn?$AAi?$AAP?$AAo?$AAr?$AAt?$AA?$AA@ 000000014002a310     scsiwmi:wmilib.obj
 0002:00000370       _load_config_used          000000014002a370     BufferOverflowFastFailK:loadcfg.obj
 0003:00000000       WPP_GLOBAL_Control         000000014002c000     arcdebug.obj
 0003:00000008       gDebugFlags                000000014002c008     arcdebug.obj
 0003:00000010       gNativeModeAdapters        000000014002c010     archba.obj
 0003:00000340       gNumNativeModeAdapters     000000014002c340     archba.obj
 0003:00000344       gARCOEMFlags               000000014002c344     archba.obj
 0003:00000348       gARCProductId              000000014002c348     archba.obj
 0003:00000350       gARCApiId                  000000014002c350     archba.obj
 0003:00000360       gARCSASRxSubsystemInfo     000000014002c360     archba.obj
 0003:00000670       gARCSASRktSubsystemInfo    000000014002c670     archba.obj
 0003:000006e0       gARCSASArkSubsystemInfo    000000014002c6e0     archba.obj
 0003:00000710       gARCSASPMCSubsystemInfo    000000014002c710     archba.obj
 0003:00000a30       gARCVendor                 000000014002ca30     arcinit.obj
 0003:00000a38       gAdapterGuid               000000014002ca38     wmi.obj
 0003:00000a48       gIoChannelGuid             000000014002ca48     wmi.obj
 0003:00000a58       gDiskArrayGuid             000000014002ca58     wmi.obj
 0003:00000a68       gPhysicalDiskGuid          000000014002ca68     wmi.obj
 0003:00000a78       gAdapterMethodGuid         000000014002ca78     wmi.obj
 0003:00000a90       __security_cookie          000000014002ca90     BufferOverflowFastFailK:gs_support.obj
 0003:00000a98       __security_cookie_complement 000000014002ca98     BufferOverflowFastFailK:gs_support.obj
 0003:00000ad0       gAdapterAddCount           000000014002cad0     arcinit.obj
 0003:00000ad4       gLatency                   000000014002cad4     arcinit.obj
 0003:00000ad8       gLoopbackInPushFib         000000014002cad8     arcinit.obj
 0003:00000ae0       gTraceContext              000000014002cae0     arcinit.obj
 0003:00000b80       gAdapterTable              000000014002cb80     <common>
 0003:00000d80       gDriverObject              000000014002cd80     <common>
 0003:00000da0       WPP_MAIN_CB                000000014002cda0     <common>
 0005:00000000       GsDriverEntry              000000014002e000 f   BufferOverflowFastFailK:gs_driverentry.obj
 0005:0000002c       __security_init_cookie     000000014002e02c f   BufferOverflowFastFailK:gs_support.obj
 0005:0000005c       __IMPORT_DESCRIPTOR_ntoskrnl 000000014002e05c     ntoskrnl:ntoskrnl.exe
 0005:00000070       __IMPORT_DESCRIPTOR_HAL    000000014002e070     hal:HAL.dll
 0005:00000084       __IMPORT_DESCRIPTOR_storport 000000014002e084     storport:storport.sys
 0005:00000098       __NULL_IMPORT_DESCRIPTOR   000000014002e098     ntoskrnl:ntoskrnl.exe

 entry point at        0005:00000000

 Static symbols

 0002:fffd5fff       __guard_fids__guard_icall_checks_enforced 000000023fffffff     BufferOverflowFastFailK:guard_support.obj
 0002:fffd5fff       __guard_fids__             000000023fffffff     BufferOverflowFastFailK:guard_support.obj
 0000:fffce000       .debug$S                   0000000140000000     storport:storport.sys
 0002:fffd6000       __guard_fids_UpdateThorHBAMappingTable 0000000140000000     timer.obj
 0002:fffd6000       __guard_fids_RequestTimer  0000000140000000     timer.obj
 0002:fffd6000       __guard_fids_WppInitKm     0000000140000000     arcinit.obj
 0002:fffd6000       __guard_fids__             0000000140000000     archba.obj
 0002:fffd6000       __guard_fids_InitializeWmiInterface 0000000140000000     wmi.obj
 0002:fffd6000       __guard_fids_InitializeDPCs 0000000140000000     arcinit.obj
 0002:fffd6000       __guard_fids_FindAdapter   0000000140000000     arcinit.obj
 0002:fffd6000       __guard_fids_HwInitializeAdapter 0000000140000000     arcinit.obj
 0002:fffd6000       __guard_fids_DriverEntry   0000000140000000     arcinit.obj
 0000:fffce000       .debug$S                   0000000140000000     ntoskrnl:ntoskrnl.exe
 0000:fffce000       .debug$S                   0000000140000000     ntoskrnl:ntoskrnl.exe
 0000:fffce000       .debug$S                   0000000140000000     storport:storport.sys
 0000:fffce000       .debug$S                   0000000140000000     storport:storport.sys
 0000:fffce000       .debug$S                   0000000140000000     storport:storport.sys
 0000:fffce000       .debug$S                   0000000140000000     storport:storport.sys
 0000:fffce000       .debug$S                   0000000140000000     storport:storport.sys
 0000:fffce000       .debug$S                   0000000140000000     storport:storport.sys
 0000:fffce000       .debug$S                   0000000140000000     storport:storport.sys
 0000:fffce000       .debug$S                   0000000140000000     storport:storport.sys
 0000:fffce000       .debug$S                   0000000140000000     storport:storport.sys
 0000:fffce000       .debug$S                   0000000140000000     storport:storport.sys
 0000:fffce000       .debug$S                   0000000140000000     storport:storport.sys
 0000:fffce000       .debug$S                   0000000140000000     storport:storport.sys
 0000:fffce000       .debug$S                   0000000140000000     storport:storport.sys
 0000:fffce000       .debug$S                   0000000140000000     storport:storport.sys
 0000:fffce000       .debug$S                   0000000140000000     storport:storport.sys
 0000:fffce000       .debug$S                   0000000140000000     storport:storport.sys
 0000:fffce000       .debug$S                   0000000140000000     storport:storport.sys
 0000:fffce000       .debug$S                   0000000140000000     storport:storport.sys
 0000:fffce000       .debug$S                   0000000140000000     hal:HAL.dll
 0001:00001d80       $LN72                      0000000140002d80     rxdevice.obj
 0001:00004c44       $LN194                     0000000140005c44     arcdebug.obj
 0001:00004c5c       $LN193                     0000000140005c5c     arcdebug.obj
 0001:00008fa0       $LN14                      0000000140009fa0     arcinit.obj
 0001:0000fa98       $LN43                      0000000140010a98     arcinit.obj
 0001:0000ff60       $LN67                      0000000140010f60     arcinit.obj
 0001:000108bc       $LN231                     00000001400118bc     arcinit.obj
 0001:00010d90       $LN125                     0000000140011d90     arcinit.obj
 0001:00011484       $LN319                     0000000140012484     arcinit.obj
 0001:000123dc       $LN71                      00000001400133dc     arcinit.obj
 0001:00013fe0       $LN132                     0000000140014fe0     cmddelivery.obj
 0001:00014008       $LN131                     0000000140015008     cmddelivery.obj
 0001:000140a4       $LN130                     00000001400150a4     cmddelivery.obj
 0001:000140c8       $LN129                     00000001400150c8     cmddelivery.obj
 0001:000158f4       $LN157                     00000001400168f4     cmddelivery.obj
 0001:0001590c       $LN156                     000000014001690c     cmddelivery.obj
 0001:000172e4       $LN192                     00000001400182e4     cmdproc.obj
 0001:000172fc       $LN191                     00000001400182fc     cmdproc.obj
 0001:00017324       $LN190                     0000000140018324     cmdproc.obj
 0001:00017334       $LN189                     0000000140018334     cmdproc.obj
 0001:00019928       $LN102                     000000014001a928     ioctl.obj
 0001:0001c20c       $LN381                     000000014001d20c     ioctl.obj
 0001:0001c24c       $LN380                     000000014001d24c     ioctl.obj
 0001:0001ceb8       $LN130                     000000014001deb8     comm.obj
 0001:0001ced8       $LN129                     000000014001ded8     comm.obj
 0001:0001cf00       $LN128                     000000014001df00     comm.obj
 0001:0001d4a4       $LN34                      000000014001e4a4     comm.obj
 0001:0001d4c0       $LN33                      000000014001e4c0     comm.obj
 0001:0001eac0       $$000000                   000000014001fac0     BufferOverflowFastFailK:amdsecgs.obj
 0001:0001f290       $$000000                   0000000140020290     BufferOverflowFastFailK:guard_dispatch.obj
 0001:0001f2c0       $$000000                   00000001400202c0     ntoskrnl:memcpy.obj
 0001:0001f600       $$000000                   0000000140020600     ntoskrnl:memset.obj
 0002:00000628       $unwind$RxCheckAdapterHealth 000000014002a628     rxdevice.obj
 0002:00000634       $unwind$RxNewCommProcessInterrupt 000000014002a634     rxdevice.obj
 0002:0000064c       $chain$0$RxNewCommProcessInterrupt 000000014002a64c     rxdevice.obj
 0002:00000660       $chain$3$RxNewCommProcessInterrupt 000000014002a660     rxdevice.obj
 0002:0000067c       $chain$4$RxNewCommProcessInterrupt 000000014002a67c     rxdevice.obj
 0002:0000067c       $chain$6$RxNewCommProcessInterrupt 000000014002a67c     rxdevice.obj
 0002:00000690       $chain$5$RxNewCommProcessInterrupt 000000014002a690     rxdevice.obj
 0002:000006ac       $chain$7$RxNewCommProcessInterrupt 000000014002a6ac     rxdevice.obj
 0002:000006c0       $unwind$RxInterruptHandler 000000014002a6c0     rxdevice.obj
 0002:000006d0       $chain$0$RxInterruptHandler 000000014002a6d0     rxdevice.obj
 0002:000006e8       $chain$4$RxInterruptHandler 000000014002a6e8     rxdevice.obj
 0002:000006e8       $chain$2$RxInterruptHandler 000000014002a6e8     rxdevice.obj
 0002:000006e8       $chain$6$RxInterruptHandler 000000014002a6e8     rxdevice.obj
 0002:00000700       $chain$8$RxInterruptHandler 000000014002a700     rxdevice.obj
 0002:00000714       $chain$9$RxInterruptHandler 000000014002a714     rxdevice.obj
 0002:00000728       $unwind$NonMSIXInterruptHandler 000000014002a728     rxdevice.obj
 0002:0000073c       $chain$3$NonMSIXInterruptHandler 000000014002a73c     rxdevice.obj
 0002:0000075c       $chain$4$NonMSIXInterruptHandler 000000014002a75c     rxdevice.obj
 0002:00000770       $unwind$PMCDpcResponseHandler 000000014002a770     rxdevice.obj
 0002:0000077c       $chain$5$PMCDpcResponseHandler 000000014002a77c     rxdevice.obj
 0002:000007a4       $chain$6$PMCDpcResponseHandler 000000014002a7a4     rxdevice.obj
 0002:000007b8       $chain$8$PMCDpcResponseHandler 000000014002a7b8     rxdevice.obj
 0002:000007cc       $chain$9$PMCDpcResponseHandler 000000014002a7cc     rxdevice.obj
 0002:000007e0       $unwind$PMCInterruptHandler 000000014002a7e0     rxdevice.obj
 0002:000007f0       $chain$2$PMCInterruptHandler 000000014002a7f0     rxdevice.obj
 0002:0000080c       $chain$3$PMCInterruptHandler 000000014002a80c     rxdevice.obj
 0002:00000824       $unwind$RxPullMessageUnitQueueCompletedFib 000000014002a824     rxdevice.obj
 0002:00000840       $chain$1$RxPullMessageUnitQueueCompletedFib 000000014002a840     rxdevice.obj
 0002:00000858       $chain$2$RxPullMessageUnitQueueCompletedFib 000000014002a858     rxdevice.obj
 0002:0000086c       $unwind$RxPushMessageUnitQueueFib 000000014002a86c     rxdevice.obj
 0002:0000087c       $chain$0$RxPushMessageUnitQueueFib 000000014002a87c     rxdevice.obj
 0002:00000890       $chain$1$RxPushMessageUnitQueueFib 000000014002a890     rxdevice.obj
 0002:000008a4       $unwind$PMCPushMessageUnitQueueFib 000000014002a8a4     rxdevice.obj
 0002:000008b0       $chain$0$PMCPushMessageUnitQueueFib 000000014002a8b0     rxdevice.obj
 0002:000008c4       $chain$1$PMCPushMessageUnitQueueFib 000000014002a8c4     rxdevice.obj
 0002:000008dc       $chain$2$PMCPushMessageUnitQueueFib 000000014002a8dc     rxdevice.obj
 0002:000008f0       $unwind$RxSendSynchCommand 000000014002a8f0     rxdevice.obj
 0002:0000090c       $unwind$RxStartAdapter     000000014002a90c     rxdevice.obj
 0002:00000928       $unwind$RxWaitForAdapterToBoot 000000014002a928     rxdevice.obj
 0002:00000934       $chain$0$RxWaitForAdapterToBoot 000000014002a934     rxdevice.obj
 0002:0000094c       $chain$1$RxWaitForAdapterToBoot 000000014002a94c     rxdevice.obj
 0002:00000960       $unwind$DumpHandles        000000014002a960     rxdevice.obj
 0002:00000960       $unwind$DumpHandlesZeroPointer 000000014002a960     rxdevice.obj
 0002:0000097c       $unwind$RevCheckCompatibility 000000014002a97c     revision.obj
 0002:0000098c       $unwind$GetDriverParameter 000000014002a98c     helpers.obj
 0002:000009a8       $unwind$MatchRegistryString 000000014002a9a8     helpers.obj
 0002:000009b8       $unwind$LongToAscii        000000014002a9b8     helpers.obj
 0002:000009c8       $chain$0$LongToAscii       000000014002a9c8     helpers.obj
 0002:000009dc       $chain$1$LongToAscii       000000014002a9dc     helpers.obj
 0002:000009f0       $unwind$CompareStrings     000000014002a9f0     helpers.obj
 0002:000009fc       $unwind$StorWmiTraceMessage 000000014002a9fc     arcdebug.obj
 0002:00000a08       $unwind$ArcPrintf          000000014002aa08     arcdebug.obj
 0002:00000a20       $chain$1$ArcPrintf         000000014002aa20     arcdebug.obj
 0002:00000a38       $chain$2$ArcPrintf         000000014002aa38     arcdebug.obj
 0002:00000a4c       $chain$3$ArcPrintf         000000014002aa4c     arcdebug.obj
 0002:00000a60       $chain$4$ArcPrintf         000000014002aa60     arcdebug.obj
 0002:00000a70       $chain$5$ArcPrintf         000000014002aa70     arcdebug.obj
 0002:00000a80       $chain$6$ArcPrintf         000000014002aa80     arcdebug.obj
 0002:00000a94       $unwind$WPP_SF_s           000000014002aa94     arcdebug.obj
 0002:00000aa0       $unwind$RealSprintf        000000014002aaa0     arcdebug.obj
 0002:00000ab0       $chain$1$RealSprintf       000000014002aab0     arcdebug.obj
 0002:00000ac8       $chain$6$RealSprintf       000000014002aac8     arcdebug.obj
 0002:00000aec       $chain$7$RealSprintf       000000014002aaec     arcdebug.obj
 0002:00000afc       $chain$8$RealSprintf       000000014002aafc     arcdebug.obj
 0002:00000b10       $unwind$MainTimeThread     000000014002ab10     timer.obj
 0002:00000b28       $chain$4$MainTimeThread    000000014002ab28     timer.obj
 0002:00000b4c       $chain$7$MainTimeThread    000000014002ab4c     timer.obj
 0002:00000b4c       $chain$5$MainTimeThread    000000014002ab4c     timer.obj
 0002:00000b6c       $chain$6$MainTimeThread    000000014002ab6c     timer.obj
 0002:00000b90       $chain$8$MainTimeThread    000000014002ab90     timer.obj
 0002:00000ba4       $chain$9$MainTimeThread    000000014002aba4     timer.obj
 0002:00000bb8       $unwind$VMCloseAllCompletionTimer 000000014002abb8     timer.obj
 0002:00000bc4       $chain$0$VMCloseAllCompletionTimer 000000014002abc4     timer.obj
 0002:00000bdc       $chain$1$VMCloseAllCompletionTimer 000000014002abdc     timer.obj
 0002:00000bf0       $unwind$UpdateThorHBAMappingTable 000000014002abf0     timer.obj
 0002:00000c00       $chain$0$UpdateThorHBAMappingTable 000000014002ac00     timer.obj
 0002:00000c14       $chain$2$UpdateThorHBAMappingTable 000000014002ac14     timer.obj
 0002:00000c2c       $chain$3$UpdateThorHBAMappingTable 000000014002ac2c     timer.obj
 0002:00000c3c       $chain$4$UpdateThorHBAMappingTable 000000014002ac3c     timer.obj
 0002:00000c50       $unwind$Reset_IOP_CompletionTimer 000000014002ac50     timer.obj
 0002:00000c5c       $chain$0$Reset_IOP_CompletionTimer 000000014002ac5c     timer.obj
 0002:00000c74       $chain$2$Reset_IOP_CompletionTimer 000000014002ac74     timer.obj
 0002:00000c8c       $chain$4$Reset_IOP_CompletionTimer 000000014002ac8c     timer.obj
 0002:00000ca0       $chain$5$Reset_IOP_CompletionTimer 000000014002aca0     timer.obj
 0002:00000cb4       $unwind$StopTimer          000000014002acb4     timer.obj
 0002:00000cc8       $unwind$RequestTimer       000000014002acc8     timer.obj
 0002:00000ce0       $unwind$CheckingFWAfterPowerStateChange 000000014002ace0     timer.obj
 0002:00000cf0       $chain$0$CheckingFWAfterPowerStateChange 000000014002acf0     timer.obj
 0002:00000d08       $chain$3$CheckingFWAfterPowerStateChange 000000014002ad08     timer.obj
 0002:00000d20       $chain$4$CheckingFWAfterPowerStateChange 000000014002ad20     timer.obj
 0002:00000d34       $unwind$DriverEntry        000000014002ad34     arcinit.obj
 0002:00000d4c       $chain$0$DriverEntry       000000014002ad4c     arcinit.obj
 0002:00000d60       $chain$1$DriverEntry       000000014002ad60     arcinit.obj
 0002:00000d74       $unwind$HwInitializeAdapter 000000014002ad74     arcinit.obj
 0002:00000d9c       $unwind$FindAdapter        000000014002ad9c     arcinit.obj
 0002:00000db8       $chain$1$FindAdapter       000000014002adb8     arcinit.obj
 0002:00000dd0       $chain$2$FindAdapter       000000014002add0     arcinit.obj
 0002:00000de4       $unwind$ResetAdapter       000000014002ade4     arcinit.obj
 0002:00000df8       $chain$5$ResetAdapter      000000014002adf8     arcinit.obj
 0002:00000e20       $chain$6$ResetAdapter      000000014002ae20     arcinit.obj
 0002:00000e34       $unwind$SMNormalModeInitAdapter 000000014002ae34     arcinit.obj
 0002:00000e40       $chain$1$SMNormalModeInitAdapter 000000014002ae40     arcinit.obj
 0002:00000e58       $chain$2$SMNormalModeInitAdapter 000000014002ae58     arcinit.obj
 0002:00000e6c       $unwind$InitializeDPCs     000000014002ae6c     arcinit.obj
 0002:00000e80       $chain$1$InitializeDPCs    000000014002ae80     arcinit.obj
 0002:00000e98       $chain$2$InitializeDPCs    000000014002ae98     arcinit.obj
 0002:00000eac       $unwind$ReturningLocalOutstandingRequestsToOS 000000014002aeac     arcinit.obj
 0002:00000eac       $unwind$HWSoftReset        000000014002aeac     arcinit.obj
 0002:00000ebc       $unwind$CleanHostSideRRQ   000000014002aebc     arcinit.obj
 0002:00000ec8       $unwind$EventTracingCleanup 000000014002aec8     arcinit.obj
 0002:00000ec8       $unwind$ScsiPortWmiPostProcess 000000014002aec8     scsiwmi:wmilib.obj
 0002:00000ed4       $unwind$AllocateConsumerProducerCommArea 000000014002aed4     arcinit.obj
 0002:00000ef0       $unwind$AllocateMessageUnitQueueCommArea 000000014002aef0     arcinit.obj
 0002:00000f0c       $unwind$ConfigureContainersRuntime 000000014002af0c     arcinit.obj
 0002:00000f30       $chain$0$ConfigureContainersRuntime 000000014002af30     arcinit.obj
 0002:00000f44       $chain$1$ConfigureContainersRuntime 000000014002af44     arcinit.obj
 0002:00000f54       $unwind$SendEvent2OSDelayed 000000014002af54     arcinit.obj
 0002:00000f6c       $unwind$GetElapsedSeconds  000000014002af6c     arcinit.obj
 0002:00000f6c       $unwind$HwScsiWmiExecuteMethod 000000014002af6c     wmi.obj
 0002:00000f6c       $unwind$GsDriverEntry      000000014002af6c     BufferOverflowFastFailK:gs_driverentry.obj
 0002:00000f7c       $unwind$IsAdapterReadyForConfigCommand 000000014002af7c     arcinit.obj
 0002:00000f7c       $unwind$HandleAdapterGetConfig 000000014002af7c     arcinit.obj
 0002:00000f7c       $unwind$HandleAdapterCommitConfig 000000014002af7c     arcinit.obj
 0002:00000f7c       $unwind$HandleAdapterConfigIssues 000000014002af7c     arcinit.obj
 0002:00000f94       $unwind$CheckMSIxPossibility 000000014002af94     arcinit.obj
 0002:00000f9c       $chain$0$CheckMSIxPossibility 000000014002af9c     arcinit.obj
 0002:00000fb0       $chain$1$CheckMSIxPossibility 000000014002afb0     arcinit.obj
 0002:00000fc4       $chain$2$CheckMSIxPossibility 000000014002afc4     arcinit.obj
 0002:00000fdc       $chain$3$CheckMSIxPossibility 000000014002afdc     arcinit.obj
 0002:00000ff0       $unwind$SendInitStructure  000000014002aff0     arcinit.obj
 0002:00001008       $unwind$InitializeConsumerProducerCommRegion 000000014002b008     arcinit.obj
 0002:0000101c       $unwind$MapDeviceBase      000000014002b01c     arcinit.obj
 0002:00001038       $unwind$IOPReset           000000014002b038     arcinit.obj
 0002:00001054       $unwind$DumpFibsSentToFW60SecondsBefore 000000014002b054     arcinit.obj
 0002:00001060       $chain$4$DumpFibsSentToFW60SecondsBefore 000000014002b060     arcinit.obj
 0002:00001084       $chain$5$DumpFibsSentToFW60SecondsBefore 000000014002b084     arcinit.obj
 0002:00001098       $unwind$ReturningOutstandingSentToFWBeforeIOPResetToOS 000000014002b098     arcinit.obj
 0002:000010a4       $chain$3$ReturningOutstandingSentToFWBeforeIOPResetToOS 000000014002b0a4     arcinit.obj
 0002:000010c4       $chain$4$ReturningOutstandingSentToFWBeforeIOPResetToOS 000000014002b0c4     arcinit.obj
 0002:000010d8       $chain$5$ReturningOutstandingSentToFWBeforeIOPResetToOS 000000014002b0d8     arcinit.obj
 0002:000010e8       $chain$6$ReturningOutstandingSentToFWBeforeIOPResetToOS 000000014002b0e8     arcinit.obj
 0002:000010fc       $unwind$ReturnOutstandingFibOnTargetDevice 000000014002b0fc     arcinit.obj
 0002:0000110c       $chain$2$ReturnOutstandingFibOnTargetDevice 000000014002b10c     arcinit.obj
 0002:00001128       $chain$3$ReturnOutstandingFibOnTargetDevice 000000014002b128     arcinit.obj
 0002:0000113c       $chain$4$ReturnOutstandingFibOnTargetDevice 000000014002b13c     arcinit.obj
 0002:0000114c       $chain$5$ReturnOutstandingFibOnTargetDevice 000000014002b14c     arcinit.obj
 0002:00001160       $unwind$SetFwTime          000000014002b160     arcinit.obj
 0002:00001178       $chain$0$SetFwTime         000000014002b178     arcinit.obj
 0002:0000118c       $chain$4$SetFwTime         000000014002b18c     arcinit.obj
 0002:000011ac       $chain$5$SetFwTime         000000014002b1ac     arcinit.obj
 0002:000011c4       $chain$6$SetFwTime         000000014002b1c4     arcinit.obj
 0002:000011d4       $chain$7$SetFwTime         000000014002b1d4     arcinit.obj
 0002:000011e8       $unwind$SetArcsasFwTime    000000014002b1e8     arcinit.obj
 0002:000011f8       $unwind$SetPciSlotNumber   000000014002b1f8     arcinit.obj
 0002:0000120c       $unwind$SendWellnessCmnd   000000014002b20c     arcinit.obj
 0002:00001228       $unwind$GetThorHbaPhyDevInfo 000000014002b228     arcinit.obj
 0002:00001244       $unwind$ArcLogEventString  000000014002b244     arcinit.obj
 0002:00001250       $unwind$LogSystemEvent     000000014002b250     arcinit.obj
 0002:0000125c       $unwind$SendEvent2OS       000000014002b25c     arcinit.obj
 0002:0000127c       $unwind$WppTraceCallback   000000014002b27c     arcinit.obj
 0002:00001290       $chain$0$WppTraceCallback  000000014002b290     arcinit.obj
 0002:000012a4       $chain$1$WppTraceCallback  000000014002b2a4     arcinit.obj
 0002:000012b8       $unwind$DynamicallyThrottleLunQueueDepth 000000014002b2b8     arcinit.obj
 0002:000012d8       $unwind$SA4StatusBatching  000000014002b2d8     arcinit.obj
 0002:000012e8       $unwind$SA4ACI2Interface   000000014002b2e8     arcinit.obj
 0002:000012f8       $unwind$SMCrashDumpModeInitAdapter 000000014002b2f8     arcinit.obj
 0002:00001310       $unwind$SendEvent2OSChild  000000014002b310     arcinit.obj
 0002:0000132c       $unwind$StartIo            000000014002b32c     cmddelivery.obj
 0002:00001348       $chain$0$StartIo           000000014002b348     cmddelivery.obj
 0002:0000135c       $chain$1$StartIo           000000014002b35c     cmddelivery.obj
 0002:00001370       $unwind$PostProcessScsiCommand 000000014002b370     cmddelivery.obj
 0002:00001388       $unwind$SendFib            000000014002b388     cmddelivery.obj
 0002:000013a4       $unwind$HandleMSIXInterrupt 000000014002b3a4     cmddelivery.obj
 0002:000013b4       $unwind$QueueRawIoReadWriteRequest 000000014002b3b4     cmddelivery.obj
 0002:000013c8       $chain$0$QueueRawIoReadWriteRequest 000000014002b3c8     cmddelivery.obj
 0002:000013dc       $chain$1$QueueRawIoReadWriteRequest 000000014002b3dc     cmddelivery.obj
 0002:000013f0       $unwind$CompleteQueuedRequest 000000014002b3f0     cmddelivery.obj
 0002:00001404       $unwind$DequeueRawIoReadWriteRequest 000000014002b404     cmddelivery.obj
 0002:00001418       $chain$0$DequeueRawIoReadWriteRequest 000000014002b418     cmddelivery.obj
 0002:0000142c       $chain$1$DequeueRawIoReadWriteRequest 000000014002b42c     cmddelivery.obj
 0002:00001440       $unwind$ProcessContainerInquiry 000000014002b440     cmddelivery.obj
 0002:00001460       $unwind$ProcessScsiCommand 000000014002b460     cmddelivery.obj
 0002:00001488       $unwind$QueuePrintf        000000014002b488     cmddelivery.obj
 0002:0000149c       $unwind$SendRawIoFib       000000014002b49c     cmddelivery.obj
 0002:000014ac       $chain$2$SendRawIoFib      000000014002b4ac     cmddelivery.obj
 0002:000014cc       $chain$4$SendRawIoFib      000000014002b4cc     cmddelivery.obj
 0002:000014e8       $chain$5$SendRawIoFib      000000014002b4e8     cmddelivery.obj
 0002:000014fc       $unwind$SendSynchFib       000000014002b4fc     cmddelivery.obj
 0002:00001514       $chain$0$SendSynchFib      000000014002b514     cmddelivery.obj
 0002:00001528       $chain$1$SendSynchFib      000000014002b528     cmddelivery.obj
 0002:0000153c       $unwind$DequeueCertainLD   000000014002b53c     cmddelivery.obj
 0002:00001550       $chain$0$DequeueCertainLD  000000014002b550     cmddelivery.obj
 0002:00001564       $chain$1$DequeueCertainLD  000000014002b564     cmddelivery.obj
 0002:00001578       $unwind$PollSmartHBAFIBCompletion 000000014002b578     cmddelivery.obj
 0002:00001594       $unwind$AdapterControl     000000014002b594     cmdproc.obj
 0002:000015a8       $unwind$BuildIo            000000014002b5a8     cmdproc.obj
 0002:000015cc       $unwind$BuildHBAFib        000000014002b5cc     cmdproc.obj
 0002:000015e8       $unwind$BuildRawIoFib      000000014002b5e8     cmdproc.obj
 0002:00001600       $unwind$BuildRawIoScatterGather 000000014002b600     cmdproc.obj
 0002:00001618       $chain$0$BuildRawIoScatterGather 000000014002b618     cmdproc.obj
 0002:0000162c       $chain$1$BuildRawIoScatterGather 000000014002b62c     cmdproc.obj
 0002:00001640       $chain$2$BuildRawIoScatterGather 000000014002b640     cmdproc.obj
 0002:00001654       $chain$3$BuildRawIoScatterGather 000000014002b654     cmdproc.obj
 0002:00001664       $unwind$BuildRawIo2ScatterGather 000000014002b664     cmdproc.obj
 0002:00001684       $unwind$ConvertRawIo2ScatterGather 000000014002b684     cmdproc.obj
 0002:00001690       $chain$1$ConvertRawIo2ScatterGather 000000014002b690     cmdproc.obj
 0002:000016a8       $chain$3$ConvertRawIo2ScatterGather 000000014002b6a8     cmdproc.obj
 0002:000016c0       $chain$4$ConvertRawIo2ScatterGather 000000014002b6c0     cmdproc.obj
 0002:000016d0       $chain$5$ConvertRawIo2ScatterGather 000000014002b6d0     cmdproc.obj
 0002:000016e4       $unwind$BuildReadWriteFib  000000014002b6e4     cmdproc.obj
 0002:00001700       $unwind$BuildScatterGather 000000014002b700     cmdproc.obj
 0002:00001700       $unwind$BuildScatterGather64 000000014002b700     cmdproc.obj
 0002:00001700       $unwind$SendConsumerProducerFib 000000014002b700     comm.obj
 0002:0000171c       $unwind$BuildRawIo2ScatterGather4HBAIoctl 000000014002b71c     cmdproc.obj
 0002:00001738       $unwind$BuildHBAIoctlFib   000000014002b738     cmdproc.obj
 0002:00001754       $unwind$BuildSrbFib        000000014002b754     cmdproc.obj
 0002:00001770       $unwind$InitializeFib      000000014002b770     cmdproc.obj
 0002:0000177c       $unwind$PrepareBMIC15      000000014002b77c     cmdproc.obj
 0002:00001798       $unwind$ProcessIoctl       000000014002b798     ioctl.obj
 0002:000017c0       $unwind$BuildRawScatterGather 000000014002b7c0     ioctl.obj
 0002:000017d4       $chain$1$BuildRawScatterGather 000000014002b7d4     ioctl.obj
 0002:000017ec       $chain$2$BuildRawScatterGather 000000014002b7ec     ioctl.obj
 0002:00001800       $unwind$BuildRawScatterGather64 000000014002b800     ioctl.obj
 0002:0000181c       $unwind$CSMIGetRAIDConfig  000000014002b81c     ioctl.obj
 0002:00001834       $chain$0$CSMIGetRAIDConfig 000000014002b834     ioctl.obj
 0002:0000184c       $chain$1$CSMIGetRAIDConfig 000000014002b84c     ioctl.obj
 0002:00001860       $unwind$CSMIGetRAIDInfo    000000014002b860     ioctl.obj
 0002:00001880       $unwind$CSMISTPPassThru    000000014002b880     ioctl.obj
 0002:00001898       $chain$0$CSMISTPPassThru   000000014002b898     ioctl.obj
 0002:000018ac       $chain$1$CSMISTPPassThru   000000014002b8ac     ioctl.obj
 0002:000018c4       $unwind$HandleCSMI         000000014002b8c4     ioctl.obj
 0002:000018e8       $unwind$QueueEvent         000000014002b8e8     comm.obj
 0002:00001900       $unwind$AdapterIsAlive     000000014002b900     comm.obj
 0002:0000190c       $unwind$ServiceHostResponseNormalQueue 000000014002b90c     comm.obj
 0002:00001914       $chain$6$ServiceHostResponseNormalQueue 000000014002b914     comm.obj
 0002:00001940       $chain$7$ServiceHostResponseNormalQueue 000000014002b940     comm.obj
 0002:00001954       $unwind$FreeConsumerProducerAif 000000014002b954     comm.obj
 0002:00001954       $unwind$CompleteBufferedRequest 000000014002b954     comm.obj
 0002:00001968       $chain$0$FreeConsumerProducerAif 000000014002b968     comm.obj
 0002:0000197c       $chain$1$FreeConsumerProducerAif 000000014002b97c     comm.obj
 0002:00001990       $unwind$ProcessAif         000000014002b990     comm.obj
 0002:000019a8       $chain$0$CompleteBufferedRequest 000000014002b9a8     comm.obj
 0002:000019bc       $chain$1$CompleteBufferedRequest 000000014002b9bc     comm.obj
 0002:000019d0       $unwind$ServiceHostCommandNormalQueue 000000014002b9d0     comm.obj
 0002:000019d8       $chain$3$ServiceHostCommandNormalQueue 000000014002b9d8     comm.obj
 0002:000019f8       $chain$4$ServiceHostCommandNormalQueue 000000014002b9f8     comm.obj
 0002:00001a0c       $unwind$DpcDequeueRawIoReadWriteRequest 000000014002ba0c     comm.obj
 0002:00001a18       $unwind$ProcessNormalFib   000000014002ba18     comm.obj
 0002:00001a24       $chain$3$ProcessNormalFib  000000014002ba24     comm.obj
 0002:00001a44       $chain$5$ProcessNormalFib  000000014002ba44     comm.obj
 0002:00001a5c       $chain$6$ProcessNormalFib  000000014002ba5c     comm.obj
 0002:00001a6c       $chain$7$ProcessNormalFib  000000014002ba6c     comm.obj
 0002:00001a80       $chain$8$ProcessNormalFib  000000014002ba80     comm.obj
 0002:00001aa8       $unwind$ServiceInternalAifQueue 000000014002baa8     comm.obj
 0002:00001abc       $unwind$ProcessHbaErrors   000000014002babc     comm.obj
 0002:00001ad8       $chain$3$ProcessHbaErrors  000000014002bad8     comm.obj
 0002:00001af8       $chain$4$ProcessHbaErrors  000000014002baf8     comm.obj
 0002:00001b14       $unwind$ProcessWmi         000000014002bb14     wmi.obj
 0002:00001b24       $unwind$HwScsiWmiFunctionControl 000000014002bb24     wmi.obj
 0002:00001b24       $unwind$__GSHandlerCheck   000000014002bb24     ntoskrnl:gshandler.obj
 0002:00001b24       $unwind$HwScsiWmiQueryDataBlock 000000014002bb24     wmi.obj
 0002:00001b24       $unwind$__GSHandlerCheckCommon 000000014002bb24     ntoskrnl:gshandler.obj
 0002:00001b30       $xdatasym                  000000014002bb30     BufferOverflowFastFailK:amdsecgs.obj
 0002:00001b38       $xdatasym                  000000014002bb38     BufferOverflowFastFailK:guard_dispatch.obj
 0002:00001b40       $xdatasym                  000000014002bb40     ntoskrnl:memcpy.obj
 0002:00001b48       $xdatasym                  000000014002bb48     ntoskrnl:memset.obj
 0002:00001b4c       $unwind$ScsiPortWmiDispatchFunction 000000014002bb4c     scsiwmi:wmilib.obj
 0002:00001b5c       $unwind$ScsiWmipProcessRequest 000000014002bb5c     scsiwmi:wmilib.obj
 0002:00001b7c       $unwind$ScsiWmipPostProcess 000000014002bb7c     scsiwmi:wmilib.obj
 0002:00001b90       $unwind$ScsiWmipFindGuid   000000014002bb90     scsiwmi:wmilib.obj
 0003:0000000c       ?NeedToReadStatus@?1??CheckingFWAfterPowerStateChange@@9@9 000000014002c00c     timer.obj
 0003:0000000d       ?NeedToCheckMSIX@?1??CheckingFWAfterPowerStateChange@@9@9 000000014002c00d     timer.obj
 0003:00000aa0       ?CalledCnt@?1??CheckForDupHandles@@9@9 000000014002caa0     rxdevice.obj
 0003:00000aa8       ?CalledCnt@?1??CheckFWPulseInCrashDumpMode@@9@9 000000014002caa8     timer.obj
 0003:00000aac       ?TimerAge@?1??CheckingFWAfterPowerStateChange@@9@9 000000014002caac     timer.obj
 0003:00000ab0       ?status@?1??CheckingFWAfterPowerStateChange@@9@9 000000014002cab0     timer.obj
 0003:00000ab4       ?DelayCnt4DualFWFlushSoftReset@?1??CheckingFWAfterPowerStateChange@@9@9 000000014002cab4     timer.obj
 0003:00000ab8       ?pSavedDevExt@?1??CheckingFWAfterPowerStateChange@@9@9 000000014002cab8     timer.obj
 0003:00000ac0       ?TimerAge@?1??Reset_IOP_CompletionTimer@@9@9 000000014002cac0     timer.obj
 0003:00000ae8       ?NewScanStarted@?1??ConfigureContainersRuntime@@9@9 000000014002cae8     arcinit.obj
 0003:00000ae9       ?LoopCount@?1??ConfigureContainersRuntime@@9@9 000000014002cae9     arcinit.obj
 0003:00000aea       ?busChange@?1??ConfigureContainersRuntime@@9@9 000000014002caea     arcinit.obj
 0003:00000aeb       ?initialized@?1??DriverEntry@@9@9 000000014002caeb     arcinit.obj
 0003:00000aec       ?containerCount@?1??ConfigureContainersRuntime@@9@9 000000014002caec     arcinit.obj
 0003:00000af0       ?diskInfoResponse@?1??ConfigureContainersRuntime@@9@9 000000014002caf0     arcinit.obj
 0003:00000b58       ?pSavedDevExt@?1??ConfigureContainersRuntime@@9@9 000000014002cb58     arcinit.obj
 0003:00000b60       ?SkipSecondSynchCmd@?1??ConfigureContainersRuntime@@9@9 000000014002cb60     arcinit.obj
 0003:00000b64       ?ShutdownSent@?1??BuildIo@@9@9 000000014002cb64     cmdproc.obj
 0004:00000000       $pdata$RxCheckAdapterHealth 000000014002d000     rxdevice.obj
 0004:0000000c       $pdata$RxNewCommProcessInterrupt 000000014002d00c     rxdevice.obj
 0004:00000018       $pdata$0$RxNewCommProcessInterrupt 000000014002d018     rxdevice.obj
 0004:00000024       $pdata$3$RxNewCommProcessInterrupt 000000014002d024     rxdevice.obj
 0004:00000030       $pdata$4$RxNewCommProcessInterrupt 000000014002d030     rxdevice.obj
 0004:0000003c       $pdata$5$RxNewCommProcessInterrupt 000000014002d03c     rxdevice.obj
 0004:00000048       $pdata$6$RxNewCommProcessInterrupt 000000014002d048     rxdevice.obj
 0004:00000054       $pdata$7$RxNewCommProcessInterrupt 000000014002d054     rxdevice.obj
 0004:00000060       $pdata$RxInterruptHandler  000000014002d060     rxdevice.obj
 0004:0000006c       $pdata$0$RxInterruptHandler 000000014002d06c     rxdevice.obj
 0004:00000078       $pdata$2$RxInterruptHandler 000000014002d078     rxdevice.obj
 0004:00000084       $pdata$4$RxInterruptHandler 000000014002d084     rxdevice.obj
 0004:00000090       $pdata$6$RxInterruptHandler 000000014002d090     rxdevice.obj
 0004:0000009c       $pdata$8$RxInterruptHandler 000000014002d09c     rxdevice.obj
 0004:000000a8       $pdata$9$RxInterruptHandler 000000014002d0a8     rxdevice.obj
 0004:000000b4       $pdata$NonMSIXInterruptHandler 000000014002d0b4     rxdevice.obj
 0004:000000c0       $pdata$3$NonMSIXInterruptHandler 000000014002d0c0     rxdevice.obj
 0004:000000cc       $pdata$4$NonMSIXInterruptHandler 000000014002d0cc     rxdevice.obj
 0004:000000d8       $pdata$PMCDpcResponseHandler 000000014002d0d8     rxdevice.obj
 0004:000000e4       $pdata$5$PMCDpcResponseHandler 000000014002d0e4     rxdevice.obj
 0004:000000f0       $pdata$6$PMCDpcResponseHandler 000000014002d0f0     rxdevice.obj
 0004:000000fc       $pdata$8$PMCDpcResponseHandler 000000014002d0fc     rxdevice.obj
 0004:00000108       $pdata$9$PMCDpcResponseHandler 000000014002d108     rxdevice.obj
 0004:00000114       $pdata$PMCInterruptHandler 000000014002d114     rxdevice.obj
 0004:00000120       $pdata$2$PMCInterruptHandler 000000014002d120     rxdevice.obj
 0004:0000012c       $pdata$3$PMCInterruptHandler 000000014002d12c     rxdevice.obj
 0004:00000138       $pdata$RxPullMessageUnitQueueCompletedFib 000000014002d138     rxdevice.obj
 0004:00000144       $pdata$1$RxPullMessageUnitQueueCompletedFib 000000014002d144     rxdevice.obj
 0004:00000150       $pdata$2$RxPullMessageUnitQueueCompletedFib 000000014002d150     rxdevice.obj
 0004:0000015c       $pdata$RxPushMessageUnitQueueFib 000000014002d15c     rxdevice.obj
 0004:00000168       $pdata$0$RxPushMessageUnitQueueFib 000000014002d168     rxdevice.obj
 0004:00000174       $pdata$1$RxPushMessageUnitQueueFib 000000014002d174     rxdevice.obj
 0004:00000180       $pdata$PMCPushMessageUnitQueueFib 000000014002d180     rxdevice.obj
 0004:0000018c       $pdata$0$PMCPushMessageUnitQueueFib 000000014002d18c     rxdevice.obj
 0004:00000198       $pdata$1$PMCPushMessageUnitQueueFib 000000014002d198     rxdevice.obj
 0004:000001a4       $pdata$2$PMCPushMessageUnitQueueFib 000000014002d1a4     rxdevice.obj
 0004:000001b0       $pdata$RxSendSynchCommand  000000014002d1b0     rxdevice.obj
 0004:000001bc       $pdata$RxStartAdapter      000000014002d1bc     rxdevice.obj
 0004:000001c8       $pdata$RxWaitForAdapterToBoot 000000014002d1c8     rxdevice.obj
 0004:000001d4       $pdata$0$RxWaitForAdapterToBoot 000000014002d1d4     rxdevice.obj
 0004:000001e0       $pdata$1$RxWaitForAdapterToBoot 000000014002d1e0     rxdevice.obj
 0004:000001ec       $pdata$DumpHandles         000000014002d1ec     rxdevice.obj
 0004:000001f8       $pdata$DumpHandlesZeroPointer 000000014002d1f8     rxdevice.obj
 0004:00000204       $pdata$RevCheckCompatibility 000000014002d204     revision.obj
 0004:00000210       $pdata$GetDriverParameter  000000014002d210     helpers.obj
 0004:0000021c       $pdata$MatchRegistryString 000000014002d21c     helpers.obj
 0004:00000228       $pdata$LongToAscii         000000014002d228     helpers.obj
 0004:00000234       $pdata$0$LongToAscii       000000014002d234     helpers.obj
 0004:00000240       $pdata$1$LongToAscii       000000014002d240     helpers.obj
 0004:0000024c       $pdata$CompareStrings      000000014002d24c     helpers.obj
 0004:00000258       $pdata$StorWmiTraceMessage 000000014002d258     arcdebug.obj
 0004:00000264       $pdata$ArcPrintf           000000014002d264     arcdebug.obj
 0004:00000270       $pdata$1$ArcPrintf         000000014002d270     arcdebug.obj
 0004:0000027c       $pdata$2$ArcPrintf         000000014002d27c     arcdebug.obj
 0004:00000288       $pdata$3$ArcPrintf         000000014002d288     arcdebug.obj
 0004:00000294       $pdata$4$ArcPrintf         000000014002d294     arcdebug.obj
 0004:000002a0       $pdata$5$ArcPrintf         000000014002d2a0     arcdebug.obj
 0004:000002ac       $pdata$6$ArcPrintf         000000014002d2ac     arcdebug.obj
 0004:000002b8       $pdata$WPP_SF_s            000000014002d2b8     arcdebug.obj
 0004:000002c4       $pdata$RealSprintf         000000014002d2c4     arcdebug.obj
 0004:000002d0       $pdata$1$RealSprintf       000000014002d2d0     arcdebug.obj
 0004:000002dc       $pdata$6$RealSprintf       000000014002d2dc     arcdebug.obj
 0004:000002e8       $pdata$7$RealSprintf       000000014002d2e8     arcdebug.obj
 0004:000002f4       $pdata$8$RealSprintf       000000014002d2f4     arcdebug.obj
 0004:00000300       $pdata$MainTimeThread      000000014002d300     timer.obj
 0004:0000030c       $pdata$4$MainTimeThread    000000014002d30c     timer.obj
 0004:00000318       $pdata$5$MainTimeThread    000000014002d318     timer.obj
 0004:00000324       $pdata$6$MainTimeThread    000000014002d324     timer.obj
 0004:00000330       $pdata$7$MainTimeThread    000000014002d330     timer.obj
 0004:0000033c       $pdata$8$MainTimeThread    000000014002d33c     timer.obj
 0004:00000348       $pdata$9$MainTimeThread    000000014002d348     timer.obj
 0004:00000354       $pdata$VMCloseAllCompletionTimer 000000014002d354     timer.obj
 0004:00000360       $pdata$0$VMCloseAllCompletionTimer 000000014002d360     timer.obj
 0004:0000036c       $pdata$1$VMCloseAllCompletionTimer 000000014002d36c     timer.obj
 0004:00000378       $pdata$UpdateThorHBAMappingTable 000000014002d378     timer.obj
 0004:00000384       $pdata$0$UpdateThorHBAMappingTable 000000014002d384     timer.obj
 0004:00000390       $pdata$2$UpdateThorHBAMappingTable 000000014002d390     timer.obj
 0004:0000039c       $pdata$3$UpdateThorHBAMappingTable 000000014002d39c     timer.obj
 0004:000003a8       $pdata$4$UpdateThorHBAMappingTable 000000014002d3a8     timer.obj
 0004:000003b4       $pdata$Reset_IOP_CompletionTimer 000000014002d3b4     timer.obj
 0004:000003c0       $pdata$0$Reset_IOP_CompletionTimer 000000014002d3c0     timer.obj
 0004:000003cc       $pdata$2$Reset_IOP_CompletionTimer 000000014002d3cc     timer.obj
 0004:000003d8       $pdata$4$Reset_IOP_CompletionTimer 000000014002d3d8     timer.obj
 0004:000003e4       $pdata$5$Reset_IOP_CompletionTimer 000000014002d3e4     timer.obj
 0004:000003f0       $pdata$StopTimer           000000014002d3f0     timer.obj
 0004:000003fc       $pdata$RequestTimer        000000014002d3fc     timer.obj
 0004:00000408       $pdata$CheckingFWAfterPowerStateChange 000000014002d408     timer.obj
 0004:00000414       $pdata$0$CheckingFWAfterPowerStateChange 000000014002d414     timer.obj
 0004:00000420       $pdata$3$CheckingFWAfterPowerStateChange 000000014002d420     timer.obj
 0004:0000042c       $pdata$4$CheckingFWAfterPowerStateChange 000000014002d42c     timer.obj
 0004:00000438       $pdata$DriverEntry         000000014002d438     arcinit.obj
 0004:00000444       $pdata$0$DriverEntry       000000014002d444     arcinit.obj
 0004:00000450       $pdata$1$DriverEntry       000000014002d450     arcinit.obj
 0004:0000045c       $pdata$HwInitializeAdapter 000000014002d45c     arcinit.obj
 0004:00000468       $pdata$FindAdapter         000000014002d468     arcinit.obj
 0004:00000474       $pdata$1$FindAdapter       000000014002d474     arcinit.obj
 0004:00000480       $pdata$2$FindAdapter       000000014002d480     arcinit.obj
 0004:0000048c       $pdata$ResetAdapter        000000014002d48c     arcinit.obj
 0004:00000498       $pdata$5$ResetAdapter      000000014002d498     arcinit.obj
 0004:000004a4       $pdata$6$ResetAdapter      000000014002d4a4     arcinit.obj
 0004:000004b0       $pdata$SMNormalModeInitAdapter 000000014002d4b0     arcinit.obj
 0004:000004bc       $pdata$1$SMNormalModeInitAdapter 000000014002d4bc     arcinit.obj
 0004:000004c8       $pdata$2$SMNormalModeInitAdapter 000000014002d4c8     arcinit.obj
 0004:000004d4       $pdata$InitializeDPCs      000000014002d4d4     arcinit.obj
 0004:000004e0       $pdata$1$InitializeDPCs    000000014002d4e0     arcinit.obj
 0004:000004ec       $pdata$2$InitializeDPCs    000000014002d4ec     arcinit.obj
 0004:000004f8       $pdata$ReturningLocalOutstandingRequestsToOS 000000014002d4f8     arcinit.obj
 0004:00000504       $pdata$CleanHostSideRRQ    000000014002d504     arcinit.obj
 0004:00000510       $pdata$EventTracingCleanup 000000014002d510     arcinit.obj
 0004:0000051c       $pdata$AllocateConsumerProducerCommArea 000000014002d51c     arcinit.obj
 0004:00000528       $pdata$AllocateMessageUnitQueueCommArea 000000014002d528     arcinit.obj
 0004:00000534       $pdata$ConfigureContainersRuntime 000000014002d534     arcinit.obj
 0004:00000540       $pdata$0$ConfigureContainersRuntime 000000014002d540     arcinit.obj
 0004:0000054c       $pdata$1$ConfigureContainersRuntime 000000014002d54c     arcinit.obj
 0004:00000558       $pdata$SendEvent2OSDelayed 000000014002d558     arcinit.obj
 0004:00000564       $pdata$GetElapsedSeconds   000000014002d564     arcinit.obj
 0004:00000570       $pdata$IsAdapterReadyForConfigCommand 000000014002d570     arcinit.obj
 0004:0000057c       $pdata$CheckMSIxPossibility 000000014002d57c     arcinit.obj
 0004:00000588       $pdata$0$CheckMSIxPossibility 000000014002d588     arcinit.obj
 0004:00000594       $pdata$1$CheckMSIxPossibility 000000014002d594     arcinit.obj
 0004:000005a0       $pdata$2$CheckMSIxPossibility 000000014002d5a0     arcinit.obj
 0004:000005ac       $pdata$3$CheckMSIxPossibility 000000014002d5ac     arcinit.obj
 0004:000005b8       $pdata$HandleAdapterConfigIssues 000000014002d5b8     arcinit.obj
 0004:000005c4       $pdata$SendInitStructure   000000014002d5c4     arcinit.obj
 0004:000005d0       $pdata$HandleAdapterGetConfig 000000014002d5d0     arcinit.obj
 0004:000005dc       $pdata$HandleAdapterCommitConfig 000000014002d5dc     arcinit.obj
 0004:000005e8       $pdata$InitializeConsumerProducerCommRegion 000000014002d5e8     arcinit.obj
 0004:000005f4       $pdata$MapDeviceBase       000000014002d5f4     arcinit.obj
 0004:00000600       $pdata$IOPReset            000000014002d600     arcinit.obj
 0004:0000060c       $pdata$HWSoftReset         000000014002d60c     arcinit.obj
 0004:00000618       $pdata$DumpFibsSentToFW60SecondsBefore 000000014002d618     arcinit.obj
 0004:00000624       $pdata$4$DumpFibsSentToFW60SecondsBefore 000000014002d624     arcinit.obj
 0004:00000630       $pdata$5$DumpFibsSentToFW60SecondsBefore 000000014002d630     arcinit.obj
 0004:0000063c       $pdata$ReturningOutstandingSentToFWBeforeIOPResetToOS 000000014002d63c     arcinit.obj
 0004:00000648       $pdata$3$ReturningOutstandingSentToFWBeforeIOPResetToOS 000000014002d648     arcinit.obj
 0004:00000654       $pdata$4$ReturningOutstandingSentToFWBeforeIOPResetToOS 000000014002d654     arcinit.obj
 0004:00000660       $pdata$5$ReturningOutstandingSentToFWBeforeIOPResetToOS 000000014002d660     arcinit.obj
 0004:0000066c       $pdata$6$ReturningOutstandingSentToFWBeforeIOPResetToOS 000000014002d66c     arcinit.obj
 0004:00000678       $pdata$ReturnOutstandingFibOnTargetDevice 000000014002d678     arcinit.obj
 0004:00000684       $pdata$2$ReturnOutstandingFibOnTargetDevice 000000014002d684     arcinit.obj
 0004:00000690       $pdata$3$ReturnOutstandingFibOnTargetDevice 000000014002d690     arcinit.obj
 0004:0000069c       $pdata$4$ReturnOutstandingFibOnTargetDevice 000000014002d69c     arcinit.obj
 0004:000006a8       $pdata$5$ReturnOutstandingFibOnTargetDevice 000000014002d6a8     arcinit.obj
 0004:000006b4       $pdata$SetFwTime           000000014002d6b4     arcinit.obj
 0004:000006c0       $pdata$0$SetFwTime         000000014002d6c0     arcinit.obj
 0004:000006cc       $pdata$4$SetFwTime         000000014002d6cc     arcinit.obj
 0004:000006d8       $pdata$5$SetFwTime         000000014002d6d8     arcinit.obj
 0004:000006e4       $pdata$6$SetFwTime         000000014002d6e4     arcinit.obj
 0004:000006f0       $pdata$7$SetFwTime         000000014002d6f0     arcinit.obj
 0004:000006fc       $pdata$SetArcsasFwTime     000000014002d6fc     arcinit.obj
 0004:00000708       $pdata$SetPciSlotNumber    000000014002d708     arcinit.obj
 0004:00000714       $pdata$SendWellnessCmnd    000000014002d714     arcinit.obj
 0004:00000720       $pdata$GetThorHbaPhyDevInfo 000000014002d720     arcinit.obj
 0004:0000072c       $pdata$ArcLogEventString   000000014002d72c     arcinit.obj
 0004:00000738       $pdata$LogSystemEvent      000000014002d738     arcinit.obj
 0004:00000744       $pdata$SendEvent2OS        000000014002d744     arcinit.obj
 0004:00000750       $pdata$WppTraceCallback    000000014002d750     arcinit.obj
 0004:0000075c       $pdata$0$WppTraceCallback  000000014002d75c     arcinit.obj
 0004:00000768       $pdata$1$WppTraceCallback  000000014002d768     arcinit.obj
 0004:00000774       $pdata$DynamicallyThrottleLunQueueDepth 000000014002d774     arcinit.obj
 0004:00000780       $pdata$SA4StatusBatching   000000014002d780     arcinit.obj
 0004:0000078c       $pdata$SA4ACI2Interface    000000014002d78c     arcinit.obj
 0004:00000798       $pdata$SMCrashDumpModeInitAdapter 000000014002d798     arcinit.obj
 0004:000007a4       $pdata$SendEvent2OSChild   000000014002d7a4     arcinit.obj
 0004:000007b0       $pdata$StartIo             000000014002d7b0     cmddelivery.obj
 0004:000007bc       $pdata$0$StartIo           000000014002d7bc     cmddelivery.obj
 0004:000007c8       $pdata$1$StartIo           000000014002d7c8     cmddelivery.obj
 0004:000007d4       $pdata$PostProcessScsiCommand 000000014002d7d4     cmddelivery.obj
 0004:000007e0       $pdata$SendFib             000000014002d7e0     cmddelivery.obj
 0004:000007ec       $pdata$HandleMSIXInterrupt 000000014002d7ec     cmddelivery.obj
 0004:000007f8       $pdata$QueueRawIoReadWriteRequest 000000014002d7f8     cmddelivery.obj
 0004:00000804       $pdata$0$QueueRawIoReadWriteRequest 000000014002d804     cmddelivery.obj
 0004:00000810       $pdata$1$QueueRawIoReadWriteRequest 000000014002d810     cmddelivery.obj
 0004:0000081c       $pdata$CompleteQueuedRequest 000000014002d81c     cmddelivery.obj
 0004:00000828       $pdata$DequeueRawIoReadWriteRequest 000000014002d828     cmddelivery.obj
 0004:00000834       $pdata$0$DequeueRawIoReadWriteRequest 000000014002d834     cmddelivery.obj
 0004:00000840       $pdata$1$DequeueRawIoReadWriteRequest 000000014002d840     cmddelivery.obj
 0004:0000084c       $pdata$ProcessContainerInquiry 000000014002d84c     cmddelivery.obj
 0004:00000858       $pdata$ProcessScsiCommand  000000014002d858     cmddelivery.obj
 0004:00000864       $pdata$QueuePrintf         000000014002d864     cmddelivery.obj
 0004:00000870       $pdata$SendRawIoFib        000000014002d870     cmddelivery.obj
 0004:0000087c       $pdata$2$SendRawIoFib      000000014002d87c     cmddelivery.obj
 0004:00000888       $pdata$4$SendRawIoFib      000000014002d888     cmddelivery.obj
 0004:00000894       $pdata$5$SendRawIoFib      000000014002d894     cmddelivery.obj
 0004:000008a0       $pdata$SendSynchFib        000000014002d8a0     cmddelivery.obj
 0004:000008ac       $pdata$0$SendSynchFib      000000014002d8ac     cmddelivery.obj
 0004:000008b8       $pdata$1$SendSynchFib      000000014002d8b8     cmddelivery.obj
 0004:000008c4       $pdata$DequeueCertainLD    000000014002d8c4     cmddelivery.obj
 0004:000008d0       $pdata$0$DequeueCertainLD  000000014002d8d0     cmddelivery.obj
 0004:000008dc       $pdata$1$DequeueCertainLD  000000014002d8dc     cmddelivery.obj
 0004:000008e8       $pdata$PollSmartHBAFIBCompletion 000000014002d8e8     cmddelivery.obj
 0004:000008f4       $pdata$AdapterControl      000000014002d8f4     cmdproc.obj
 0004:00000900       $pdata$BuildIo             000000014002d900     cmdproc.obj
 0004:0000090c       $pdata$BuildHBAFib         000000014002d90c     cmdproc.obj
 0004:00000918       $pdata$BuildRawIoFib       000000014002d918     cmdproc.obj
 0004:00000924       $pdata$BuildRawIoScatterGather 000000014002d924     cmdproc.obj
 0004:00000930       $pdata$0$BuildRawIoScatterGather 000000014002d930     cmdproc.obj
 0004:0000093c       $pdata$1$BuildRawIoScatterGather 000000014002d93c     cmdproc.obj
 0004:00000948       $pdata$2$BuildRawIoScatterGather 000000014002d948     cmdproc.obj
 0004:00000954       $pdata$3$BuildRawIoScatterGather 000000014002d954     cmdproc.obj
 0004:00000960       $pdata$BuildRawIo2ScatterGather 000000014002d960     cmdproc.obj
 0004:0000096c       $pdata$ConvertRawIo2ScatterGather 000000014002d96c     cmdproc.obj
 0004:00000978       $pdata$1$ConvertRawIo2ScatterGather 000000014002d978     cmdproc.obj
 0004:00000984       $pdata$3$ConvertRawIo2ScatterGather 000000014002d984     cmdproc.obj
 0004:00000990       $pdata$4$ConvertRawIo2ScatterGather 000000014002d990     cmdproc.obj
 0004:0000099c       $pdata$5$ConvertRawIo2ScatterGather 000000014002d99c     cmdproc.obj
 0004:000009a8       $pdata$BuildReadWriteFib   000000014002d9a8     cmdproc.obj
 0004:000009b4       $pdata$BuildScatterGather  000000014002d9b4     cmdproc.obj
 0004:000009c0       $pdata$BuildScatterGather64 000000014002d9c0     cmdproc.obj
 0004:000009cc       $pdata$BuildRawIo2ScatterGather4HBAIoctl 000000014002d9cc     cmdproc.obj
 0004:000009d8       $pdata$BuildHBAIoctlFib    000000014002d9d8     cmdproc.obj
 0004:000009e4       $pdata$BuildSrbFib         000000014002d9e4     cmdproc.obj
 0004:000009f0       $pdata$InitializeFib       000000014002d9f0     cmdproc.obj
 0004:000009fc       $pdata$PrepareBMIC15       000000014002d9fc     cmdproc.obj
 0004:00000a08       $pdata$ProcessIoctl        000000014002da08     ioctl.obj
 0004:00000a14       $pdata$BuildRawScatterGather 000000014002da14     ioctl.obj
 0004:00000a20       $pdata$1$BuildRawScatterGather 000000014002da20     ioctl.obj
 0004:00000a2c       $pdata$2$BuildRawScatterGather 000000014002da2c     ioctl.obj
 0004:00000a38       $pdata$BuildRawScatterGather64 000000014002da38     ioctl.obj
 0004:00000a44       $pdata$CSMIGetRAIDConfig   000000014002da44     ioctl.obj
 0004:00000a50       $pdata$0$CSMIGetRAIDConfig 000000014002da50     ioctl.obj
 0004:00000a5c       $pdata$1$CSMIGetRAIDConfig 000000014002da5c     ioctl.obj
 0004:00000a68       $pdata$CSMIGetRAIDInfo     000000014002da68     ioctl.obj
 0004:00000a74       $pdata$CSMISTPPassThru     000000014002da74     ioctl.obj
 0004:00000a80       $pdata$0$CSMISTPPassThru   000000014002da80     ioctl.obj
 0004:00000a8c       $pdata$1$CSMISTPPassThru   000000014002da8c     ioctl.obj
 0004:00000a98       $pdata$HandleCSMI          000000014002da98     ioctl.obj
 0004:00000aa4       $pdata$QueueEvent          000000014002daa4     comm.obj
 0004:00000ab0       $pdata$AdapterIsAlive      000000014002dab0     comm.obj
 0004:00000abc       $pdata$ServiceHostResponseNormalQueue 000000014002dabc     comm.obj
 0004:00000ac8       $pdata$6$ServiceHostResponseNormalQueue 000000014002dac8     comm.obj
 0004:00000ad4       $pdata$7$ServiceHostResponseNormalQueue 000000014002dad4     comm.obj
 0004:00000ae0       $pdata$FreeConsumerProducerAif 000000014002dae0     comm.obj
 0004:00000aec       $pdata$0$FreeConsumerProducerAif 000000014002daec     comm.obj
 0004:00000af8       $pdata$1$FreeConsumerProducerAif 000000014002daf8     comm.obj
 0004:00000b04       $pdata$ProcessAif          000000014002db04     comm.obj
 0004:00000b10       $pdata$SendConsumerProducerFib 000000014002db10     comm.obj
 0004:00000b1c       $pdata$CompleteBufferedRequest 000000014002db1c     comm.obj
 0004:00000b28       $pdata$0$CompleteBufferedRequest 000000014002db28     comm.obj
 0004:00000b34       $pdata$1$CompleteBufferedRequest 000000014002db34     comm.obj
 0004:00000b40       $pdata$ServiceHostCommandNormalQueue 000000014002db40     comm.obj
 0004:00000b4c       $pdata$3$ServiceHostCommandNormalQueue 000000014002db4c     comm.obj
 0004:00000b58       $pdata$4$ServiceHostCommandNormalQueue 000000014002db58     comm.obj
 0004:00000b64       $pdata$DpcDequeueRawIoReadWriteRequest 000000014002db64     comm.obj
 0004:00000b70       $pdata$ProcessNormalFib    000000014002db70     comm.obj
 0004:00000b7c       $pdata$3$ProcessNormalFib  000000014002db7c     comm.obj
 0004:00000b88       $pdata$5$ProcessNormalFib  000000014002db88     comm.obj
 0004:00000b94       $pdata$6$ProcessNormalFib  000000014002db94     comm.obj
 0004:00000ba0       $pdata$7$ProcessNormalFib  000000014002dba0     comm.obj
 0004:00000bac       $pdata$8$ProcessNormalFib  000000014002dbac     comm.obj
 0004:00000bb8       $pdata$ServiceInternalAifQueue 000000014002dbb8     comm.obj
 0004:00000bc4       $pdata$ProcessHbaErrors    000000014002dbc4     comm.obj
 0004:00000bd0       $pdata$3$ProcessHbaErrors  000000014002dbd0     comm.obj
 0004:00000bdc       $pdata$4$ProcessHbaErrors  000000014002dbdc     comm.obj
 0004:00000be8       $pdata$ProcessWmi          000000014002dbe8     wmi.obj
 0004:00000bf4       $pdata$HwScsiWmiExecuteMethod 000000014002dbf4     wmi.obj
 0004:00000c00       $pdata$HwScsiWmiQueryDataBlock 000000014002dc00     wmi.obj
 0004:00000c00       $pdata$HwScsiWmiFunctionControl 000000014002dc00     wmi.obj
 0004:00000c0c       $pdata$GsDriverEntry       000000014002dc0c     BufferOverflowFastFailK:gs_driverentry.obj
 0004:00000c30       $pdata$__GSHandlerCheckCommon 000000014002dc30     ntoskrnl:gshandler.obj
 0004:00000c3c       $pdata$__GSHandlerCheck    000000014002dc3c     ntoskrnl:gshandler.obj
 0004:00000c60       $pdata$ScsiPortWmiDispatchFunction 000000014002dc60     scsiwmi:wmilib.obj
 0004:00000c6c       $pdata$ScsiWmipProcessRequest 000000014002dc6c     scsiwmi:wmilib.obj
 0004:00000c78       $pdata$ScsiPortWmiPostProcess 000000014002dc78     scsiwmi:wmilib.obj
 0004:00000c84       $pdata$ScsiWmipPostProcess 000000014002dc84     scsiwmi:wmilib.obj
 0004:00000c90       $pdata$ScsiWmipFindGuid    000000014002dc90     scsiwmi:wmilib.obj
 0005:000001a0       .idata$6                   000000014002e1a0     ntoskrnl:ntoskrnl.exe
 0005:000001ca       .idata$6                   000000014002e1ca     hal:HAL.dll
 0005:0000038a       .idata$6                   000000014002e38a     storport:storport.sys
 0006:000000d0       $R000000                   000000014002f0d0     archba.res
 0006:00000420       $R000350                   000000014002f420     archba.res
